:100000000C9477210C94A8210C94A8210C94A8217D
:100010000C94A8210C94A8210C94A8210C94A8213C
:100020000C94A8210C944E460C944E460C944E46CB
:100030000C94A8210C94A8210C94A8210C94A8211C
:100040000C94A8210C94A8210C94A8210C94A8210C
:100050000C94A8210C94A8210C94A8210C94204E57
:100060000C94A8210C9490430C9467430C94A82101
:100070000C94A8210C94A8210C94A8210C94A821DC
:100080000C94A8210C94A8210C94A8210C94A821CC
:100090000C94A8210C94A8210C94A8210C94C03B8A
:1000A0000C94A8210C94A8210C94A8210C94A821AC
:1000B0000C94A8210C94A8210C94A8210C94A8219C
:1000C0000C94A8210C94A8210C94A8210C94A8218C
:1000D0000C94A8210C94A8210C94A8210C94A8217C
:1000E0000C94A821A74AAB4AB24AA14AB24AA34AF1
:1000F000AF4ABF4AB24AB24AB24AB24AB24AB24A16
:10010000B24AB24AB64AB24AB24AB24AB24AB24A0B
:10011000284C2B4C1A4C1E4C244C624C2F4C334C0C
:10012000394C3D4C414C474C4B4C4F4C624C554C20
:10013000594C5D4C00407A10F35A00A0724E1809D9
:100140000010A5D4E80000E87648170000E40B543E
:10015000020000CA9A3B000000E1F505000080960D
:100160009800000040420F000000A086010000003F
:10017000102700000000E8030000000064000000F9
:1001800000000A00000000000100000000002C76C2
:10019000D888DC674F0823DFC1DFAE59E1B1B796DD
:1001A000E5E3E453C63AE651997696E8E6C284263A
:1001B000EB898C9B62ED407C6FFCEFBC9C9F40F216
:1001C000BAA56FA5F490055A2AF75C936B6CF96792
:1001D0006DC11BFCE0E40D47FEF520E6B500D0ED57
:1001E000902E0300943577050080841E08000020BF
:1001F0004E0A000000C80C333333330F986E12835D
:100200001141EF8D2114893BE65516CFFEE6DB1830
:10021000D1844B381BF77C1D901DA4BBE4242032F5
:1002200084725E228100C9F124ECA1E53D27000023
:1002300000400000000000E0FF0300000000F8FFA5
:100240003F000000003F007C000000800700E0014C
:100250000000E0010080070000F00000000F000037
:10026000380000001C00001CE0011E3800000EF0E9
:10027000000F7000000778000FE00000037880078F
:10028000C00080033C8003C00180013CC0038003A8
:10029000C0001EE0010003C0000EE0010003E0000A
:1002A0000FF0000007608007F0FCFF066080FF7F12
:1002B000FCFF0660C0FF3FFE7F0E30C0FF3FFF3FE8
:1002C0000C30E0011E07000C30F0008E07000C30EF
:1002D000F0008F03000C307800C703000C3038802A
:1002E000C701000C303CC0E301000C601EE0F300CD
:1002F000000E700EE0F1FF000E600FF0F87F0006B8
:10030000E00FF0FC7F0006C00000FC3F0007C000CB
:10031000001E000003C001000E0080038001000FDA
:100320000080018003000700C0010007800300E097
:10033000000006C003006000001EC0010070000045
:100340001CE0010038000078F000001E0000E070A2
:1003500000000F0000C00300C0030000800F00F089
:1003600001000000FE007E00000000F8FF1F0000FA
:10037000000080FF030000000000000000000000FB
:10038000000000000000000000000000BF000303A8
:1003900004040204050B0DFFFE08FE08FE016402C2
:1003A000CF08B7200500E60421088223C5411213B7
:1003B0002208337745442500231077A15524188956
:1003C0009922215324188901240FA59E556C92422D
:1003D0005B8A4852662100251287228E4C220949E9
:1003E000A2E168441489CC240026108722CE4C2236
:1003F00092C866129344329A08270631F7C400283F
:100400000BA31A554412D129240A290DA31A4548D1
:10041000149268894842002A0733364524072B0A7C
:1004200056A6955064128A002C0742DA0445022D24
:1004300006146E05012E0622E204012F0C84225DB3
:10044000522C140BC56200300B85A2CD44C217C9D3
:100450000400310783A34D451F320A85A2CD444DC8
:10046000495B01330D85A2CD444D249451241300E2
:10047000340E86A26550368A4842129B5002350CD3
:1004800085A2C54D461C51241300360D85A2CD44CE
:1004900042A34858241300370B85A2454D492692A4
:1004A0002901380E85A2CD4442914C242C9209009A
:1004B000390D85A2CD44C222A1512413003A07620E
:1004C000E20491003B0882DA049122013C08546660
:1004D00095444D013D0735AA45B5003E0954668552
:1004E0004C4509003F0C85A2CD444DA426878800C9
:1004F00040179ADE5E4D1A0A4922A224492C24098B
:10050000A58424B238AC06410F8722D67026114943
:100510004412C9414613420C86E2454544BA8898C4
:100520002E00430E87221649449C2A4644220A0084
:10053000440B86E20549A2C48B8404450985A2C503
:100540004D76532B460A85A2C54D46916903470E49
:1005500087221649449C8A6A12916812480A86E2E8
:100560008588E930E224490782E2C483004A0A858B
:10057000A29DDE289209004B0F87E28548A2441B0A
:10058000D224221599004C0885A2854CDF0A4D1013
:1005900089A286B466BB58522813528814124E0E94
:1005A000872286AC54A2442811529B004F0C87220C
:1005B000D64CA2C64DA23602500B86E24545C47405
:1005C000112A02510D971ED64CA2C625A28D0E08E7
:1005D000520B86E24545C474113109530C86E20D75
:1005E00045546423492800540986E28549A84F00F0
:1005F000550A86E285889F241400560F8722868C30
:100600002651928824B2E1340657138AE286484480
:100610001291543449940E3191502402580E87227D
:10062000868C26511BCE246A3401590D886286902F
:10063000281169A38AD5005A0A86E28551A6365345
:10064000345B08A31A4545BF0C5C0C8422452C186A
:100650000BC682B1005D08A31AC544BF145E0844EE
:10066000728DA4240A5F06169A8501600722FE4453
:100670002800610B66A2CD2824A2E82411620B8514
:10068000A2854C469170B100630964624D65A41265
:1006900019640A85A29D8A858B8400650C65A2CDAC
:1006A00044729049241300660A8521D5444492E996
:1006B00004670C859A8D64C24542934C00680A8594
:1006C000A2854C4691F022690782E284E8506A0ACA
:1006D000A3D98C50A2170A006B0D86A28550454203
:1006E0009A91244A026C0782E2C483006D0E68620C
:1006F0004644178A8422A148280A6E0965A2454407
:100700008517016F0A65A2CD44C2453201700B8581
:100710009A4544858B452603710A859A8D64C245A6
:1007200042537209642245A422D204730B65A2CD00
:10073000446548914C00740A84218D484211691324
:10074000750965A28584179500760B65A285844599
:1007500092340B01771067228624428950229A2412
:1007600022890400780C66E28548429351442401B2
:10077000790C859A85848B84241389007A0965A273
:10078000454DA4AD007B0BA45A9544A422136913D4
:100790007C07A1DBC461007D0CA45A854CA4261102
:1007A0006911017E0725AE8D1600A00500E604A1A3
:1007B00008821B852C7210A20F859E5D6822998489
:1007C000222189641403A30D85A2D54412119164DA
:1007D0002A1301A40B66A6453042CA89120CA50E45
:1007E00086E245503892842226914904A607A1DB6F
:1007F000048900A70FA59ACD44449B8448911949C8
:100800003201A80713FE442400A91288A3162D184C
:1008100009A9842292A06892182301AA08536FC5DF
:1008200048121BAB0936E68D84229208AC0735EBE3
:10083000453101AD06146E0501AE1488A3162D18BE
:10084000895024A1886424094512632400AF06134B
:10085000FEC400B0073336CD0A00B10B76A2955026
:100860006412CA2106B20843F2CC246500B30843DF
:10087000F2C4243601B40722FE8C0400B50A859A1E
:10088000858497CA4C06B616A69ACD21129944269D
:1008900021492C128BC422B1482C1201B70612EE4A
:1008A0008400B80622DACC00B90742F2CC2401BA9F
:1008B00007536F058536BB0A36E6854424A14800F8
:1008C000BC1388624E2C244B0A86C2A1584816A13C
:1008D000042300BD1187624E2C220BA585A2115165
:1008E0002429D300BE138862C62896188989C2A11C
:1008F000584816A1042300BF0D859A951C2213A900
:1009000049241300C013B722561C10870E6712919A
:100910004424911C643401C112B72266340E1DCEEA
:10092000242289482239C86802C212B7225E3412D2
:1009300007AE49441291447290D104C313B7225EAA
:1009400024168903D7242289482239C86802C41191
:10095000A72256240E5C9388242289E420A309C58B
:1009600013B7225E34128D0E6712914424911C64D9
:100970003401C60F89A2D68928114A2A6A36914CB9
:1009800054C70FA71A1649449C2A464422625406AB
:10099000C80CB5A24D340EB8C96E6A05C90BB5A214
:1009A0005D3AE026BBA915CA0CB5A2552C12BEC9EA
:1009B0006E6A05CB0AA5A24DF24D76532BCC09B237
:1009C000E24428743808CD08B2E28CEC7010CE08EE
:1009D000B3E14C46897ECF0AA4E144282AD22F00F5
:1009E000D01087E10D4D221259942422891209005A
:1009F000D112B7225E2416898364A51225428990FC
:100A0000DA04D210B7225E1C1007CE246ADC246AF6
:100A10002300D30FB72266340E9D49D4B849D4467B
:100A200000D410B7225E341207CE246ADC246A2375
:100A300000D511B7225E241689036712356E12B5F0
:100A40001100D60FA72256240E9C49D4B849D4468B
:100A500000D70B56A685484293514402D8118722ED
:100A6000D624A2A912A1444A1295C80800D90CB6EE
:100A7000E255380E11F1938402DA0CB6E2653A447D
:100A8000C44F120A00DB0DB6E25530128788F849D0
:100A90004201DC0CA6E24D280E10F1938402DD1019
:100AA000B8626E380E141225226D54B11A00DE0C95
:100AB00086E285B02262BA088500DF0C85A2CD44AB
:100AC000B412116D8900E00E96A255380E1A8544B5
:100AD000149D2402E10E96A25D300E1B8544149DE8
:100AE0002402E20F96A2553012078D42228A4E123E
:100AF00001E31096A25524148983462111452789C4
:100B000000E40D86A24D3A68141251749208E50F64
:100B100096A25530120C8E42228A4E1201E60F68C0
:100B2000628E2524911C243289960900E70C845A90
:100B30004D65A41219852400E80E95A24D340E9936
:100B4000480E32896402E90E95A25D3A642239C8E2
:100B500024920900EA0F95A2552C12074C240799FC
:100B6000443201EB0E85A24D3A602239C824920925
:100B700000EC0892E244287428ED0792E28CEC50D5
:100B8000EE0993E24C36895E00EF0A83E2442426A4
:100B9000D10B00F00E95A24D9228129B48B8482622
:100BA00000F10B95A24DEE80880A2F02F20D95A25E
:100BB0004D340E9948B8482600F30C95A25D3A646E
:100BC00022E1229900F40E95A2552C12074C245CC8
:100BD000241300F50C95A24DEE9089848B6402F6E7
:100BE0000C85A24D3A6022E1229900F70A56A6959B
:100BF0001C62878800F80F67A1D524A2549288242C
:100C000092C80800F90B95A24D340E90F0A212FA8A
:100C10000B95A25D3A40C28B4A00FB0B95A2552C66
:100C20001296F0A212FC0A85A24DB284179500FD1F
:100C30000EB59A5D3A40C2454292894400FE0EA527
:100C40009A854C469190562C321900FF0DA59A4D6D
:100C5000B2848B842413890000000000BF000303CA
:100C600005050305061217FFFB0EFC0EFC02280407
:100C7000DD0F02200600309600210AC31596F850B9
:100C8000111E04220AA5349F9070194500231DAB44
:100C900011AE9488256289EC3039CC2462895822BF
:100CA0003B4C0E33895822960801241D0AD2A90D07
:100CB000DB0E915144320A8EA265733564095942A4
:100CC0009343CC1C074501251EAD15C2218A6C2219
:100CD0006D2251D022A5C88171A0842A3186D444C6
:100CE000DA4C420A00261ECD15BAA343CCA3A95064
:100CF0003A9203EAA099CC241A998434E96C56BB41
:100D0000CC6A032708A23493384800280F46969DE2
:100D10001BCD6433D9FE281C0A17291246929D1850
:100D20000E8543E16CBFC966B2D10C002A0FC7140F
:100D3000A78B492292DA4C228A45002B0D0835AE4A
:100D400013AB1D0E32B11A002C0AC3B495384828D3
:100D500021002D0765909A78082E076314963808AD
:100D60002F10C51196D33492298D64A2914C0D0099
:100D7000300FA911AA1B9E266BFE36593ACE0031C0
:100D80000BA615AA1B1D0EB2FD033212A911AAAAA9
:100D90005D66B6F17458AB51970F07023313A91172
:100DA000AAAA5D46939978482D936D26CAAD04345E
:100DB00015A911AA9D126B36C96832124D4693C30C
:100DC000813A5E013515A911AA38440E91F1F874E3
:100DD000888CC8639BE95032013614A911AA321DD0
:100DE00022B3F2647488908C8DA6C9AD043710A923
:100DF00011AA78204F97A7E3E9783A5E053812A93F
:100E000011AAAA5D666E935B6DB2E636B99500399C
:100E100014A911AAAA5D46C64613E5109A8C6B93D5
:100E200043C8043A0A43159A38C8A107013B0CA3EA
:100E3000B59938C8A1070925043C0D2915AE1E96A1
:100E40006AC43980DC3C3D0BA974AE78A0830E07E0
:100E5000023E0E2915AE1837D301435AA938063F72
:100E600011C815AAB11C48A6E190B8BA0E9EAE01F1
:100E7000402B30B6C9BD030E442A690E529B484C24
:100E8000279A484692C9488A243589484D32398C78
:100E90004694E11C810E3EC8414700411ACC15BA68
:100EA000A443E800B3482C928E86A3A1DA7074188C
:100EB0001D2663E701421ACB19BA381E4433CA70A3
:100EC000329CCC4607D16132BC3A1E2E87180043B3
:100ED0001BCC15BAAC1E44B4D1F46A07CD4173D013
:100EE0001C449D4C27B4D9415A034416CC15BA383A
:100EF000040FA321653A19FBEB6448398C0E4100BD
:100F0000451ACA19B6F82007CC0173C01C70901C92
:100F10002473C01C3007CC010F06461CCA15B2F85A
:100F20002007CC0173C01C70901C2473C01C3007B8
:100F3000CC0173C01C00471BCC15BEAC1E44B4D101
:100F4000F46A07CD41B383EC309D4C2734D26166FF
:100F500011480DCC15BA18FBF9F041ECE70149072F
:100F6000C31596F8074A0DC911AADE9F6DB60BE5A9
:100F700056024B1CCD15BA985286A4196D449C504C
:100F8000CF76C079421D1167B421694A19134C0B01
:100F9000C915AE18EF7F3E1C084D21CE15C29843EF
:100FA000EC90F3217C101E8687E121229258441296
:100FB0008B486222994836994D364E1ACC15BA188C
:100FC0005F1F8207994566199944A6894D623C04C2
:100FD0000FD1F3004F1BCD15BE2C1F644CD309F568
:100FE0000EB003EC003BE04A998E68B483B8085019
:100FF00019CB15B638C40E93E1D5E3E17288CD2143
:1010000073C81C3287CC2100511FEDF5BD2C1F6425
:101010004CD309F50EB003EC003BE024A18C4CA4AA
:10102000DA417C88032500521ECC15BA38040FA380
:1010300021653A994E8694C3E8201B8EA693E964F5
:101040003A994EA6045316CB15B6BA1D24B4EB1D1F
:10105000623EDB2157EB8D72909D00541CCB11AE8C
:10106000F8109C43E69039640E9943E69039640E7B
:101070009943E690396408550ECC15BA18FB3F4FDA
:1010800086A3C3D0065621CD11B69803EC80C9744F
:10109000349D4985B3E16C3A194FE600891C5287AB
:1010A000D44173D81400571DCF15C698CD6C33DBCF
:1010B000CCB632DABFA8CC241A251A2BD5D978366B
:1010C0009ECD00581BCC11B2189B27C311A3486CAE
:1010D00007D001669174341B8E8693B17900591F35
:1010E000CD11B69803EC80C974B6389B4EC69339BF
:1010F000A00E9AC3E6B0396C0E9BC3A6005A12CA62
:1011000015B278B003C6EB80F176C0781DF0605B55
:101110000B4596993898F6FF74185C0DC51196909A
:10112000A9CDB4CDD4661A5D0B459299388CF6FFE3
:1011300074305E10EAD0AA9403C854916C34124AF9
:1011400086035F074A90A978306007657097982DED
:1011500061134A15AE2ADE6463DA89B23619512A60
:10116000230A01621ACA15B29803E68039600E9804
:10117000900E12D264E8F1343948262400631149F4
:1011800015AEA31D2223F376C068728891006419FE
:10119000CA15B207CC0173C01C30A24C0E92D1D13B
:1011A000E364443988280365124915AEA39D46C6F9
:1011B000C3831C309A1C622400660EC7119E2395BF
:1011C00086A3C369B89F006719CA95B1A24C0E9255
:1011D000D1D1E3644439882873C064343A04690087
:1011E000680DC915AE18EF4239986CFE36690AC30E
:1011F000159638C80E1F046A0D458E95DA0E18ED47
:101200003F1D2A006B12C915AA18EF3459B2158B6D
:10121000B6C96865741B6C07C31596F8076D184F3F
:1012200015C6989028874389649BD966B6996D66E0
:101230009BD966B6056E0C4915AE98500E269BBF1D
:101240000D6F114A15B2231E422B438F93D1E81024
:10125000A4017019CA95B198900E12D264E8F134C5
:10126000394826A439600E9803E6007119CA95B171
:10127000A24C0E92D1D1E3644439882873C01C304B
:1012800007CC0103720B46159E981C0EB37D0373A9
:10129000104915AE321D68E643EC6C3B904C00746F
:1012A0000DA6119A992D1D2AB3BD9508750B4915E8
:1012B000AE98F9A783853276114911A698B94D9653
:1012C00026A3C9AC581DCF0077194F11BE98CD6C1D
:1012D00033DBCA684B65345199558A34EA6C3C9BC0
:1012E0000178114915AE98D9266BD5696D329AAC43
:1012F000D9067914C995AD98B94D9626A3C9AC58AD
:101300001D2F4BA953007A0C4815AA78900EF77A36
:1013100038087B0D4796A19C2DEEB6BAB8D7057C50
:1013200008429695F843007D0E4792A1982EEEBA9A
:10133000B6B8B745007E0A6994AE211D4C1400A0D2
:101340000600309600A10BC39999380825878702BB
:10135000A219C8D5A98E0362A5C3A81413C5244138
:10136000497026B998E2803000A317AA11AE2B1E4F
:1013700022B3C91C30878CAF73C078F170885400D9
:10138000A4110955AE901E284B32914C34991CA8DB
:1013900002A513A911AA98B94D9626B3D241363B9E
:1013A000C8C6DB00A60A42969578101E0E02A71941
:1013B0004992A9AA5D66B673ED249B088D9299E8BF
:1013C00048BED926B71200A80845949F905004A99A
:1013D00021CE15BE340F6772881A93692453924345
:1013E00044728848181B996834891C221B8E8D0012
:1013F000AA0E26B5A2A1C424279264123E14AB13F0
:101400000A31AE9B8C26A3C968329B0C27C3C970D6
:1014100032AC0DA974AE78A003E400394000AD07EA
:1014200065909A7808AE23CD15BE2C4B657248287E
:10143000628A8444233591D2485414A989D4221154
:1014400099242407C8968B00AF0745949F380CB0A9
:101450000CC6F09EA11C42A4438402B10F2915AE14
:101460001BCF0E07DA780E3D1C08B20D06B19AA10B
:101470001C42B209657628B30E06B19AA11C42A29D
:1014800099E910A100B4086570979A2C01B50DC9AF
:1014900095AD98F9A7C38162DE0CB6254992A9BA29
:1014A00050241549455291542415114536114A844A
:1014B00012A14428114A8412A14428114A2400B7D9
:1014C0000642D49620B80AA5749D910D0F1400B958
:1014D0000904B19A3A8CF400BA0D26B5A2A1883855
:1014E00049E8804301BB140A31AE980C27C3C97088
:1014F000329B8C26A3C9683203BC21AE11BE92CAAE
:10150000A832A2582896C90132914C249A496463A2
:10151000115524918A6C62A15802BD22AF11BE926E
:101520000AA942A21C2094036472884C4213494CBD
:101530001291AA7428A4CAC6429BD000BE1FAE1145
:10154000BEA18A8C2235E9504A128A542416C988D1
:10155000229A03246489B2C428D502BF11C895A970
:101560009BAE83A78B43E292E940B100C01F4C16AB
:10157000BA9AC3E64039063A840E308BC422E96831
:10158000381AAA0D4787D16132761EC1204C16BA8F
:1015900007CC2173881C031D42079845629174345F
:1015A0001C0DD586A3C3E830193B0FC21F4C16BAD9
:1015B0009D43CA9339221D42079845629174341C99
:1015C0000DD586A3C3E830193B0FC31F4C16BA9C38
:1015D000058FB1392A1D42079845629174341C0D5C
:1015E000D586A3C3E830193B0FC4204C16BA138923
:1015F0004562911C950EA103CC22B1483A1A8E8601
:101600006AC3D16174988C9D07C5224C16BAA40395
:101610004462911C4087D02174805924164947C3E5
:10162000D1506D383A8C0E93B1F300C626D015CA4E
:101630003C140F353B4C32074DE6A0C91C243A88B8
:101640004607D13AE410071CE480D91C303BD80E81
:1016500003C7246C76B9AC1E44B4D1F46A07CD41FB
:1016600073D01C449D4C27B4D9415A07C86173A05C
:101670001C50075001C8204A1AB69A43E62039F890
:10168000F02007CC0173C01C70901C2473C01C3068
:1016900007CC010F06C91D4A1AB65E96237C90033B
:1016A000E68039600E38480E9239600E9803E68065
:1016B0000703CA1F4A1AB61C172773E0E1410E98A8
:1016C00003E68039E0203948E68039600E98031E31
:1016D0000CCB204A1AB65214094572E8E1410E9823
:1016E00003E68039E0203948E68039600E98031E11
:1016F0000CCC0C450E96980DE580D1FE1FCD0D4506
:1017000016969A4CE490D1FE9F00CE0D470E969A05
:1017100055D641C3FD3F01CF0D4612961031C90188
:10172000B3FD3F01D01FCE0DBA3A840FC3216D3AED
:101730001B8FC607DA81361A8FC6A3E96C483B0CAB
:101740000F4100D11F4C16BA9C058FB139CAF8FA67
:10175000103CC82C32CBC824324D6C12E32178885F
:101760009E07D2214D16BE9B03E7503996F241C623
:10177000349D50EF003BC00EB003AE94E988463B69
:10178000888B00D3224D16BE07CC4173901C53F9B1
:1017900020639A4EA877801D6007D80157CA744409
:1017A000A31DC44500D4224D16BE9D83EA80C91CEA
:1017B000B97C90314D27D43BC00EB003EC802B6533
:1017C0003AA2D10EE22200D5214D16BE9D45AFB101
:1017D0003972F920639A4EA877801D6007D80157A7
:1017E000CA7444A31DC44500D6234D16BE14C901B6
:1017F00022394024472E1F644CD309F50EB003EC68
:10180000003BE04A998E68B483B808D7100A31AE1D
:10181000184E46332B996A1B4D8603D822CF11BE32
:10182000ADC90E34E2228D2619CD446BB1D14836B4
:101830009A084745DA7448A31D68B22A00D9144CA7
:1018400016BA9BC3E64039D2D8FF79321C1D8636C2
:1018500000DA154C16BA07CC2173881C6DECFF3CDE
:10186000198E0E431B00DB144C16BA9D43CA9339E4
:10187000C2D8FF79321C1D863600DC154C16BA130F
:10188000894562911C65ECFF3C198E0E431B00DDFF
:10189000254D12B607CC4173901C750EB00326D3AC
:1018A000D9E26C3A194FE6803A680E9BC3E6B0392C
:1018B0006C0E9B02DE1BCB15B69843E69039E41004
:1018C0003B4C8657C7C3E5109B43E690390400DFC5
:1018D0000EC815AAA25946BEECE4CB6502E018CAB0
:1018E00015AE9943E6203952F1361AD34E94B5C954
:1018F0008852195108E116CA15AE5E9623156FA3DA
:1019000031ED44599B8C2895118500E217CA15AE1C
:101910001B17277384E26D34A69D286B9311A532A3
:10192000A210E318CA15AE9AC86E92394AF1361A57
:10193000D34E94B5C98852195108E418CA15AE524D
:101940001409457284E26D34A69D286B9311A5326B
:10195000A210E518CA15AEA28A842229B9781B8D77
:101960006927CADA6444A98C2804E6194E15C2A274
:10197000D40E25D16C481B1D2ACBA3F1A474384C7E
:10198000482500E717E975A9A31D2223F376C0684F
:10199000728851E580394458A401E817C915AE99F9
:1019A00003E610390AED34321E1EE480D1E4102320
:1019B00001E915C915AE9E4EE528B4D3C8787890D4
:1019C000034693438C04EA16C915AE9BD6267330A2
:1019D000ED34321E1EE480D1E4102301EB17C9154B
:1019E000AE5213C9447230ED34321E1EE480D1E48D
:1019F000102301EC0CC50D96980DE580D1FE01ED8C
:101A00000DC515969A4CE490D1FE0900EE0DC70D58
:101A1000969A55D641C3FD1300EF0CC5119690B0B0
:101A20008847FB1700F017CA15B291832443AA48D0
:101A30005C3B8456861E27A3D1214803F111C915AA
:101A4000AE9A884E9239704239986CFE36F217CAB7
:101A500015B29943E620391AF1105A197A9C8C462E
:101A600087200D00F314CA15B25E96A3110FA1953D
:101A7000A1C7C9687408D200F416CA15B21B17278B
:101A80007314E221B432F438198D0E411A00F5179F
:101A9000CA15B29AC86E923912F1105A197A9C8CF2
:101AA0004687200D00F617CA15B252140945721464
:101AB000E221B432F438198D0E411A00F70E0935BF
:101AC000AE1BCFA187031D3A9E01F8184C11B2241A
:101AD000890EB2D16C549A982CA3D26C343B8844B2
:101AE0004400F911C915AE9903E6103974E69F0E4A
:101AF00016CA00FA0FC915AE9E4EE5D0997F3A5826
:101B00002803FB10C915AE9BD62673D8CC3F1D2CDD
:101B10009401FC11C915AE5213C94472D8CC3F1DB3
:101B20002C9401FD174996AD5D9583676E93A5C909
:101B300068322B56C7CB52EA1400FE204A96B19861
:101B400003E68039600E98900E12D264E8F13439C1
:101B50004826A439600E9803E600FF194996AD5255
:101B600013C94472D8CC6DB234194D66C5EA7859A0
:101B70004A9D02000000000000000000000000007C
:101B80000000000000000000000000000000000055
:101B90000000000000000000000000000000000045
:101BA0000000000000000000000000000000000035
:101BB0000000000000000000000000000000000025
:101BC0000000000000000000000000000000607045
:101BD00000000000000000000000000000001C8069
:101BE00001000000000000000000000000000300F1
:101BF00007000000000000000000000000C001001D
:101C00000C000000000000000000000000C0010007
:101C100038000000000000000000000000E00000AC
:101C2000380000000000000000000000007000000C
:101C3000F00000000000000000000000003800007C
:101C4000E00000000000000000000000003C000078
:101C5000E00100000000000000000000003C000067
:101C6000E00100000000000000000000003E000055
:101C7000C00300000000000000000000003E000063
:101C8000C00300000000000000000000001E000073
:101C9000C00300000000000000000000001F000062
:101CA000C00700000000000000000000003F8005A9
:101CB000C00700000000000000000000003FF0FF2F
:101CC000E00700000000000000000000003FFEFFF1
:101CD000E30700000000000000000000003FFFFFDD
:101CE000E70700000000000000000000007FFFFA8E
:101CF000F7070000000000000000000000FF1E8049
:101D0000FB070000000000000000000080FF05004D
:101D1000F90F00000000000000000000E0FF0100DB
:101D2000FC3F00000000000000000000F0FF030086
:101D3000FE7F00000000000000000000F8FF0F80A0
:101D4000FFFF00000000000000000000FCFF7FF02B
:101D5000FFFF03000000000000000000FEFFFFFD89
:101D6000FFFF03000000000000000000FFFBFFFD7C
:101D7000FFFD070000000000000000803F807FF0B2
:101D80000FE00F0000000000000000800F3C7EF01C
:101D9000E3810F0000000000000000C0073C3CE0B1
:101DA000E1011F0000000000000000C0013C38E01D
:101DB000E0031C0000000000000000C0013C306097
:101DC000E0011C0000000000000000E0003C0000FA
:101DD000E001380000000000000000E0003CE03DB1
:101DE000E001300000000000000000600078C01F2B
:101DF000F001300000000000000000600078C01F0B
:101E0000F0003000000000000000002000F8C01FBB
:101E1000F8002000000000000000006000F0C10F8A
:101E20007C002000000000000000002000F0811F66
:101E30007C002000000000000000002000E0870F70
:101E40003F002000000000000000000000C0DF9FF5
:101E50001F002000000000000000002000C0DFDFA5
:101E60000F00100000000000000000400000DFDF55
:101E70000F00100000000000000000000000CE9FD6
:101E80000300000000000000000000000000E8BFA8
:101E90000000000000000000000000000000E07FE3
:101EA0000000000000000000000000000000F07FC3
:101EB0000000000000000000000000000200F8FF29
:101EC0000000020000000000000000000600FCFF0F
:101ED0000100010000000000000000000800FFFFFA
:101EE00007800000000000000000000030C0FFFD7F
:101EF0001FE000000000000000000000E0FF7FF095
:101F0000FF1F0000000000000000000080FF3FE015
:101F1000FF0F0000000000000000000000FC0700B0
:101F2000FF010000000000000000000000000000B1
:101F300000000000000000000000000000000000A1
:101F40000000000000000000000000000000000091
:101F50000000000000000000000000000000000081
:101F60000000000000000000000000000000000071
:101F70000000000000000000000000000000000061
:101F80000000000000000000000000000000000051
:101F90000000000000000000000000000000000041
:101FA0000000000000000000000000000000000031
:101FB0000000000000000000000000000000000021
:101FC0000000000000000000000000000000000011
:101FD00000000000000000000000000000080000F9
:101FE000100000000000000000000000000C0000D5
:101FF00018000000000000000000000000180000B1
:102000000C00000000000000000000000030000094
:10201000040000000000000000000000006000005C
:1020200006000000000000000000000000C00000EA
:1020300003000000000000000000000000C019982C
:1020400001000000000000000000000000001FE888
:1020500000000000000000000000000000001678F2
:1020600000000000000000000000000000001E78DA
:1020700000000000000000000000000000001C3C08
:1020800000000000000000000000000000007C1EB6
:102090000000000000000000000000000000781FA9
:1020A0000000000000000000000000000000F80F29
:1020B0000000000000000000000000000000F00729
:1020C0000000000000000000000000000000E00729
:1020D0000000000000000000000000000000E00719
:1020E0000000000000000000000000000000F00FF1
:1020F0000000000000000000000000000000F81FC9
:1021000000000000000000000000000000007C3F14
:1021100000000000000000000000000000007E7EC3
:1021200000000000000000000000000000003F7CF4
:1021300000000000000000000000000000001FF888
:1021400000000000000000000000000000800FF808
:1021500001000000000000000000000000F807F08F
:102160000B000000000000000000000000E403E09D
:1021700017000000000000000000000000F201C095
:1021800027000000000000000000000000F90180AE
:10219000CF000000000000000000000080FD018072
:1021A0009F0100000000000000000000C0FC03C010
:1021B0003F0300000000000000000000E0FE07F008
:1021C000FF0700000000000000000000E0FF3FFCEF
:1021D000FF0300000000000000000000E0FF7FFEA1
:1021E000FF0300000000000000000000C09F7FFF10
:1021F000FD0300000000000000000000C07F7E3EE4
:10220000FC0300000000000000000000E03F380E6A
:10221000FE0700000000000000000000F03F00008A
:10222000FC0700000000000000000000F039000082
:102230009C0F00000000000000000000F8380000C3
:102240009E1F000000000000000000007C780000DD
:102250000E3F000000000000000000007E7800003B
:102260000E3E000000000000000000007F30000073
:102270000EFE000000000000000000803F00000093
:1022800000FE000000000000000000803F00000091
:1022900000FC010000000000000000C01F00000062
:1022A00000FC030000000000000000E01F00000030
:1022B00000F8070000000000000000F00F00000020
:1022C00000F80F0000000000000000F80F00000000
:1022D00000F00F0000000000000000F80F000000F8
:1022E00000F01F0000000000000000F807000000E0
:1022F00000F00F0000000000000000E007000000F8
:1023000000E0070000000000000000800300000063
:1023100000E00100000000000000000001000000DB
:10232000004000000000000000000000000000006D
:10233000000000000000000000000000000000009D
:10234000000000000000000000000000000000008D
:10235000000000000000000000000000000000007D
:10236000000000000000000000000000000000006D
:10237000000000000000000000000000000000005D
:10238000000000000000000000000000000000004D
:10239000000000000000000000000000000000003D
:1023A000000000000000000000000000000000002D
:1023B000000000000000000000000000000000001D
:1023C000000000000000000000000000000000000D
:1023D000000000000000000000000000000C0000F1
:1023E000300000000000000000000000003C000081
:1023F00078000000000000000000000000FC000069
:102400003E000000000000000000000000FC018011
:102410003F000000000000000000000000FC03C1BD
:102420007F000000000000000000000000FCF3CF6F
:102430003F000000000000000000000000FCF3CF9F
:102440003F000000000000000000000000FC03C08E
:102450003F000000000000000000000000FC03C07E
:102460007F000000000000000000000000FCF99F59
:102470003F000000000000000000000000F8FD3FE9
:102480003F000000000000000000000000F0FC3FE2
:102490000F00000000000000000000000060FE7F50
:1024A0000600000000000000000000000040FEFFE9
:1024B0000000000000000000000000000000FFFF1E
:1024C0000000000000000000000000000000FFFF0E
:1024D0000100000000000000000000000080FFFF7D
:1024E0000100000000000000000000000080FFFF6D
:1024F00003000000000000000000000000C0FFFF1B
:1025000003000000000000000000000000E0FFFFEA
:1025100007000000000000000000000000E0FFFFD6
:1025200007000000000000000000000000F0FFFFB6
:102530000F00000000000000000000000070FFFF1E
:102540000F0000000000000000000000000000007C
:10255000000000000000000000000000000000007B
:1025600000000000000000000000000000F8FFFF75
:102570001F000000000000000000000000F8FFFF46
:102580003F000000000000000000000000F8FFFF16
:102590001F000000000000000000000000F8FFFF26
:1025A0001F000000000000000000000000F8FFFF16
:1025B0001F000000000000000000000000F8FFFF06
:1025C0001F000000000000000000000000F8E3CF42
:1025D0001F000000000000000000000000F8E3C73A
:1025E0001F000000000000000000000000F8C1878C
:1025F0003F000000000000000000000000F8C18360
:102600001F000000000000000000000000F861044E
:102610001F000000000000000000000000F83DFC6A
:102620001F000000000000000000000000F83FFC58
:102630001F000000000000000000000000F87FFC08
:102640001F000000000000000000000000F8FFFF75
:102650001F000000000000000000000000F87FFEE6
:102660001F000000000000000000000000F83FFC18
:102670001F000000000000000000000000F81FF82C
:102680001F000000000000000000000000F81FF81C
:102690001F000000000000000000000000F03FFCF0
:1026A0000F000000000000000000000000F0FFFF2D
:1026B0000F000000000000000000000000E0FFFF2D
:1026C0000F000000000000000000000000E0FFFF1D
:1026D00007000000000000000000000000C0FFFF35
:1026E0000300000000000000000000000000FFFFE9
:1026F0000100000000000000000000000000FFFFDB
:102700000000000000000000000000000000FC3F8E
:102710000000000000000000000000000000E007D2
:1027200000000000000000000000000000000000A9
:102730000000000000000000000000000000000099
:102740000000000000000000000000000000000089
:102750000000000000000000000000000000000079
:102760000000000000000000000000000000000069
:1027700000000000000000BF000404050604060776
:102780002026FFF919F919FA03D3085319D920069D
:1027900000C03009210E255B70093F503164BE7DB9
:1027A000A00022102B51180A64F01B12A284881278
:1027B0000100233F32C36F6A640692193886E0181D
:1027C0007264C891194866D003110F443C10F1405F
:1027D00010998183060E1A3886D003110F443C10DD
:1027E000F140D0187264C891194866E01882638875
:1027F00001243090CB4E7AC2C52263E3C284884A5A
:1028000084A41192464C127109136A89309D90720A
:1028100062D0884123448990124EDC2C342C5C3ADF
:1028200000254AFA4AB04B63051E1C974EE098619A
:10283000E3468D12386AD0C05163468E1A3374CC89
:10284000B469449F190F6094A8F100C69C16937652
:10285000CCB462468D1C336AA4A05103078D1A378D
:102860006CCCC061E9061E143B08002635345310B9
:102870006BA593AE5C498660198265481621A9361E
:102880002DE2B36A88AC2152C990324A482521769C
:10289000865CA172650CA179308445A134A58A02B9
:1028A000270C245118090F5A08110100281DE84B64
:1028B0006D5983C810224388D020DA10A23F2A44E1
:1028C0005784488D22358AD400291FE84B6D09A30F
:1028D00028224588D428425411A2BF294388A24106
:1028E000140D223488D028002A186AC9B649024536
:1028F0000511126284881688489941324DA0200043
:102900002B10104A706A84E9D9831F10234CCF0022
:102910002C0E65512D090FD44832629240002D07CC
:10292000A9C873093F2E08A55030090F142F1A2883
:1029300043306972254CAA51C2A41A254C2A61520F
:102940008D12269530C900301D0F4B504AE752AD0D
:102950006952A64429ADD2E1EF526955A24C913695
:10296000ABD21D023110EA52507AC3489579F0E09B
:1029700018FDFF01321E104B504AE716B57161C6B3
:1029800044A965E9D215355AD4A485179AB4E983C8
:102990001F103325104B504AE716B56952AA04B1EF
:1029A00012E44890235BB4E049A368AD4D97D9AADF
:1029B000224E1AAD3B05003426104B508A658B9A87
:1029C000BC101D0972438811213686141942148DDA
:1029D00022438ACC30320F7E409230DD00351E0F0C
:1029E0004B502A6C7833962E4AB169D28490D16AC2
:1029F000C9224BA6A8481346EA4C0136250F4B5076
:102A00005AE614B16951A80431B494142281C485E2
:102A10000B33ABD2E12E55893245DAAC4A580A0065
:102A2000371A104B500A7F40966C596ACB922D4B47
:102A3000B62CD96AC9D6B46C0D01382A1143505A44
:102A40000757352A5355117244C8112147A4549988
:102A5000AA96AD6A53AA44B99458A62B61C688A316
:102A6000560B4F0139250F4B505A0553AD6952A6ED
:102A700044A974B84BB5C68427284811214B1619B0
:102A8000894245D8B04A580A003A0C255A70090FB5
:102A9000D443F540013B12E55A6D090FD443F5408C
:102AA0008D2423260904003C18104A70EA624B1E4C
:102AB00053B4848DB29327D52D5CA7F26C71013D80
:102AC0000A8F51710A7F0F077F3E18104A700AC2A1
:102AD000099F54B78E9DCACBD43059A4EC2461E130
:102AE000003F203053904AE716B57161C644A9658E
:102AF000E9D2153569F2E0499365C9560F75D93A9F
:102B0000034060DDCB2DCCE701357F10D8D8C9B2AA
:102B1000E58813230F82D47830D4951833D99A21BD
:102B2000C388181A318A10A943C446991A37CA10A3
:102B3000B95186C68D3A346ED48841E3468D184427
:102B40008AD0103284CA9019F46010A123C74615A8
:102B500022481E2C79B0E5412223FD20F87B104A43
:102B60000141343643F08AE6419807801C6BC5DA90
:102B700016295AA46891928548162A58A85C317281
:102B8000C58A3D08F620D483410F06152C53B4485E
:102B9000D1124617174232335B100BAE1E847920D8
:102BA000E4819072260A962858A260898225CA1567
:102BB0007910E6419807421E8C2858A2A43E7C90CA
:102BC000E2C18807421E014336354B107B68193A33
:102BD0007B10E89A82454A9A285AA2A87A10E541C1
:102BE0009407511E447910E541940752B444D11220
:102BF000068D142C73E8D083600ED92203442D3542
:102C000053100B0D1F847A20E8C19872474A162989
:102C100069A26889A26BF5A74B4B943451B248B9AD
:102C2000230FC63C10F42054430045213253D00AF0
:102C30000F443C10F140C40311A5EBF583200F8233
:102C40003C08F22048E9FAFAC10F184611305390B7
:102C50000A7F90B6DEBEF845D9FA6F014733364B8E
:102C6000308B88193E7B20EAD01983458C9628BB8F
:102C70001E447920E581940752EE0FC296285BC26C
:102C8000680993464E217950E6C52826C3120D489F
:102C9000103353F00A25F55F3EF88395FA5F164925
:102CA0000925533009FF07054A132F4B50AAF5FF9A
:102CB000A92ABD5AF3A0489B6587004B37345310AF
:102CC0000B054D143451CE483133A50C153255C681
:102CD00058997245CC9530B872254386ED8C182BE7
:102CE00064AA90A952868A992957A69C9182264A5D
:102CF000AE344C0E3053900A65EBFFFFF6C10F085F
:102D00004D473753700B275DBE7B10EE41B807E18E
:102D10001E887A30CAC5A8112A468D504186840A79
:102D20003224549021A164CC1025248828214144C8
:102D30000909224A48105133628C9A336ACEA83965
:102D4000A3A890A2428A2A4E273353100B25172E90
:102D500064C7AE5933578F5410525146091925454F
:102D6000D4105153421109559E75C7E196054F2D58
:102D7000374B307B895BBE7B200A0D2273664C1A71
:102D8000295BA46C89D2FA7589B245CA163169C625
:102D90009C2134A81E887BD9381D0050203253D086
:102DA0000AADDE3C08F240443113E516EADD321389
:102DB0000F443C08E28859E9FA6B00513457CB4F75
:102DC0007B895BBE7B200A0D2273664C1A295BC28D
:102DD000EC6AFD32CCBA21258A9520624A8D2944BD
:102DE000888C3D18F660D8837149C883120200525E
:102DF000333353100B8F1E087930E2C188822BF5D4
:102E0000B04439130F843C08F320CC0321E54C1463
:102E10002C51B044C112054B142C51B044C11205C1
:102E20005716532B334BD06A47D7B57A54C84CB991
:102E300022048B902452FCB4CA760ED92237AE52AB
:102E4000658982254C997910C819CB6300540E33DB
:102E500043900AFF205CF1FAFFBF0355163353106D
:102E60000B25F5FFBF5C67E2CC9107625E354C0530
:102E7000005634344BD00A4595962858A460918268
:102E80006508122A56A8582962C40A152B548E10B8
:102E9000414204099124429408512244D522C6DAC1
:102EA000B8F500080257523D4BF00BC58C2DB3828C
:102EB00098B122C48C152166AC482144650A212AA8
:102EC0005308512142880A111A328854116A481550
:102ED000A1A418114A8A11A11D914143C8111934A6
:102EE000842022948850224279ECA831B3C6CC1AAF
:102EF000334C90344172005833344BD00A068B184F
:102F00003362AC9055858A192958A46089A24A1366
:102F1000233E6EFA34DAB42A4B983352AE8C2943EE
:102F2000A54A993156C49C0983065934344BD00ABA
:102F30000619163166A658211B152B54CC48C12200
:102F400005972A4D8CF8F4F1F200CA03280FA03C33
:102F500080F200CA03280FA03C80F2000A025A1B2C
:102F6000314B900A7F80B8AC516BCB1AB5D6A8B55F
:102F7000658D5A6BD4EC831F205B0EE8536D090FEF
:102F80001AD1FFFF1F3D485C1F29433009E2C48D61
:102F9000936ED83871C3C6891B364EBA61E3C40D2F
:102FA0001B276ED838095D0EE8436D090F12D1FF5B
:102FB000FF1F3D685E19CED1745A240D5A870C1537
:102FC000114244084D4388082122C330235F085230
:102FD000404D0A1F18600CA5507A0943880C213215
:102FE00000611F4F4A504AA8983429A42C19C143A4
:102FF0004B5A9C49960C99A2070F4CA4206286005C
:1030000062213053900A84E92786482471F2C25025
:103010008962E912E25D3A55255E382181864C21AC
:1030200000631C4F4A505AE614B16152A804A974B7
:1030300068E92E19894225DAAC526708006420300D
:103040004B90CAF4232364501071F1A2D0B284F8DB
:1030500030598942269EA4208382501902651E5051
:103060004A505A0655B17152A844B1740F3E604C93
:10307000B8189142451AB14A590C0066142A437097
:103080005985CC9C29458C9A076F88D1FF370067FA
:103090002930CB8C4A46C8A020E2E245A165CA127D
:1030A000E23099B212854C3C7183829011C2C9946E
:1030B000953062C40D33440068162F53900A64E9BA
:1030C0003784482071E1C290B264E8F0BF23690CF4
:1030D000245330090F023EF883006A1106C42C29DC
:1030E000744E84FEFF4F1E982801006B282F5370EA
:1030F0000A64E967A94A102A42A60C9142244A258B
:1031000053A56AD1A22265C8942154841411522572
:1031100088252B6C0924533009FF81026D305852E9
:10312000D00B644895218122C503140FDE9C5155B4
:103130000A193164C4901143460C193164C49011CA
:1031400043460C193164C490114346016E144F522A
:10315000900A64CA9048E1E2812165E8F07F470067
:103160006F1D514A905A0757B57952AA44397529AB
:1031700071994E5D895245DEB45A780A0070233049
:10318000D38C0A640A9140E3E485A112C59425C456
:103190006132658B4ABC7042020D994284E963003A
:1031A000711F30CB8C5A45C8A020E2E245A16509C9
:1031B000F161B212854C3C7192829011C2F403729B
:1031C000134A52B009848CA078F02050A952C4E868
:1031D0009F017320504A705AE716352954845809C4
:1031E0006225CA265CB74EE9BA74244A9570C30CAE
:1031F00011007413C94A7029A468F3800929FAAF31
:103200008E9C31540075144F52900AE4F07F974A17
:10321000D103132E529029430076285142700AE5BB
:10322000D4952855A45419528448112A538A0C3134
:1032300032C4C890234190044112248F5E5BB818B9
:103240000077405942500BA54AA9AA8254292285E9
:103250002A2973A60C993384C89C214466C4184259
:10326000444810214562CC086224C68C204662CCBA
:10327000086268D0993268CAA02993E4889223052D
:10328000007823504A700AC516992854A648A122EE
:10329000C4D4A1344BD6E44974AA8A902A52A650C9
:1032A0000943CB0A792730CB6C0AC5342342AA489C
:1032B000A122856854A4501162448811219610C33C
:1032C000A39696ADB4E449A34689027A114E4A30DA
:1032D0000A3F5858A1391BD6E5830F167B1909D42C
:1032E000AC49658C1C29448AFE512142E34895A2D1
:1032F000FFEA8CA1027C09E35B2D09FFC1007D1A66
:1033000009D4AC0985CC1C2A45FF552972830815C0
:103310002245FFE4889942007E0FCED0722A434DA9
:103320002D31B2CAE81000A00600C03009A10E0578
:10333000536D090FD40E99170F3E50A22E0FCB4E8E
:10334000AAC1438B3CA68849932221D40449220474
:103350008D3032C2888823228E889814814898291B
:10336000D166553A93A2830705A3271143506A06F5
:1033700057357262A848B112C54A942351D870518A
:10338000560C4BD3B8301564843CF8808830230049
:10339000A420EF49520A234F947840A20DAD888CA7
:1033A0001B326EC8B821A4C850D3E2018912270786
:1033B000A5261243500A051596285686182942C498
:1033C00008912342900849A4684D9374E4923849C7
:1033D000472E89D33B00A60DE35B2D091FA407F3FD
:1033E000E08101A73510CC4C4AE8542D3252A6108A
:1033F0009942648C1E45896E519B31280831DB8CC3
:10340000C42112488A34529812A9D922C4881023A0
:1034100052A80C23560A4D01A80A8AC07A094470A2
:103420004200A9503A43109BE801342657B028B90E
:10343000E1A3C6831833CC989851A8468C22424AFF
:10344000C4A061834A0D1B45683C0042E301101A89
:103450000F80D07800A4868D2A346C90292284862F
:103460000843356498A941E3010C234BB05C51E754
:103470002A01AA1709CA9429654E8C2934C6041357
:1034800033665890180FE60103AB22AC59514AC17C
:10349000C28812326804193424060D1934840C8948
:1034A0002225C81019344694A06001AC0A50497214
:1034B0000A7F40983EAD07A9C873093FAE503A4312
:1034C000108BE901342657902CB9E1A3C6241A3396
:1034D0004891984183C88C183591885113891036CA
:1034E0006A50B141A38A252B86AED89861C5C69093
:1034F000323568948851D30C19348AC844C3460CB9
:103500001A0F6018E18105893A570900AF076AC0B0
:103510007A091FB0144951B729658E8811218A563E
:1035200022C40839530400B114D04A706A84E9D91E
:10353000831F10234CEF217CF00302B216EAC17402
:1035400029665010396468DC305214152236ECC1FB
:1035500003B319EAC1743984501039646818A15250
:10356000E5C819327484049A3200B40CA6607A2932
:1035700024884C330600B5152FD38C0AE4F07F97CE
:103580004AD1830F42A0208296BE05B64BF1434D2F
:103590004A6D9C9C118446101A3169C4A41193464B
:1035A0004C1A316904A1118446D4195167C495118C
:1035B0002A46A818A162848A112A46A818A1628402
:1035C0008A112A46A818A162848A112A46A818A13D
:1035D00062848A110300B70AA4D0351922588800E2
:1035E000B80E07D16C29A2242A4428451100B90C31
:1035F000E6D17439431E8499FF01BA150ACA942989
:1036000066904C31C88E460C1982C63CB8070FBB79
:10361000218CD9510AC102891233680819226488A1
:103620000C1A326804193424060D1125265820007E
:10363000BC461A4390FB60860A1D4974D8C97107BD
:10364000070F1C3C6EF4B8D1C3860F1B3E6AD844EA
:10365000C3880D1A556CCCB0C2A3448C1D2564ECF4
:10366000A02143478919394AD0C851CB862D1B3C2C
:103670006EF4B8D14300BD42194B90FB20868A1CE2
:103680003A729CC18106C78E1B3C6CF4B0D1A386F4
:103690008F1A3E6890A94182108D194384CC9041C5
:1036A000130E9A6E2CB9A1E486921B4A7024C19124
:1036B0002407AA19A966A402BE4C194B702B6607F1
:1036C000A11C4484E0A0E9460D1A3698D8D0626364
:1036D0008B8D35341EC0989183C60C1A3268C82071
:1036E00022940C228364502133630C8F193176901D
:1036F00090B163C40C1D33E9987583D60D1D3876DF
:10370000E0D82100BF1E104B8D6A656B0F35616AD2
:103710004B9A3C78D2D272D9A92A61E4849B36CCE8
:103720001001C040F643F06AE4019107441E10798D
:1037300040E421340FC23C00E4582BD6B648D122D5
:10374000458B942C44B250C142E58A912B56EC41F2
:10375000B007A11E0C7A30A86099A2458A9630BAAB
:10376000B800C140F643F0CAE4819007421E0879D0
:1037700020E421350FC23C00E4582BD6B648D122B4
:10378000458B942C44B250C142E58A912B56EC41B2
:10379000B007A11E0C7A30A86099A2458A9630BA6B
:1037A000B800C241F643F0AAE2019107621EC09040
:1037B000D183C643661E847900C8B156AC6D91A210
:1037C000458A1629598864A18285CA152357ACD821
:1037D00083600F423D18F46050C132458B142D6157
:1037E000747101C33CD643F08A6404AB552C863C0B
:1037F00074E6419807801C6BC5DA16295AA46891B3
:10380000928548162A58A85C3172C58A3D08F62070
:10381000D483410F06152C53B448D112461717C450
:103820003FF643F06A440813214C843011F2B0365D
:103830000FC23C00E4582BD6B648D122458B942CBD
:1038400044B250C142E58A912B56EC41B007A11E0B
:103850000C7A30A86099A2458A9630BAB800C54360
:10386000F643F09AE481480F2250781081C2831009
:10387000221E087928CD03408EB5626D8B142D521F
:10388000B448C942240B152C54AE18B962C51E04A5
:103890007B10EAC1A007830A96295AA46809A38B62
:1038A0000BC64B3F43108C0F4E3E38F9E0E00384CB
:1038B00045C88322431E5019F280CA9007443D98A0
:1038C00042E4C114220FA6D0B352CF4A3D2BF5AA31
:1038D000187910EF41BC07F0203C8007E1019423E8
:1038E0005EF08188820F4E3E38F94000C74515CC06
:1038F000EC7A68193A7B10E89A82454A16295AA24E
:10390000A87A10E5419407511E447910E5419407C7
:1039100052B444D112068D142C73E8D083600ED9B2
:103920009E07211E907830E5018D0733DC3C8092A4
:1039300000C82CF253D03AE4019007401E007900F1
:10394000E4813E10F140C403110F4494AED70F82BE
:103950003C08F220C88320A5EBEB073F60C925F2A5
:1039600053D09AA4E91EF003110F443C10F14044D7
:10397000E97AFD20C883200F823C0852BABE7EF04F
:103980000306CA2BF253D08AE20190363B64E4A0CE
:10399000F1E01E887820E2818807224AD7EB0741B0
:1039A0001E047910E44190D2F5F5831F30CB2AF242
:1039B00053D03AD4912147861C19F2903E10F14021
:1039C000C403110F4494AED70F823C08F220C88381
:1039D00020A5EBEB073F60CC0FE8433009A4E8B427
:1039E0004CFDFFFF0500CD0FE853304964E8B84CAB
:1039F000FDFFFF0D00CE14EA433049E24899193229
:103A000062D0E052F5FFFF3700CF11EA433009449E
:103A100070421E5CA9FAFFFF1B00D03C373BF03A16
:103A20002E1F847B20ECC1A852A80A1A2A68A86419
:103A3000A192668A9629FA40D803610F8495295A83
:103A4000A6689992854A162A59A860A962A71E08F5
:103A50007B20ECA13300D12FD353106B64442A5444
:103A600029863CD0920B17B263D7AC99AB472A0892
:103A7000A928A3848C92226A88A829A188842ACFA5
:103A8000BAE370CB02D238F74B307BE44191074563
:103A90001E147950E4214CDCF2DD03516810993397
:103AA00063D248D922654B94D6AF4B942D52B68839
:103AB0004933E60CA141F540DCCBC6E900D338F729
:103AC0004B30DBE4C19007431E0C7930E4214DDC20
:103AD000F2DD03516810993363D248D922654B94C3
:103AE000D6AF4B942D52B6884933E60CA141F54030
:103AF000DCCBC6E900D439F74B30BBE24191076318
:103B00001EC490E183C64396B8E5BB07A2D020321D
:103B100067C6A491B245CA9628AD5F97285BA46C8E
:103B2000119366CC194283EA81B8978DD301D535BC
:103B3000D74B309B64442B562D863C74895BBE7BEF
:103B4000200A0D2273664C1A295BA46C89D2FA757F
:103B500089B245CA163169C69C2134A81E887BD912
:103B6000381D00D637F74B307B444813214D843441
:103B700011F2304FDCF2DD03516810993363D24803
:103B8000D922654B94D6AF4B942D52B6884933E673
:103B90000CA141F540DCCBC6E900D7200F52702ABA
:103BA00021C38C1B516A8D096B56A53B782ED51A03
:103BB00013D6AC2A316E4CC82000D849384B307B24
:103BC000A9463519F560D483516850192C64F04C1E
:103BD0004134E548102938A444B931258A0D2A51C9
:103BE0006A548942C34A941957A2CCB82225C69573
:103BF0004158E6A02173A6D0A07A30EC81B011CD57
:103C0000062504D921F353105BE4419007411E04BB
:103C10007910E48196D4FFFF729D8933471E88791D
:103C2000D5301500DA19F35310BBC4E91E7049FDF5
:103C3000FF2FD7993873E48198570D5301DB20F398
:103C400053109BE24110373C64E8A0F1004BEAFFBF
:103C50007FB9CEC499230FC4BC6A980A00DC20F354
:103C600053104B6408922148862019F21097D4FF14
:103C7000FF729D8933471E8879D5301500DD40F4E9
:103C80004BD0BAE4019007401E007900E4811B6428
:103C900068C2989962856C54AC503123058B145CD2
:103CA000AA3431E2D3C7CB03280FA03C80F200CA6C
:103CB00003280FA03C80F200CA03280800DE22324D
:103CC00053D00AA5AB6EF5E6419007228A9928B732
:103CD00050EF96997820E24190378E4AD76B00DFFB
:103CE000333153904A2695B57153C848A922C48AE6
:103CF000102B42AA0C2133640C9139430609A913F5
:103D0000E44A9053983B6526C8A4208384CC19329A
:103D1000A500E0252F4B504A84098F9E1E42544C2B
:103D20009A1452968C1CA2252DCE2443874CD18305
:103D300007265210314300E1242F4B509A44C9CE3C
:103D40001E52544C9A1452968C1CA2252DCE2443FC
:103D5000874CD18307265210314300E2282F4B5065
:103D60007A82891A1C326CD078C85031695248590D
:103D700032728896B438930C1D32450F1E98484114
:103D8000C40C01E3270F4B505A6444295225863C4A
:103D900074A8983429A42C1939444B5A9C49860E8E
:103DA00099A2070F4CA420628600E4290F4B503AD9
:103DB0004448112145841411F290A162D2A490B21A
:103DC00064E4102D697126193A648A1E3C30918290
:103DD000881902E52B2F4B506A4485880C14325009
:103DE000482142C98344C5A4492165C9C8215AD282
:103DF000E24CB264C8143D78602205113304E63504
:103E00007A4AB05BA60AAA48F5E0D08333850C1540
:103E10002146093162458B957A60E4418A072A4A36
:103E2000912D46B618B145861E3C08B262519A746F
:103E3000C54C01E7252FCB4C5AE614B16152A804BA
:103E4000B16468695B2C19894225DAAC526754B4B5
:103E5000E0D283079A2C0600E825304B504AA4494B
:103E60000F9F1E6283AAD8382954A21809720F3EE8
:103E7000604CB818914245DCB04A590C00E9243036
:103E80004B509A6409CF1E7283AAD8382954A218BD
:103E900009720F3E604CB818914245DCB04A590C8B
:103EA00000EA28304B507AA2C99A1C326ED078486A
:103EB0000DAA62E3A450896224C83DF88031E16212
:103EC000440A1571C32A653100EB29104B503A445E
:103ED00088112146841811F2901A54C5C649A112BE
:103EE000C548907BF00163C2C588142AE28655CA92
:103EF0006200EC10274B300984088D9A1E0819FACD
:103F0000FF07ED112653302944A619321E0011FA7D
:103F1000FF2700EE142A3B3049E24899193262D05B
:103F20007880C4E8FFDF00EF100A3B30094470429C
:103F30001E2031FAFF3700F02B514B902AC24985E1
:103F40002B422EE5C97443CC0532998C519B27A591
:103F50004A94539712CB74EA56993063E44DAB857B
:103F6000A700F11C0F53904A6444295225863C4413
:103F700044CC9040E2E2812155E9F07F4700F223F2
:103F8000314B905AC4890FA71EF283ABDA3C2955F6
:103F9000A29CBA94B84CA7AE44A9226F5A2D3C05F6
:103FA00000F323314B909A84494F4D1E160757B5A5
:103FB0007952AA4439752971994E5D895245DEB40A
:103FC0005A780A00F426314B908AC2091B1D3270C0
:103FD000D078880FAE6AF3A4548972EA52E2329D17
:103FE000BA12A58ABC69B5F01400F525114B905A98
:103FF00064C4295327863CE40757B57952AA44394B
:10400000752971994E5D895245DEB45A780A00F6D9
:1040100026114B903A94912146861819F2101F5C94
:10402000D5E649A912E5D4A5C4653A75254A15799E
:10403000D36AE12900F712104A706A84690FE1839C
:104040001F90879030CD00F82E553A907A8746AD74
:1040500018F5991953C50C953A446A04214243084E
:10406000911943A8C49842A70A99B2C6D8AB57235E
:10407000560D3A0700F9192F53903A84098F9E1E66
:104080002A72F8BF4BA5E881091729C89421FA18AC
:104090002F53908A44C9CE1E3A72F8BF4BA5E881CF
:1040A000091729C89421FB1D2F53906A82891A1C75
:1040B000326CD07868C8E1FF2E95A207265CA42058
:1040C000538600FC1E2F53902A64089121448610C9
:1040D00019F2302187FFBB548A1E987091824C19C7
:1040E00002FD2B10CC6C9A64299E1ECA629A952000
:1040F00046A4509142F4A808A922C488104B9710F6
:10410000E1514BCB565AF2A451A34401FE2410D4E2
:104110008C0A84E92786482479F1C2D03265097176
:10412000984CD9A2122F9C904043A61061FA180017
:10413000FF35F0CB6C3A4488112146841811F250B7
:1041400015D3AC04A922858A142253885091424584
:10415000481521468458BA84088F5A5AB6D29227F5
:104160008D1A250A0000000000000622766D247FCB
:1041700020390F5C50104008063F065B4F666D7D8E
:10418000077F6F303058484C535F777F395E7971C5
:104190003D76060E753815373F7367336D783E1CD4
:1041A0002A766E5B39300F1308105F7C585E7B7186
:1041B0006F74040C753015545C7367506D781C1C5B
:1041C0002A76665B79064F40000000200023002617
:1041D0000029002C002F003200000100000301061E
:1041E00001090100002200250028002B002E0031CB
:1041F00000340002010000050108010B010505055E
:1042000005070508080808020202020A0A0808044D
:10421000040404010101010101010103030303037B
:10422000030303040707070C0C0C0C0C0C0C0C020A
:1042300002020206060606060606060B0B0B0B0B11
:104240000B0B0B010210202008081020401020400A
:10425000800201020108040201010204081020404A
:104260008080402010080402018004020180402068
:104270001008040201080402010102040810204091
:104280008001020408102040800000210024002743
:10429000002A002D00300033000101000004010756
:1042A000010A0100000A0B02090C0D0E08070304A5
:1042B00001000000000000000000000000000000FD
:1042C00000000000000000000000000000000012DC
:1042D00011100000000000000000000000000000BD
:1042E0000000000000000000000007619E5E112435
:1042F0001FBECFEFD1E2DEBFCDBF00E00CBF19E0A3
:10430000A0E0B2E0ECE1F7ED00E00BBF02C00790E7
:104310000D92A033B107D9F721E1A0E3B9E001C0C4
:104320001D92AD32B207E1F711E2C6E7D1E200E03B
:1043300006C021970109802FFE010E944569C537FB
:10434000D10780E00807A9F70E946A4E0C947D6BA4
:104350000C9400003F924F925F926F927F928F92E7
:104360009F92AF92BF92CF92DF92EF92FF920F9304
:104370001F93CF93DF93CDB7DEB7AD970FB6F89409
:10438000DEBF0FBECDBF28E2F22E38E3A32E42E3FC
:10439000B42E53E0E52E6DE2962E71E4872EE5E50E
:1043A0003E2E80918E0981110C94F72B89EF93E0BA
:1043B0000E941438882309F400C14EEF53E068E0EE
:1043C00081E00E9429340E94F13448E054E064E125
:1043D00089E00E94293440E154E06EE189E00E94C6
:1043E00029344EE154E068E289E00E94293447E232
:1043F00054E06CE389E00E9429340E94E64B0E945D
:104400005E35182F8823D9F364E071E08FE00E94B5
:104410000D4B0E9406351133B9F481E080930B02F5
:1044200007E713E220E440E860E080E00E942437E0
:104430000E94E64B68EE73E080E090E00E94914DB0
:1044400063E374E00C94D12A123349F482E0809340
:104450000B0281E080938E0907E71FE109C0133347
:10446000B1F4E0920B0281E080938E0907E71BE133
:1044700020E440E860E080E00E9424370E94E64BA0
:1044800068EE73E080E090E00E94914D8ACF133295
:1044900021F46CE374E00C94D12A1A3209F08AC03A
:1044A0000E9406350E945E358823E1F3853309F0CA
:1044B00078CF0E945E358823E1F3833309F071CF12
:1044C0000E945E358823E1F3863309F06ACF0E94AB
:1044D0005E358823E1F3863309F063CF0E945E35B1
:1044E0008823E1F3893309F05CCF81E080933409BC
:1044F00045E454E066E182E00E94293444E554E05A
:1045000061E28EE00E9429340E94E64B62E071E095
:104510008FE00E940D4B68EB7BE080E090E00E9412
:10452000914D0E9406358FC188EB94E00E941438AB
:10453000811137CF83EC94E00E941438811131CF80
:104540008CE394E00E941438882309F48BC10E9404
:1045500006354AE254E068E081E00E9429340E9476
:10456000F13449EC54E064E189E00E94293449EDDA
:1045700054E06EE189E00E94293443EE54E06CE39C
:1045800089E00E9429340E94E64B0E945E35182F74
:104590008823D9F364E071E08FE00E940D4B0E9404
:1045A0000635113309F455C1123309F458C11332D9
:1045B00009F449C10E94094AF4CE83E394E00E94C1
:1045C0001438882309F4B0CF0E94063541E055E045
:1045D00068E081E00E9429340E94F1344FE554E004
:1045E00064E189E00E94293446E654E06EE189E006
:1045F0000E9429344EE654E068E289E00E942934A2
:1046000048E754E06CE389E00E9429340E94E64BBD
:104610000E945E35182F8823D9F364E071E08FE0A3
:104620000E940D4B0E940635113309F0CCC011E0F9
:10463000109368098CE59CE00E94363440E854E011
:1046400068E289E10E9429340E94E64B8CE893E0FD
:104650000E94363468EE73E080E090E00E94914D55
:104660000E94063549E854E066E181E00E94293461
:1046700049E954E061E281E00E9429340E94E64B5E
:1046800010930C0201E092E0D92E80910C0285304B
:1046900009F463C00E945E35182F8823B1F364E0EB
:1046A00071E08FE00E940D4B10337CF3C0900C0240
:1046B00081E0C81212C060ED610F60930502109294
:1046C000110C88E09CE00E94EA34C092110C63E176
:1046D00073E088E09CE00E940F3580910C028230EC
:1046E00051F460ED610F609304020093110C88E0B7
:1046F0009CE00E94EA3480910C02833051F460ED1A
:10470000610F60930302D092110C88E09CE00E943C
:10471000EA3480910C028430E1F460ED610F609323
:104720000202E092110C88E09CE00E94EA34809141
:104730000C028F5F80930C020093060268EE73E018
:1047400080E090E00E94914D88E09CE00E949837C4
:104750009CCF8F5F80930C0298CF0E9406354FE963
:1047600054E064E184E10E9429348CE59CE00E94DD
:10477000363489E18093090DF0920A0D60910502AB
:1047800080E99CE00E94EA349092090DF0920A0DB3
:104790006091040280E99CE00E94EA348092090D55
:1047A000F0920A0D6091030280E99CE00E94EA34D5
:1047B0003092090DF0920A0D6091020280E99CE0AE
:1047C0000E94EA340FC01233E9F482E08093680952
:1047D0008CE59CE00E9436344EEA54E068E284E1C5
:1047E0000E9429340E94E64B8CE893E00E94363404
:1047F00068EE73E080E090E00E94914D81E080934C
:104800008E09CFCD133309F0D2CEE092680911E0C2
:1048100010938E098CE59CE00E94363441E754E009
:1048200068E28EE10E9429340E94E64B8CE893E016
:104830000E94363468EE73E080E090E00E94914D73
:1048400010938E09AECD69EF73E0ABC6133209F059
:10485000B1CE6BEE74E0A5C6133209F0ABCE67EFB4
:1048600074E09FC68BEE94E00E9414388823E9F12F
:104870000E9406354CEC54E068E080E00E94293448
:104880000E94F1344EEF54E064E189E00E94293443
:1048900040E154E06EE189E00E9429344EE154E0A9
:1048A00068E289E00E94293443EE54E06CE389E039
:1048B0000E9429340E94E64B0E945E35182F8823FF
:1048C000D9F364E071E08FE00E940D4B0E94063541
:1048D000113309F4BCC2123309F490C3133309F441
:1048E0007EC5133209F066CED4CD87EF94E00E94E6
:1048F0001438882309F449C00E9406354CED54E071
:1049000068E081E00E9429340E94F13446E355E0DA
:1049100064E189E00E94293440E455E06EE189E0D9
:104920000E9429344EE455E068E289E00E9429346F
:104930004FE555E062E389E00E94293443EE54E0FC
:104940006CE389E00E9429340E94E64B0E945E35A8
:10495000182F8823D9F364E071E08FE00E940D4B9B
:104960000E940635113319F46FE675E01AC612334A
:1049700019F466E775E015C6133309F410C614334D
:1049800009F015CE6EE875E00CC68BE095E00E944C
:104990001438882309F44BC00E94063549E955E0D4
:1049A00068E080E00E9429340E94F13446EA55E034
:1049B00064E189E00E94293444EB55E06EE189E02E
:1049C0000E94293442EC55E068E289E00E942934D3
:1049D00041ED55E062E389E00E94293443EE54E062
:1049E0006CE389E00E9429340E94E64B0E945E3508
:1049F000182F8823D9F364E071E08FE00E940D4BFB
:104A00000E940635113319F460EE75E0CAC5123301
:104A100019F46EEE75E0C5C5133319F46CEF75E04B
:104A2000C0C5143309F012CF65E076E0BAC580EE58
:104A300095E00E941438882309F488C00E94063546
:104A400049EA55E068E080E00E9429340E94F13490
:104A500044E156E064E189E00E9429344EE156E0E9
:104A60006EE189E00E94293449E256E068E289E07B
:104A70000E94293444E356E062E389E00E9429342D
:104A800043EE54E06CE389E00E94293483E090E037
:104A90000E9454488F3079F030F48530B1F44FE300
:104AA00056E064E10FC08E3151F08C3371F44FE366
:104AB00056E062E307C04FE356E06EE103C04FE308
:104AC00056E068E280E00E9429340E94E64B0E9492
:104AD0005E35182F8823D9F364E071E08FE00E94DF
:104AE0000D4B0E940635113351F442E456E063E267
:104AF00088E20E9429340E94E64B65E00BC0123325
:104B000061F441E456E063E288E20E9429340E94A5
:104B1000E64B6FE083E090E092C1133351F44CE434
:104B200056E063E288E20E9429340E94E64B6EE17F
:104B3000F1CF143309F08EC147E556E063E288E215
:104B40000E9429340E94E64B6CE3E4CF8EEE95E0A0
:104B50000E941438882309F488C00E94063547EB68
:104B600055E068E080E00E9429340E94F13442E67A
:104B700056E064E189E00E9429344BE656E06EE19C
:104B800089E00E94293445E756E068E289E00E9406
:104B9000293440E856E062E389E00E94293443EE7C
:104BA00054E06CE389E00E94293484E090E00E94A4
:104BB0005448853079F030F48130B1F44FE356E059
:104BC00064E10FC08A3051F08F3071F44FE356E04A
:104BD00062E307C04FE356E06EE103C04FE356E0E7
:104BE00068E280E00E9429340E94E64B0E945E3514
:104BF000182F8823D9F364E071E08FE00E940D4BF9
:104C00000E940635113351F44BE856E063E288E226
:104C10000E9429340E94E64B61E024C0123351F413
:104C200042E456E063E288E20E9429340E94E64BA7
:104C300065E018C0133351F444E956E063E288E2BA
:104C40000E9429340E94E64B6AE00CC0143309F03C
:104C500001C141E456E063E288E20E9429340E94E7
:104C6000E64B6FE084E090E0EAC08CEF95E00E94B4
:104C70001438882309F46FC00E94063545EC55E0CE
:104C800068E080E00E9429340E94F1344FE956E048
:104C900064E189E00E94293449EA56E06EE189E046
:104CA0000E94293444EB56E068E289E00E942934EE
:104CB00043EE54E06CE389E00E94293485E090E003
:104CC0000E9454488A3041F08F3051F0853071F4A1
:104CD0004FE356E064E107C04FE356E06EE103C0E6
:104CE0004FE356E068E280E00E9429340E94E64BE0
:104CF0000E945E35182F8823D9F364E071E08FE0BD
:104D00000E940D4B0E940635113351F44AE059E0E0
:104D100063E288E20E9429340E94E64B65E018C0F5
:104D2000123351F447E159E063E288E20E942934EA
:104D30000E94E64B6AE00CC0133309F08BC045E2D9
:104D400059E063E288E20E9429340E94E64B6FE05A
:104D500085E090E074C085E096E00E9414388823D6
:104D600009F47CC00E94063544ED55E068E080E01F
:104D70000E9429340E94F1344FE956E064E189E051
:104D80000E94293449EA56E06EE189E00E94293404
:104D900044EB56E068E289E00E94293443EE54E097
:104DA0006CE389E00E94293489E090E00E94544835
:104DB0008A3041F08F3051F0853071F44FE356E086
:104DC00064E107C04FE356E06EE103C04FE356E0F5
:104DD00068E280E00E9429340E94E64B0E945E3522
:104DE000182F8823D9F364E071E08FE00E940D4B07
:104DF0000E940635113351F44AE059E063E288E23B
:104E00000E9429340E94E64B65E017C0123351F42A
:104E100047E159E063E288E20E9429340E94E64BB0
:104E20006AE00BC01333B1F445E259E063E288E273
:104E30000E9429340E94E64B6FE089E090E00E94D6
:104E4000404868EE73E080E090E00E94914D6BE096
:104E500075E0A7C3133209F0ADCBF9CF87E195E038
:104E60000E9414388823A9F10E9406354FEB56E0C2
:104E700068E080E00E9429340E94F13446EA55E05F
:104E800064E189E00E94293442ED56E06EE189E058
:104E90000E94293443EE54E06CE389E00E942934F7
:104EA0000E94E64B0E945E35182F8823D9F364E0F8
:104EB00071E08FE00E940D4B0E940635113319F40A
:104EC0006FED76E06EC3123309F0C0CC63EF76E08D
:104ED00068C38FED96E00E941438882309F495C0CA
:104EE0000E94063549EA55E068E080E00E942934D6
:104EF0000E94F13444E156E064E189E00E942934E3
:104F00004EE156E06EE189E00E94293449E256E024
:104F100068E289E00E94293444E356E062E389E0D4
:104F20000E94293443EE54E06CE389E00E94293466
:104F300086E090E00E9454488F3079F030F485305C
:104F4000B1F44FE356E064E10FC08E3151F08C3381
:104F500071F44FE356E062E307C04FE356E06EE1C1
:104F600003C04FE356E068E280E00E9429340E94CB
:104F7000E64B0E945E35182F8823D9F364E071E078
:104F80008FE00E940D4B0E940635113351F442E42C
:104F900056E063E288E20E9429340E94E64B65E015
:104FA00023C0123351F441E456E063E288E20E94E8
:104FB00029340E94E64B6FE017C0133351F44CE4E0
:104FC00056E063E288E20E9429340E94E64B6EE1DB
:104FD0000BC01433B1F447E556E063E288E20E9467
:104FE00029340E94E64B6CE386E090E00E94404842
:104FF00068EE73E080E090E00E94914D67E175E01B
:10500000D0C2133209F0D6CAF9CF83EF96E00E94DE
:105010001438882319F00E946C60C3C989E295E0B6
:105020000E941438882309F440C00E94063546E0E7
:1050300057E068E080E00E9429340E94F13446EA9B
:1050400055E064E189E00E94293444E157E06EE1D3
:1050500089E00E94293442EC55E068E289E00E9430
:10506000293443EE54E06CE389E00E9429340E9425
:10507000E64B0E945E35182F8823D9F364E071E077
:105080008FE00E940D4B0E940635113319F463E244
:1050900077E087C2123319F462E377E082C21333F8
:1050A00009F0D4CB62E477E07CC283E297E00E940F
:1050B0001438882309F488C00E94063549EA55E06F
:1050C00068E080E00E9429340E94F13444E156E017
:1050D00064E189E00E9429344EE156E06EE189E006
:1050E0000E94293449E256E068E289E00E942934AE
:1050F00044E356E062E389E00E94293443EE54E041
:105100006CE389E00E9429348BE090E00E945448CF
:105110008F3079F030F48530B1F44FE356E064E13C
:105120000FC08E3151F08C3371F44FE356E062E3DF
:1051300007C04FE356E06EE103C04FE356E068E27C
:1051400080E00E9429340E94E64B0E945E35182FB1
:105150008823D9F364E071E08FE00E940D4B0E9438
:105160000635113351F442E456E063E288E20E94CE
:1051700029340E94E64B65E024C0123351F441E427
:1051800056E063E288E20E9429340E94E64B6FE019
:1051900018C0133351F44CE456E063E288E20E94F5
:1051A00029340E94E64B6EE10CC0143309F01AC199
:1051B00047E556E063E288E20E9429340E94E64B0C
:1051C0006CE38BE090E003C182E397E00E94143827
:1051D000882309F488C00E94063547E157E068E05B
:1051E00080E00E9429340E94F13442E656E064E1F6
:1051F00089E00E9429344BE656E06EE189E00E9486
:10520000293445E756E068E289E00E94293440E805
:1052100056E062E389E00E94293443EE54E06CE3F7
:1052200089E00E9429348CE090E00E945448853047
:1052300079F030F48130B1F44FE356E064E10FC00F
:105240008A3051F08F3071F44FE356E062E307C0CB
:105250004FE356E06EE103C04FE356E068E280E0C2
:105260000E9429340E94E64B0E945E35182F882345
:10527000D9F364E071E08FE00E940D4B0E94063587
:10528000113351F44BE856E063E288E20E9429347E
:105290000E94E64B61E024C0123351F442E456E030
:1052A00063E288E20E9429340E94E64B65E018C060
:1052B000133351F444E956E063E288E20E94293452
:1052C0000E94E64B6AE00CC0143309F08BC041E445
:1052D00056E063E288E20E9429340E94E64B6FE0C8
:1052E0008CE090E074C082E497E00E941438882338
:1052F00009F47CC00E94063545EC55E068E080E08A
:105300000E9429340E94F1344FE956E064E189E0BB
:105310000E94293449EA56E06EE189E00E9429346E
:1053200044EB56E068E289E00E94293443EE54E001
:105330006CE389E00E9429348AE090E00E9454489E
:105340008A3041F08F3051F0853071F44FE356E0F0
:1053500064E107C04FE356E06EE103C04FE356E05F
:1053600068E280E00E9429340E94E64B0E945E358C
:10537000182F8823D9F364E071E08FE00E940D4B71
:105380000E940635113351F44AE059E063E288E2A5
:105390000E9429340E94E64B65E017C0123351F495
:1053A00047E159E063E288E20E9429340E94E64B1B
:1053B0006AE00BC01333B1F445E259E063E288E2DE
:1053C0000E9429340E94E64B6FE08AE090E00E9440
:1053D000404868EE73E080E090E00E94914D69E201
:1053E00075E0DFC0133209F0E5C8F9CF8FE695E02C
:1053F0000E941438882321F00E94BD5F0C94D121B3
:1054000086E795E00E941438882321F00E94D85E38
:105410000C94D12181E895E00E941438882351F141
:105420000E9406354CE457E068E080E00E94293491
:105430000E94F1344AE557E064E189E00E94293492
:1054400043EE54E06CE389E00E9429340E94E64B6D
:105450000E945E35182F8823D9F364E071E08FE055
:105460000E940D4B0E940635113309F0F5C969E61B
:1054700077E097C089E697E00E941438882309F402
:105480009AC00E9406354AE757E068E080E00E9433
:1054900029340E94F13446E857E064E189E00E9433
:1054A00029344DE857E06EE189E00E94293444E94F
:1054B00057E068E289E00E9429344BE957E062E353
:1054C00089E00E94293443EE54E06CE389E00E94B5
:1054D000293487E090E00E945448853099F030F4F8
:1054E0008230B1F44FE356E062E30FC08A3031F00E
:1054F000883C71F44FE356E064E107C04FE356E0A7
:105500006EE103C04FE356E068E280E00E94293478
:105510000E94E64B0E945E35182F8823D9F364E081
:1055200071E08FE00E940D4B0E940635113351F45B
:1055300043EA57E063E288E20E9429340E94E64B86
:1055400068EC23C0123351F44EEA57E063E288E27C
:105550000E9429340E94E64B6AE017C0133351F4CD
:1055600049EB57E063E288E20E9429340E94E64B4F
:1055700065E00BC01433D9F444EC57E063E288E2F1
:105580000E9429340E94E64B62E087E090E00E948E
:10559000404868EE73E080E090E00E94914D61E841
:1055A00075E088E59BE00E94DB420C94D121133228
:1055B00009F000C8F4CF80ED97E00E9414388823EA
:1055C00009F447C041EE57E06EE18EE10E942934B4
:1055D00040EF57E068E28AE00E9429340E94E64BDF
:1055E00089E1C82ED12C08EE13E02CE03DE046E026
:1055F0006BE380910B0D0E94F13C80910C0D90911A
:105600000D0D9827892798279093700980936F092B
:1056100080910E0D90910F0D9827892798279093D0
:105620006E0980936D098091100D9091110D98274E
:105630008927982790936C0980936B0964E670E042
:1056400080E090E00E94914D81E0C81AD10859F69F
:10565000A6CF8EE895E00E941438882311F40C94AC
:10566000D12186E30E944D4DBC01990F880B990B07
:105670000E948A6620E030E040EA50E40E94E96639
:1056800020E030E040E85AE30E94E96623ED3BE980
:105690004EE55EE30E9475682B013C0119A618A631
:1056A0001BA61AA61DA61CA68E010F5F1F4F22E087
:1056B00044E00E944863BC01CE0188960E94DB4210
:1056C000C301B2019CD1BC01CE0182960E94F83682
:1056D0008CA59DA5892B69F0C8A4D9A46EE270E0C1
:1056E000C6010E94626B009721F0BC016C197D0914
:1056F00002C06FEF7FEF6D5F7F4FCE0188960E94F3
:10570000E53663E070E0CE0182960E94E5361A82AB
:1057100019821C821B821E821D82BE01685D7F4F22
:10572000CE0101960E94F04263E078E0CE0101963E
:105730000E94B236BC01CE0188960E94F042CE0192
:1057400001960E9405431A8219821C821B821E82C6
:105750001D82BE016E5D7F4FCE0101960E94F04218
:1057600066E273E0CE0101960E94B236BC01CE0122
:1057700082960E94F042CE0101960E94054342E6C5
:1057800055E068E080E00E9429340E94F1348CE505
:105790009CE00E943634F092090DF0920A0DCE0181
:1057A00088960E94A9368CE893E00E943634A09235
:1057B000090DB0920A0DCE0182960E94A9360E9470
:1057C000E64B68EB7BE080E090E00E94914D67EF54
:1057D00074E088E59BE00E94DB42CE0182960E9445
:1057E0000543CE0188960E9405430C94D121AD96C5
:1057F0000FB6F894DEBF0FBECDBFDF91CF911F91E2
:105800000F91FF90EF90DF90CF90BF90AF909F905F
:105810008F907F906F905F904F903F900895CF92C0
:10582000DF92EF92FF920F931F93CF93DF936C0160
:10583000EB017B01E40EF51E00E010E0CE15DF0564
:1058400061F06991D601ED91FC910190F081E02D1C
:10585000C6011995080F191FF1CFC801DF91CF912B
:105860001F910F91FF90EF90DF90CF9008950895D2
:1058700080E090E00895CF92DF92EF92FF920F9335
:105880001F93CF93DF938C3699F03CF48236B1F0BE
:105890008736B9F410E0DFEF13C0873739F0893766
:1058A00049F0823771F410E0D0E006C01FEF03C06A
:1058B00010E005C010E0DFEFCFEF03C01FEFD0E036
:1058C000C0E085E0C82ED12CE12CF12C012F2D2F2A
:1058D0004C2FB70182EE9BE00E9416472D2F4C2FD4
:1058E000B7018DEC9BE00E94164782EE9BE00E9480
:1058F00067478DEC9BE00E9467476AE070E080E0BC
:1059000090E00E94914D00E020E040E0B70182EE7F
:105910009BE00E94164720E040E0B7018DEC9BE041
:105920000E94164782EE9BE00E9467478DEC9BE049
:105930000E9467476AE070E080E090E00E94914D2D
:105940008FEFE81AF80A88E0E816F10409F0BECFF4
:10595000E12CF12C012F2D2F4C2FB70182EE9BE073
:105960000E9416472D2F4C2FB7018DEC9BE00E9413
:10597000164782EE9BE00E9467478DEC9BE00E94F9
:1059800067478FEFE81AF80A88E0E816F10411F784
:1059900081E0C81AD10809F097CFDF91CF911F910C
:1059A0000F91FF90EF90DF90CF9008950F931F938A
:1059B000CF93DF93EC018C010C5F1F4FFC01E95882
:1059C000FF4F0190F081E02DC80119958E3F2FEF18
:1059D000920770F4FE01E658FF4FC758DF4F9C0155
:1059E00040816881C8010E94493A9881890F888363
:1059F00081E090E0DF91CF911F910F9108958F92F8
:105A00009F92AF92BF92CF92DF92EF92FF924B01A3
:105A10005C0120E030E040E151E40E940E6918167C
:105A20006CF420E030E04CE151E4C501B4010E9487
:105A3000106828E636E646E350E416C020E030E081
:105A400040EC50E4C501B4010E940E691816B4F48C
:105A500020E030E040ED50E4C501B4010E94106840
:105A600020E333E343EF5FE30E94756820E030E01A
:105A700048EC52E40E94E9666B017C0120E030E0D2
:105A800048EC52E4C701B6010E940E6918166CF08A
:105A900020E030E0A901C701B6010E94846687FFBB
:105AA0000AC0C12CD12C760106C0C12CD12C88ECA7
:105AB000E82E82E4F82EC701B6010E94DD68CB0112
:105AC000FF90EF90DF90CF90BF90AF909F908F901E
:105AD0000895EF92FF920F931F93CF93DF93823736
:105AE000B1F03CF4873669F08C36A1F410E0D0E0D8
:105AF0000AC0873721F0893769F410E006C01FEF2C
:105B000004C010E0DFEFC0E005C0DFEF02C010E02E
:105B1000D0E0CFEFE12CF12C012F2D2F4C2FB7012E
:105B200082EE9BE00E9416472D2F4C2FB7018DEC83
:105B30009BE00E94164782EE9BE00E9467478DEC37
:105B40009BE00E9467478FEFE81AF80A88E0E816A2
:105B5000F10411F7DF91CF911F910F91FF90EF901A
:105B60000895CF93DF9388E090E00E94544890918D
:105B70008E0C81110BC090FF1DC0809150098230A6
:105B8000C9F082E08093500982E721C08091840CA3
:105B900090FF20C080FD20C0909150099230D1F03C
:105BA000C091BF09D091C0092196D093C009C0937C
:105BB000BF0960C08091840C80FF83C08091500930
:105BC000813009F47EC081E08093500982E6DF9144
:105BD000CF9151CE80FD40C01092C0091092BF09F4
:105BE0001092BE091092BD0980E03AD624E140E847
:105BF00062E380E00E94564B0E94E64B81E030D683
:105C000088E090E00E94544890E02091BF093091D4
:105C1000C009281739074CF082E08093500982E7C9
:105C20002ADE1092C0091092BF0988E090E00E941D
:105C3000544890E02091BD093091BE0928173907DA
:105C40000CF43FC081E08093500982E614DE10928C
:105C5000BE091092BD0935C080915009813009F408
:105C6000BBCFC091BD09D091BE092196D093BE098A
:105C7000C093BD0988E090E00E9454488A30B9F48E
:105C8000CC0F4C2F440F440F4C0F24E162E38AE009
:105C900009C0853049F444E1C49F402D112424E11A
:105CA00062E38FE00E94564B0E94E64BA9CF8F30F3
:105CB00081F74C2F440F4C0F440F24E162E384E141
:105CC000F1CFDF91CF9108957F928F929F92AF9203
:105CD000BF92CF92DF92EF92FF920F931F93CF93D9
:105CE000DF9380E0BDD529E140E864E180E00E94D7
:105CF000564B81E0B5D545E058E068E080E0A9D595
:105D000070D687E797E2B2D509E01DE08EE0F80192
:105D10008083CAE0DDE08DE2782E788280915A0996
:105D200090915B09A0915C09B0915D09C090460912
:105D3000D0904709E0904809F0904909BC01CD0195
:105D40006C197D098E099F0928EE822E23E0922E80
:105D5000A12CB12CA50194010E94DF6780914A0912
:105D600090914B09821B930B68E572E00E943269A7
:105D700080E99CE056D687E2F801808378828091A2
:105D80005A0990915B09A0915C09B0915D09C0909E
:105D90004609D0904709E0904809F0904909BC01B4
:105DA000CD016C197D098E099F09A50194010E94FE
:105DB000DF6780914A0990914B09821B930B3CE36A
:105DC000C32ED12CB6010E943269CB014AE0E42EE9
:105DD000F12CB7010E943269BC0180E99CE021D618
:105DE0004CEA54E06AE28AE334D586E4F801808321
:105DF000788280915A0990915B09A0915C09B091D9
:105E00005D09209146093091470940914809509118
:105E10004909BC01CD01621B730B840B950BA501D5
:105E200094010E94DF6780914A0990914B09821B7F
:105E3000930BB6010E943269B7010E94326980E972
:105E40009CE0EFD58FE5F8018083788280915A0934
:105E500090915B09A0915C09B0915D0900914609A0
:105E6000109147092091480930914909BC01CD01A1
:105E7000601B710B820B930BA50194010E94DF67DD
:105E800080914A0990914B09821B930BB6010E94A5
:105E90003269B7010E943269BC0180E99CE0C1D53A
:105EA0000E94E64B8CE893E0DF91CF911F910F9118
:105EB000FF90EF90DF90CF90BF90AF909F908F902A
:105EC0007F90D4C40F931F93CF93DF93C8E0DCE09F
:105ED00019861C8680914E0990914F0968EE73E0F7
:105EE0000E943269CE019DD581E0898780914E095B
:105EF00090914F0964E670E00E943269CE0191D51D
:105F000082E0898780914E0990914F090AE010E064
:105F1000B8010E943269CE0184D583E089878091DF
:105F20004E0990914F09B8010E943269BC01CE011F
:105F3000DF91CF911F910F9174C50F931F93CF9352
:105F4000DF93C7EFDBE019861C8680914C099091A6
:105F50004D0968EE73E00E943269CE0162D581E09E
:105F6000898780914C0990914D0964E670E00E9408
:105F70003269CE0156D582E0898780914C09909193
:105F80004D090AE010E0B8010E943269CE0149D5FE
:105F900083E0898780914C0990914D09B8010E9456
:105FA0003269BC01CE01DF91CF911F910F9139C5AC
:105FB0002DD549E453E068E080E04BD412D58CE560
:105FC0009CE054D448E753E06EE18AE042D40E945A
:105FD000E64B8CE893E04AD489E77BDD10920A0215
:105FE000109245090C94E64B85E198E054D50ED506
:105FF00090913B0980916909992399F0882351F088
:1060000045E258E068E088E224D44EE258E062E1DC
:1060100080E204C04AE358E062E18BE11AD40C94B8
:10602000E64B49E453E068E0882359F080E011D45E
:10603000D8D48CE59CE01AD440EE53E06EE18EE1BA
:106040000AC080E006D4CDD48CE59CE00FD44AE7AA
:1060500053E06EE187E1FDD30E94E64B8CE893E0CC
:1060600005C48F929F92AF92BF92CF92DF92EF9230
:10607000FF920F931F93CF93DF930E94C94D6B0143
:106080007C016093B9097093BA098093BB0990931E
:10609000BC098091B5099091B609A091B709B0915A
:1060A000B80946015701881A990AAA0ABB0A209121
:1060B000550930E02F5F3F4F032E000C440B550B6A
:1060C00066E470E080E090E00E94DF67821693064D
:1060D000A406B50608F47BC080915109909152093D
:1060E0000197D0916209CB9788F080913509909102
:1060F00036090197CB9750F0D11108C08091630900
:10610000811104C08091B409811157C0C091B309B5
:10611000C11102C081E003C0C73019F48FEF809332
:106120000D026D2F70E080E090E00E948A6620E012
:1061300030E040E750E40E940E6918164CF0809160
:106140006309BB24BA94811104C0DD2321F001C08E
:10615000B12C1FEF01C010E080910D02C80FC09359
:10616000B30982EE9BE00E94CC468DEC9BE00E943E
:10617000CC4682EE9BE00E9467478DEC9BE00E943C
:106180006747D0E000E02B2D412FBE0182EE9BE05F
:106190000E9416472B2D412FBE018DEC9BE00E94E3
:1061A000164782EE9BE00E9467478DEC9BE00E94C1
:1061B000674781E08093B40902C01092B409C0928D
:1061C000B509D092B609E092B709F092B809DF910B
:1061D000CF911F910F91FF90EF90DF90CF90BF90E4
:1061E000AF909F908F9008950F931F93CF93DF935D
:1061F00080915309909154099C01215031092B330E
:10620000310578F51092110C11E01093140CCAE0CE
:10621000D0E0BE010E94326988E09CE002D4109375
:10622000110C8091530990915409BE010E9432696A
:10623000BC0188E09CE0F5D382E08093110C809152
:10624000070290910802BE010E94326988E09CE03A
:10625000E8D383E08093110C8091070290910802AB
:106260003FC0181619060CF046C01092110CC1E080
:10627000C093140C68E572E00E94326988E09CE0EB
:10628000D0D3C093110C80915309909154090CE321
:1062900010E0B8010E943269CB01CAE0D0E0BE0133
:1062A0000E943269BC0188E09CE0BBD382E080930D
:1062B000110C8091530990915409B8010E943269E0
:1062C000BE010E94326988E09CE0ABD383E08093FA
:1062D000110C8091530990915409B8010E943269C0
:1062E000BE010E943269BC0188E09CE0DF91CF9141
:1062F0001F910F9196C3DF91CF911F910F91089538
:106300000F931F93CF93DF938091350990913609B6
:106310009C01215031091092000C2B33310568F596
:1063200011E01093030CCAE0D0E0BE010E94326974
:1063300087EF9BE076D31093000C80913509909104
:106340003609BE010E943269BC0187EF9BE069D328
:1063500082E08093000C8091070290910802BE01B8
:106360000E94326987EF9BE05CD383E08093000C4E
:10637000809107029091080239C0C1E0C093030CDC
:1063800068E572E00E94326987EF9BE04AD3C093D0
:10639000000C80913509909136090CE310E0B801AA
:1063A0000E943269CB01CAE0D0E0BE010E9432698E
:1063B000BC0187EF9BE035D382E08093000C809195
:1063C000350990913609B8010E943269BE010E94D8
:1063D000326987EF9BE025D383E08093000C8091A6
:1063E000350990913609B8010E943269BE010E94B8
:1063F0003269BC0187EF9BE0DF91CF911F910F9134
:1064000010C360E177E280E090E00E94914DFED2FF
:1064100041E055E068E081E01CD2E3D28CE59CE0ED
:1064200025D248E253E06EE18EE113D20E94E64BA2
:106430008CE893E01BD21092550910926A0981E012
:106440008093060210924509109262091092690920
:1064500080930A021092440961E08AE10E94B34CE1
:1064600010925A0910925B0910925C0910925D0912
:106470001092460910924709109248091092490952
:1064800084E690E090930802809307021092370907
:10649000109238091092390910923A091092110C91
:1064A00062E173E088E09CE0BAD22ADF9DCEEF92F1
:1064B000FF920F93CF93DF9360E971E080E090E06B
:1064C0000E94914D1092110C1092140C68E478E027
:1064D00088E09CE0A4D29AD28CE59CE0C7D14DE440
:1064E00058E063E284E1B5D148E558E062E38DE22B
:1064F000B0D10E94E64B8CE893E0B8D166E071E041
:106500008FE00E940D4B89E1E82EF12CC0E0D0E035
:1065100000E020E04FEFBE0182EE9BE00E941647B4
:1065200020E04FEFBE018DEC9BE00E94164782EE0B
:106530009BE00E9467478DEC9BE00E9467476AE002
:1065400070E080E090E00E94914D20E040E0BE01CC
:1065500082EE9BE00E94164720E040E0BE018DECF9
:106560009BE00E94164782EE9BE00E9467478DECFD
:106570009BE00E9467476AE070E080E090E00E9444
:10658000914D2196C830D10519F681E0E81AF1083D
:1065900009F0BCCFDF91CF910F91FF90EF9031CFF9
:1065A000EF92FF920F93CF93DF931092110C109202
:1065B000140C6DE578E088E09CE031D227D28CE5C0
:1065C0009CE054D142E658E064E18EE142D14DE4D2
:1065D00058E063E284E13DD148E558E062E38DE2B2
:1065E00038D10E94E64B8CE893E040D165E071E041
:1065F0008FE00E940D4B89E1E82EF12CC0E0D0E045
:106600000FEF20E040E0BE0182EE9BE00E941647C3
:1066100082EE9BE00E94674720E040E0BE018DECE7
:106620009BE00E9416478DEC9BE00E9467476AE062
:1066300070E080E090E00E94914D00E020E040E0BA
:10664000BE0182EE9BE00E94164782EE9BE00E9414
:10665000674720E040E0BE018DEC9BE00E941647BA
:106660008DEC9BE00E9467476AE070E080E090E07C
:106670000E94914D2196C830D10511F681E0E81AAB
:10668000F10809F0BBCFDF91CF910F91FF90EF9010
:10669000B8CE96E0899FD0011124A25AB44F9096AB
:1066A0007C936E935F9791E091969C9391979091D4
:1066B000CA0BE091CB0BF091CC0B992339F03097BA
:1066C00051F0811108C080917A0B04C0309719F005
:1066D0005C968C9119940895FF920F931F93CF931A
:1066E000DF93C82FD62F1092A90C8A01F12CF80144
:1066F00061918F01E091960CF091970C84E99CE0F8
:1067000019958F3FFFEF9F07E1F08E3F2FEF920724
:1067100071F39C014D2F6C2F84E99CE0BAD69091C7
:10672000E80C913049F030F0923041F0933039F478
:10673000D81B05C0C80F03C0D80F01C0C81BF80E76
:10674000D6CF8F2DDF91CF911F910F91FF9008959C
:106750000F931F93CF93DF93C82FD62F86E0C89F48
:10676000F0011124E25AF44F11A2878D90A18130DB
:106770009105D1F040F082309105A1F10397E1F548
:1067800060E070E033C06623B9F161E070E08C2F07
:1067900080DF0E94C94D6093B60B7093B70B809356
:1067A000B80B9093B90B28C00E94C94D0091B60B4D
:1067B0001091B70B2091B80B3091B90BAB01BC0114
:1067C000401B510B620B730B8091C80B9091C90B4E
:1067D000A0E0B0E084179507A607B70718F462E0B9
:1067E00070E004C0D11108C063E070E08C2FDF912D
:1067F000CF911F910F914DCFDF91CF911F910F91AD
:106800000895CF938091060D81110E94F84B80E08E
:106810000E94EC4B84E99CE00E94874BC091CC0C19
:106820008091CB0CC80FE091940CF091950C81896C
:10683000C81740F084E99CE00E947D4B80E0CF9136
:106840000C94EC4B8091060D81110E94F84B8C2F1B
:10685000DFCF2FEF30E43093970C2093960C3CCF92
:10686000833008F081E08093050D0895CF93DF9386
:106870002091D80C3091D90C2817390709F4A7C0FA
:10688000EC019093D90C8093D80CFC0184918093F7
:10689000E90C3196E491E093EA0CFE013296E49122
:1068A000E093EB0CFE013396E491E093EC0CFE01D7
:1068B0003496E491E093ED0CFE013596E491E0937B
:1068C000EE0CFE013696E491E093EF0CFE01379654
:1068D000E491E093F00CFE013896E491E093F10C22
:1068E000FE013996E491E093F20CFE013A96E491B0
:1068F000E093F30CFE013B96E491E093F40CFE016F
:106900003C96E491E093F50CFE013D96E491E09312
:10691000F60CFE013E96E491E093F70CFE013F96E3
:10692000E491E093F80CFE017096E491E093F90C89
:1069300061E1CE0119D79093FB0C8093FA0C63E1CF
:10694000CE0112D79093FD0C8093FC0C65E1CE0133
:106950000BD79093FF0C8093FE0C8091D80C9091F4
:10696000D90C892BA1F18091F60C8093010D4091F7
:10697000F70C4093020D9091000D992341F1913055
:1069800069F49091F80C891714F49093010D80919B
:10699000F90C8417E4F48093020D19C03091F30CC4
:1069A0002091F50C082E000C990B622F022E000C82
:1069B000770B630F711D37FD7A95861797071CF4C7
:1069C000320F3093010D241714F42093020DDF9140
:1069D000CF910895462F50E060E070E02AE00C94DB
:1069E0001F430F930AE025EB49E061E084E99CE056
:1069F0000E94C643882341F000E024EB49E061E0B7
:106A000084E99CE00E94EC430F9108951092090DD7
:106A100010920A0D1092A90CF4DE0C94F84B0C9411
:106A20000A43CF92DF92EF92FF920F931F93CF937F
:106A3000DF936B01770FEE08FF08F7FE1FC0EC0134
:106A4000E881F9810190F081E02D6DE219958C01CA
:106A500044275527BA014C195D096E097F092AE0C0
:106A6000CE010E941F43800F911FDF91CF911F9194
:106A70000F91FF90EF90DF90CF9008952AE0B7013B
:106A8000A601DF91CF911F910F91FF90EF90DF90C2
:106A9000CF900C941F43CF93DF93BC018FEA9AE011
:106AA0000E940A43EC016AE678E08FEA9AE00E94CD
:106AB0000A438C0F9D1FDF91CF9108956F927F92B3
:106AC0008F929F92AF92BF92CF92DF92EF92FF92FE
:106AD0000F931F93CF93DF9381E08093CA0B0E94A3
:106AE000C94D0091BA0B1091BB0B2091BC0B30919A
:106AF000BD0BAB01BC01401B510B620B730B8091B2
:106B0000C60B9091C70BA0E0B0E084179507A607CD
:106B1000B70708F0E6C0C0E08091C40BC81730F09A
:106B2000712C812C912C5401839440C0E091C00BB6
:106B3000F091C10BEC0FF11D62E080810E94114DBC
:106B4000CF5FEACFC62DD0E0E091C00BF091C10B32
:106B5000EC0FFD1F80810E948B4C2496CC0FDD1F13
:106B6000C25AD44F892B09F04BC0888199818C2956
:106B70009D299983888363948091C40B681610F3D0
:106B8000E091C20BF091C30BE00FF11F61E0808137
:106B90000E94B34C8091C20B9091C30BFC01E00F9B
:106BA000F11F60E080810E94114D73948091C50BAC
:106BB000781658F5072D10E0E091C20BF091C30B49
:106BC000E00FF11F61E080810E94114DE091C20B46
:106BD000F091C30BE00FF11F60E080810E94B34C85
:106BE000D501C401072C04C0880F991FAA1FBB1F21
:106BF0000A94D2F76C017C01E094F094612CBCCF34
:106C0000888199818E219F21B4CF2EE5E22E2BE041
:106C1000F22EF7018FEF9FEF278D30A1232B21F468
:106C2000148E968F858F11A236962BE0EA39F207E3
:106C300099F7C0E096E0D92E8091C40BC81758F59B
:106C4000D0E00C2F10E0000F111F0A59144F2091B3
:106C5000C50BD217F0F4F801408151810D2E02C00E
:106C6000569547950A94E2F7642F6170C29F900190
:106C700011242D0F311DEEE5FBE080E0A58DB68DD2
:106C80002A173B0709F44DC08F5F36968A30B1F75B
:106C90002CC0CF5FD1CFC0E0F70181A18111C1E04D
:106CA000F6E0EF0EF11C2AE9E2162BE0F206A1F75E
:106CB0000E94C94D6093BA0B7093BB0B8093BC0BC1
:106CC0009093BD0BCC2369F080917F0B882349F012
:106CD00080917D0B90917E0B019719F480917A0B36
:106CE00029C01092CA0B80E025C040FF1BC0EEE512
:106CF000FBE080E090E0448D411116C0E091BE0BB6
:106D0000F091BF0BE20FF31F4081D89EF001D99E96
:106D1000F00D1124E25AF44F448F368F258F10A2C4
:106D2000178E16DDDF5F93CF019636968A30910578
:106D300011F7F8CFDF91CF911F910F91FF90EF9056
:106D4000DF90CF90BF90AF909F908F907F906F908B
:106D50000895FC01448155816081718180E99CE046
:106D60000C940F2CEF92FF920F931F93CF93DF930E
:106D7000EC017B0161157105E9F0FB010190002038
:106D8000E9F73197E61BF70BC1F00C811D810E0F5F
:106D90001F1FB8010E948342882361F02881398136
:106DA0008C819D81B701820F931F0E94766B1D839A
:106DB0000C8303C0CE010E94AA42CE01DF91CF9185
:106DC0001F910F91FF90EF900895DC0114968D9123
:106DD0009C9115976817790750F4ED91FC911197E4
:106DE000E60FF71F15967C936E9314971082089503
:106DF0000F931F93CF93DF93CDB7DEB762970FB694
:106E0000F894DEBF0FBECDBF8C01CB01F80111821B
:106E1000108213821282158214824AE0BE016F5FD3
:106E20007F4F0E940364BE016F5F7F4FC8010E94C5
:106E3000DB4262960FB6F894DEBF0FBECDBFDF9186
:106E4000CF911F910F9108955F926F927F928F92D1
:106E50009F92AF92BF92CF92DF92EF92FF920F93E9
:106E60001F93CF93DF93A82EC62FD42F6801B62E81
:106E7000B20E742E780E0B2D272D462F682F84E925
:106E80009CE00E94C643882309F442C0D95FD6958E
:106E9000D695D695ED2EF12CBC1609F439C05524A3
:106EA00053945C0E052D272D4C2F6A2D84E99CE010
:106EB0000E94C643882341F16090050D4601DA2DFA
:106EC00011E07D16F9F0F4018491812319F06092AC
:106ED000050D09C08091040D81110DC081E0611084
:106EE00080E08093050D00E021E04C2F6D2F84E9B8
:106EF0009CE00E94EC43DF5F110F19F7FFEF8F1A40
:106F00009F0ADECF6092050DCE0CDF1CC52DC4CFCD
:106F1000DF91CF911F910F91FF90EF90DF90CF9075
:106F2000BF90AF909F908F907F906F905F900895EB
:106F30000F931F93CF93DF9300D01F92CDB7DEB78F
:106F40008C0119821A821B821C8220E044E050E0EE
:106F5000BE016F5F7F4F0E94ED44F80111860F90D4
:106F60000F900F900F90DF91CF911F910F91089587
:106F7000282F30910B0A313208F04AC08091E7097E
:106F80008111FCCF90910A0A42E04093E7092093D7
:106F9000E6092FEF2093E5091092E4093093E30905
:106FA000EAEEF9E0A3ECB9E020E0321721F04191DC
:106FB0004D932F5FFACF1092C2092091C209990F09
:106FC000922B9093C2099091C109913061F4109273
:106FD000C1099091C2099093BB009091BC0093FDB0
:106FE000F8CF95EC01C095EE9093BC009091E70925
:106FF0009230E1F39091E5099F3F79F08091E509A6
:10700000803241F08091E509803331F084E005C0A1
:1070100081E003C082E001C083E01092E909109290
:107020000B0A1092E8090895FC0180915C0B909185
:107030005D0B892B21F421E0309749F413C0809136
:10704000580B9091590B309731F421E0FC0180816D
:10705000882341F006C0BF010E946D6B21E0892B9F
:1070600009F020E0822F0895CF93DF93EC01698728
:1070700018860E94C344882319F088858360888716
:107080000E94C94D6A837B838C839D83DF91CF915E
:107090000895213039F020F0223031F4861B089514
:1070A000860F0895841B0895840F0895213039F0C8
:1070B00020F0223031F4841B0895840F0895860F48
:1070C0000895861B0895DC0118964C911897ED9150
:1070D000FC911197249130E0042E02C0359527953C
:1070E0000A94E2F7842F860F883010F4E22F0DC047
:1070F00031961196FC93EE93E49198E0941B01C0B5
:10710000EE0F9A95EAF7E22B885018968C9381E05F
:1071100090E001C0880F6A95EAF781508E230895A8
:1071200085ED8093BC008091BC0084FDFCCF109263
:10713000E709089540914C0A262F30E0240F311DB5
:1071400021323105DCF42091E7092430C9F4FC0137
:1071500080E090E0861758F430914C0A2191DC01D0
:10716000A45DB54FA30FB11D2C930196F3CF809171
:107170004C0A680F60934C0A80E0089581E00895FE
:1071800082E00895089508950895E0911F11809177
:107190001E11E81730F4F0E0E45FF54F808190E0D5
:1071A00008958FEF9FEF089590911F1180911E1108
:1071B000981750F4E92FF0E0E45FF54F208130E0BC
:1071C0009F5F90931F1102C02FEF3FEFC9010895F9
:1071D00080911E1190E020911F11821B910908954A
:1071E000CF92DF92EF92FF920F931F93CF93DF9393
:1071F0007C01CB018A012091E809222389F0EB016F
:107200006B01C40ED51ECC15DD0561F06991D70167
:10721000ED91FC910190F081E02DC7011995F3CF1C
:10722000642F88DFC801DF91CF911F910F91FF90EC
:10723000EF90DF90CF900895CF93DF931F92CDB75B
:10724000DEB769832091E8092223D1F020910B0A4F
:10725000203240F021E030E0FC013383228380E0E3
:1072600090E014C08091E909E82FF0E0E651F64F74
:10727000998190838F5F8093E90980930B0A04C002
:1072800061E0CE01019656DF81E090E00F90DF9142
:10729000CF9108955F926F927F928F929F92AF925B
:1072A000BF92CF92DF92EF92FF920F931F93CF93F3
:1072B000DF935C01F62E642EEC01C85BDF4F1C816E
:1072C000DD804C0181E7880E911CEE80E11ACF2C05
:1072D000EF1408F4CE2C5B800C85202F4D2D612FF0
:1072E0008A81D7DE782E202F4D2D612F852DDEDE71
:1072F000482F662011F08A8504C0898581110AC053
:107300008B85F4018083CC2029F02C2D672DC501BD
:107310000E94EC43FE1420F0FE18D39410E0D5CF69
:107320001F0D1C83DD82DF91CF911F910F91FF9084
:10733000EF90DF90CF90BF90AF909F908F907F9015
:107340006F905F900895FC01962F6831A9F0B90104
:10735000993148F4943161F0973141F550E08CE473
:107360009BE03EDF07C09931F1F0903219F01EC06A
:107370000E94E14C81E00895A081B1811D968C911D
:10738000843018F08CE08093B800828990E0959565
:10739000879591E09093E80980930A0A1092E90991
:1073A00010920B0AE7CF81E0E3DDE4CF80E008959F
:1073B0000F931F93CF93DF93EC01862F642F8C32B2
:1073C00070F48A3208F05DC0883289F0893209F0A1
:1073D00042C070E080E090E00E94914D52C08D323A
:1073E000D1F0C8F194EB980F923020F134C08E01A7
:1073F000055E1F4FD0E0F80181918F018F3F39F07A
:10740000D03110F461E001C062E00E94114DDF5FF5
:10741000D63189F736C0433018F082E090E002C0E0
:1074200085E090E0880F991F880F991F05970197B5
:10743000F1F727C08F73C80FD11D411107C061E05C
:107440008B8D0E94114D60E08B8D11C062E08B8DA1
:107450000E94114D16C08034B0F0982F9F73FE012A
:10746000E90FF11D838D8F3F61F0903118F40E9478
:10747000B34C07C00E948B4C21E0892B09F420E01B
:107480002E8B81E001C080E0DF91CF911F910F91A1
:1074900008956F927F928F929F92AF92BF92CF92F8
:1074A000DF92EF92FF920F931F93CF93DF93EC0144
:1074B000E62EF42E8901FC01EC5AFF4F80818130C9
:1074C000C9F070F0823001F1833039F5FE01EA5BDA
:1074D000FF4F0190F081E02DCE011995E80E1DC0FF
:1074E000FE01EA5BFF4F0190F081E02DCE0119957E
:1074F000F80E13C0FE01EA5BFF4F0190F081E02D12
:10750000CE011995E81A09C0FE01EA5BFF4F019010
:10751000F081E02DCE011995F81AFE01E65BFF4FD0
:10752000E0823196F08237978081918147960F3FB4
:10753000110509F020F50136110510F0B49606C0CA
:107540000134110538F0FE01EA59FF4F20813181E5
:10755000820F931F9C012F5F3F4FF90144914423F9
:1075600009F4F1C0FC01449150E00417150711F42F
:10757000029623C0F9012491820F911DEBCFFE01E9
:10758000E659FF4F20813181820F931FFC01249126
:1075900030E0322F22273196E4912E2B2115310530
:1075A00009F4D1C00217130711F4039606C0FC01B9
:1075B0003296E4918E0F911DE9CF009709F4C3C074
:1075C0007E01F8E4EF0EF11CF701918380831086B1
:1075D00071966081C70177DDF701868372966081BD
:1075E000C70171DDD82EF70187835E01F1E7AF0E89
:1075F000B11CF5019081F701928781E0911180E043
:10760000F7018387FE01E55AFF4F1081612FC70103
:107610005ADD9FEF910F01E010E0980101C0220FA9
:107620009A95EAF7782E721AFE01E45AFF4FC0804D
:107630006C2DC70148DDCA94480101C0880CCA946A
:10764000EAF7682E6D0CFE01E35AFF4FC0806C2DE7
:10765000C70139DDCA9401C0000FCA94EAF7C82EE9
:10766000C01AF701068110160CF06EC094848618BB
:10767000292D482D672D82810CDD182FF70182837B
:10768000292D482D672D838111DDF7018383F1E0DA
:107690009F16B1F09F1678F022E09216B9F093E0B1
:1076A00099121FC0212F2D0D982F901B01E0080F5C
:1076B00081E0890F18C0202F210F082F0D0D13C056
:1076C0009D1821E0210F080F190D0DC091E0392FF1
:1076D000301B21E0210F9D1901E0080F890F130FC6
:1076E00002C0082F212F482F612FCE010E94C643D0
:1076F000882351F1F701148215828E01095A1F4F18
:107700004E01F8E58F0E911CF8016081C701DBDCAA
:10771000682EF4016081C701D6DC782E40E0662D2A
:10772000CE01B8DD41E0672DCE01B4DD61E0C701D7
:10773000CADC8111F3CFF70185818D152CF3828589
:10774000F501808301C0C12C8C2DDF91CF911F9159
:107750000F91FF90EF90DF90CF90BF90AF909F90F0
:107760008F907F906F900895FC01E60FF11D84913A
:1077700090E0982F88273196E4918E0F911D0895FF
:107780001F920F920FB60F9211240BB60F922F93E8
:107790003F934F935F936F937F938F939F93AF9399
:1077A000BF93EF93FF938091B900887F803609F4EF
:1077B0009CC068F5883209F45BC090F4803109F40C
:1077C00054C038F4882309F4F6C0883009F44DC059
:1077D000F5C0883109F44CC0803209F45DC0EEC0B8
:1077E000803409F468C048F4803309F455C0883304
:1077F00009F0E4C08093E509D8C0803509F44FC092
:10780000883509F45DC0883409F0D8C0D6C08839FD
:1078100009F4C7C0A8F4883709F467C038F488367B
:1078200009F463C0803709F460C0C8C0883809F41F
:10783000B8C0803909F45FC0803809F0BFC05BC0B0
:10784000803B09F486C038F4803A09F466C0883A6F
:1078500009F47FC0B3C0803C09F4A7C0883C09F498
:10786000A4C0883B09F48AC0A9C08091C20910C095
:107870009091E4098091E309981770F5E091E4098B
:1078800081E08E0F8093E409F0E0ED53F64F8081A4
:107890008093BB0085EC86C08093E5098EC0E091A3
:1078A000E40981E08E0F8093E4098091BB00F0E051
:1078B000ED53F64F80839091E4098091E3096EC007
:1078C000E091E40981E08E0F8093E4098091BB0090
:1078D000F0E0ED53F64F80838091E60981116DC091
:1078E00081E08093C10984EA61C083E08093E70965
:1078F00010926E0ACFCF80916E0A803208F051C08C
:10790000E0916E0A81E08E0F80936E0A8091BB0039
:10791000F0E0E25BF54F8083BDCF85EC8093BC0047
:107920001092E70980916E0A803230F4E0916E0A7D
:10793000F0E0E25BF54F108260916E0A70E0E0913A
:107940001A11F0911B118EE49AE0199510926E0AAB
:1079500035C084E08093E70910924D0A10924C0ADA
:10796000E0911C11F0911D11199580914C0A811123
:1079700005C081E080934C0A10922C0AE0914D0AD8
:1079800081E08E0F80934D0AF0E0E45DF54F808139
:107990008093BB0090914D0A80914C0A981708F48F
:1079A00079CF85E88093BC0009C085EC8093BC004A
:1079B0001092E70903C01092E509B2DBFF91EF9145
:1079C000BF91AF919F918F917F916F915F914F91F7
:1079D0003F912F910F900BBE0F900FBE0F901F90F5
:1079E00018952F923F924F925F926F927F928F9253
:1079F0009F92AF92BF92CF92DF92EF92FF920F933E
:107A00001F93CF93DF93CDB7DEB728970FB6F894C7
:107A1000DEBF0FBECDBFD82EC62E4F8349010E94B8
:107A2000C94D2B013C012D2C220CE12C1886FF2482
:107A3000F3942F81A22EB12C33243A94C801A0E0F4
:107A4000B0E08B839C83AD83BE839F81E91608F0F1
:107A500082C0F092E809D0920A0A1092E9091092C5
:107A60000B0A6C2D8CE49BE0E7DB81E081DAF0927D
:107A7000E809D0920A0A1092E90910920B0A809143
:107A8000E7098111FCCFC5018E1991098132910559
:107A900014F080E290E0813208F080E2F092E70991
:107AA000F092E6093092E5091092E4099FEF980FF1
:107AB0009093E309F092C2099091C20992299093A0
:107AC000C2099091C109913071F41092C10990914D
:107AD000C2099093BB009091BC0093FDF8CFA5EC38
:107AE000A093BC0003C0B5EEB093BC009091E70931
:107AF0009130E1F39091E409981710F48091E40932
:107B0000E3ECF9E0ACE0BAE090E0981721F02191C5
:107B10002D939F5FFACF10921F1190931E11909199
:107B20001E1180911F11981709F446C00115110507
:107B300089F10E94C94DDC01CB0184199509A60980
:107B4000B7092B813C814D815E8182179307A40781
:107B5000B50700F131C001151105A1F10E94C94D11
:107B6000DC01CB0184199509A609B70920E030E0B2
:107B700080179107A207B30728F14F81242F30E027
:107B80005885852F550F990B82179307DCF48FEFDB
:107B9000888718C0D401E885AE0FB11DE7FDBA95FE
:107BA000BA83A9838CE49BE0FFDAA981BA818C9324
:107BB000B885BF5FB887B3CF8F81813208F080E28C
:107BC000E80E43CF888528960FB6F894DEBF0FBE27
:107BD000CDBFDF91CF911F910F91FF90EF90DF907C
:107BE000CF90BF90AF909F908F907F906F905F905D
:107BF0004F903F902F900895BF92CF92DF92EF92D7
:107C0000FF920F931F93CF93DF931F921F92CDB7D5
:107C1000DEB7F82EE62EC42EB22ED02E08EE13E0DC
:107C20009E012E5F3F4F41E0DCDE882341F14C2D69
:107C300050E04B1951094F5F5F4F81E090E002C067
:107C4000880F991FBA94E2F70197042E01C0880F9C
:107C50000A94EAF72D2D01C0220F4A95EAF7382F32
:107C600030959A8193238223892B8A838983AE015D
:107C70004F5F5F4F6E2D8F2D0E94634C01C080E0DF
:107C80000F900F90DF91CF911F910F91FF90EF9088
:107C9000DF90CF90BF9008950F931F93CF93DF9302
:107CA000D82FC62F60E00E94B34C62E08C2F0E9458
:107CB000114D8C2F0E948B4C8C0161E08D2F0E9406
:107CC000B34C60E08D2F0E94B34C61E08C2F0E947A
:107CD000114D81E0012B09F080E0DF91CF911F91E0
:107CE0000F910895CF93DF93D82FC62F60E00E94A5
:107CF000B34C60E08C2F0E94B34C61E08D2F0E944A
:107D0000B34C61E08C2FDF91CF910C94B34CCF92A8
:107D1000DF92EF92FF920F931F93CF93DF936C014B
:107D20007A018B01C0E0D0E0CE15DF0581F0D801EB
:107D30006D918D01D601ED91FC910190F081E02DC6
:107D4000C6011995892B11F02196EECF7E01C7014E
:107D5000DF91CF911F910F91FF90EF90DF90CF9027
:107D60000895FC01538D448D252F30E0842F90E041
:107D7000821B930B541710F0CF9608950197089526
:107D8000FC01918D828D981761F0828DDF01A80F23
:107D9000B11D5D968C91928D9F5F9F73928F90E045
:107DA00008958FEF9FEF0895FC01918D828D9817B4
:107DB00031F0828DE80FF11D858D90E008958FEFF1
:107DC0009FEF0895FC01918D228D892F90E0805CBA
:107DD0009F4F821B91098F73992708958FEA9AE02C
:107DE000F1DF21E0892B09F420E0822F0895FC01C6
:107DF000848DDF01A80FB11DA35ABF4F2C91848D34
:107E000090E001968F739927848FA689B7892C9368
:107E1000A089B1898C91837080648C93938D848DBB
:107E2000981306C00288F389E02D80818F7D8083BE
:107E30000895EF92FF920F931F93CF93DF93EC017E
:107E400081E0888F9B8D8C8D981305C0E889F98916
:107E5000808185FD25C0F62E0B8D10E00F5F1F4F32
:107E60000F731127E02E8C8DE8120BC00FB607FCA4
:107E7000FACFE889F989808185FFF5CFCE01B7DF98
:107E8000F2CF8B8DFE01E80FF11DE35AFF4FF08218
:107E90009FB7F8940B8FEA89FB89808180620AC0C2
:107EA0009FB7F894EE89FF896083E889F98980811A
:107EB0008370806480839FBF81E090E0DF91CF91E9
:107EC0001F910F91FF90EF900895CF93DF93EC01F6
:107ED000888D8823C1F0EA89FB89808185FD05C0F2
:107EE000A889B9898C9186FD0EC00FB607FCF5CF25
:107EF000808185FFF2CFA889B9898C9185FFEDCF6C
:107F0000CE0175DFE8CFDF91CF91089580E090E05A
:107F1000892B19F063DF811125C080E090E0892B67
:107F200041F080E090E0892B21F00E940000811157
:107F30001CC080E090E0892B41F080E090E0892B2C
:107F400021F00E940000811113C080E090E0892B95
:107F5000A1F080E090E0892B81F00E940000811167
:107F60000AC008950E940000D8CF0E940000E1CF0F
:107F70000E940000EACF0C940000089580E008956C
:107F8000DC011A96ED91FC911B9720E030E01994EA
:107F9000DC011696ED91FC91179720E030E040E06F
:107FA00069E11994DC011696ED91FC91179720E098
:107FB00030E040E068E119949A01DC011696ED91F9
:107FC000FC911797462F67E11994EF92FF920F9358
:107FD0001F93CF93DF931F92CDB7DEB77C018B0148
:107FE000D8016C916731D9F078F4653190F1F801DE
:107FF00041814983D7011696ED91FC91179720E0B6
:1080000030E0C701199522C06A3198F06E3F09F53A
:10801000F8014181498369E2C701B2DF17C0F80165
:1080200081818983AE014F5F5F4F61E0C701C4DF8B
:108030000DC00F5F1F4FD7011696ED91FC9117975A
:1080400020E030E040E0C7011995CACF0E5F1F4F16
:10805000C7CF0F90DF91CF911F910F91FF90EF90BD
:108060000895462FDC011696ED91FC91179720E0BC
:1080700030E066E11994462FDC011696ED91FC91F3
:10808000179720E030E065E11994EF92FF920F938B
:108090001F93CF93DF93EC01142F79016D3079F1A9
:1080A00018F46B3011F152C06E3009F439C06F30E2
:1080B00009F04CC077DFF70183810889F8E08F9FD2
:1080C000000D112460E4CE01D6DF602F62956F7041
:1080D0006061CE01D0DF602F6F70CE01C2DFF7018B
:1080E0006481606BCE01BDDF23C0411103C06AE42F
:1080F00072E002C065E472E0CE0167DF64C0411146
:1081000007C06EE372E061DFE881F981828906C011
:1081100067E372E05ADFE881F9818389888B53C075
:1081200041DF61E8CE01A7DF612FCE019ADF0BC0EE
:10813000F701408151816281660F660F660FCE01A3
:108140003BDF1150A9F7CE0123DF3DC0693031F488
:1081500084E892E09983888382E0E0CF6A3089F5F1
:10816000EA85FB8520E030E040E068E2CE01199529
:10817000EE81FF8120E030E040E064E1CE0119951E
:1081800041E06BE4CE01FCDEE881F981448169E2E3
:10819000CE01F6DE40E06BE4CE01F2DEE881F9814B
:1081A000448169E2CE01ECDE41E06BE4CE01E8DE21
:1081B000E881F981458169E2CE01E2DE6FE472E097
:1081C0009BCF80E001C081E0DF91CF911F910F91A3
:1081D000FF90EF900895DC011896ED91FC911997AE
:1081E00020E030E040E069E11994DC011896ED915F
:1081F000FC91199720E030E040E068E11994662393
:1082000029F06A3019F0862F90E008958FEF9FEFE4
:1082100008950F93DC01D8968C91D89798E0899FA8
:1082200040191124D9968C91D997213071F468178F
:1082300008F04CC0DA968C91DA97481708F046C0DF
:10824000D196ED91FC91D2973FC0023019F4621B98
:108250006F5F04C0033011F4421B4F5FDA969C91AC
:10826000DA97302F317000FD16C0491778F5260FC8
:10827000261730F4681718F42FEF280F03C060E0BA
:10828000681720F5222311F1982F281708F4922F50
:10829000292F261B14C06817C8F4240F241730F4A4
:1082A000491718F42FEF290F05C040E0491770F463
:1082B000222361F0291708F4922F292F241BD1962D
:1082C000ED91FC91D297032FCD0119950F9108954F
:1082D000CF93DF93FC0127A9822F880F880F880F87
:1082E00082AFA081B18150968C915097803208F076
:1082F0008FE1880F880F880F81AF30AD932F990FD2
:10830000990F990F93AF51966C915197432F50E06D
:10831000420F511DC62FD0E0C417D50714F4262FE5
:10832000231B94AF492F38E0239F400D1124242FA5
:1083300045AF30EF36AF54964D915C915597413F24
:10834000510508F446AF56963C9137AFDF01A05C6B
:10835000BF4F1C9211968C9311969C93ED5BFF4F2F
:108360002083DF91CF910895EF92FF920F931F9397
:10837000CF93DF93EC01742F7770E1E0F0E0072EEC
:1083800001C0EE0F0A94EAF73E2F7C0181E7E80E68
:10839000F11CD7018C91823028F41E2F813019F402
:1083A00030E001C010E050E0487F8DA99EA9A8816F
:1083B000B9815096FC91F49FD001F59FB00D112426
:1083C000A60FB11DA80FB91F01110BC08C91812BF5
:1083D00083278D932150D1F71CC0110F330F222317
:1083E000C1F09C91912B93279C937F5F77702150D4
:1083F0007111F3CF89ADA80FB11DF70180818230D3
:1084000020F4813021F031E002C031E0E8CF11E00A
:10841000E6CFDF91CF911F910F91FF90EF900895DC
:1084200080E008950E944E6BCF93DF931F92CDB7EB
:10843000DEB76983BE016F5F7F4F0E94824C0F9051
:10844000DF91CF910895EF92FF921F93CF93DF9327
:10845000EC01162F7A01C9DE60E4CE01E5DFE88584
:10846000F9859701412F67E1CE011995CE01DF9182
:10847000CF911F91FF90EF90AECEEF92FF921F939E
:10848000CF93DF93EC01142F7901673128F4653124
:1084900040F4643101F130C0673171F06A3150F05D
:1084A0002BC0A3DE60E0CE01BFDF612FCE01BCDFB9
:1084B000CE0191DE81E021C0A701193140F068E1D1
:1084C000CE01C1DF185188E1E80EF11CF5CF612F14
:1084D000CE01B9DFEFCF8A898F3F11F488E78A8B0D
:1084E000E885F9859701412F64E1CE01DF91CF91B5
:1084F0001F91FF90EF90199480E0DF91CF911F9131
:10850000FF90EF9008950F931F93CF93DF93EC01AB
:1085100088819981009729F02A813B8126173707A6
:1085200088F48B016F5F7F4F0E946E6A009761F045
:10853000998388831B830A832C813D81232B11F42B
:10854000FC01108281E001C080E0DF91CF911F919A
:108550000F910895CF93DF93EC0188819981009763
:1085600011F00E94E569198218821D821C821B820B
:108570001A82DF91CF910895EF92FF920F931F938C
:10858000CF93DF93EC017B018A01BA01BCDF81113B
:1085900003C0CE01DFDF07C01D830C83B7018881D4
:1085A00099810E94766BCE01DF91CF911F910F913F
:1085B000FF90EF900895CF93DF93EC016115710563
:1085C00051F0FB0101900020E9F73197AF01461B04
:1085D000570BD2DF01C0BEDFCE01DF91CF910895EE
:1085E000CF93DF93EC01FB018617970751F0608171
:1085F00071816115710521F044815581BDDF01C094
:10860000A9DFCE01DF91CF910895FC018081918196
:108610000C94E5696115710579F0FB01019000206A
:10862000E9F73197AF01461B570BDC01ED91FC9147
:108630000280F381E02D199480E090E008958F92FC
:108640009F92AF92BF92EF92FF920F931F93CF939F
:10865000DF93CDB7DEB7A1970FB6F894DEBF0FBE9C
:10866000CDBF7C01FA01CB0119A2223008F42AE027
:108670008E010F5D1F4F822E912CA12CB12CBF01BA
:10868000A50194010E94DF67F901CA010150110997
:108690006A3014F4605D01C0695CD8016C93232BCF
:1086A000242B252B61F7B801C701B4DFA1960FB6C3
:1086B000F894DEBF0FBECDBFDF91CF911F910F9118
:1086C000FF90EF90BF90AF909F908F9008951F9272
:1086D0000F920FB60F9211240BB60F922F933F9368
:1086E0004F935F936F937F938F939F93AF93BF93BA
:1086F000EF93FF938FEA9AE07ADBFF91EF91BF91BE
:10870000AF919F918F917F916F915F914F913F9129
:108710002F910F900BBE0F900FBE0F901F901895CA
:108720001F920F920FB60F9211240BB60F922F9338
:108730008F939F93EF93FF93E091BF0AF091C00A4C
:108740008081E091C50AF091C60A82FD12C0908135
:108750008091C80A8F5F8F732091C90A821751F0E8
:10876000E091C80AF0E0E155F54F958F8093C80A73
:1087700001C08081FF91EF919F918F912F910F9078
:108780000BBE0F900FBE0F901F9018950F93FC011A
:10879000EE5BFF4F308131965081451728F430173A
:1087A00030F0041720F010C03017D8F30DC0FC01D2
:1087B000E05CFF4F308131968081681738F43217C2
:1087C00040F081E0261730F080E004C03217C8F393
:1087D000FBCF81E00F9108950F93DC01D396ED91CB
:1087E000FC91D4970280F381E02D19950F910895A3
:1087F00020913209309133092817390771F490918B
:10880000300980913109981741F0E0913009F0E08A
:10881000E159F54F808190E008958FEF9FEF089523
:108820001F93CF93DF93DC015C968D919C915D97B4
:10883000009739F421E030E013963C932E93129781
:108840003BC05196ED91FC91529750962C915097C8
:10885000322F30951FB75E964C915E97742F7270D1
:1088600041FD6095F8944081772311F0422B01C0BF
:1088700043234083EC012197F1F748E0508160FFEA
:1088800002C0522B01C053235083EC012197F1F712
:108890006695415099F78081772319F0832380836F
:1088A00002C0282B20831FBF5C968D919C915D9701
:1088B0000197F1F781E090E0DF91CF911F9108954A
:1088C00020913209309133092817390769F48091D2
:1088D00031092091300990E0805C9F4F821B910903
:1088E00060E470E00C94326980E090E0089520919B
:1088F00032093091330928173907B9F490913009BA
:1089000080913109981789F0E0913009F0E0E15940
:10891000F54F80812091300930E02F5F3F4F2F735A
:1089200033272093300990E008958FEF9FEF08954B
:108930000F931F93CF93DF93182F062FD42FC8E0E8
:1089400060E0812F0E94B34CD0FF02C061E001C003
:1089500060E0802F0E94B34CD69561E0812F0E9489
:10896000B34CC15069F7DF91CF911F910F910895DA
:10897000862F642FF8C7862F642F0C94114D862FF5
:10898000642F0C94114DFC018185C5D721E0892B02
:1089900009F420E0822F0895862FBDC71F93CF933F
:1089A000DF93D82FC62F142F61E08C2FDCD761E026
:1089B0008D2FD9D760E08C2FD6D7412F6C2F8D2FDC
:1089C000B7DF6C2F8D2F68D9182F6C2F8D2F8AD978
:1089D000812FDF91CF911F9108958F929F92AF9237
:1089E000BF92DF92EF92FF920F931F93CF93DF938B
:1089F00000D01F921F92CDB7DEB77C015B018A01C8
:108A0000D22EFC018681420F511D282F30E0241701
:108A1000350708F45BC0CE0101964C0185E0F401F6
:108A200011928A95E9F78D2D8770806C8983A80152
:108A3000CE0102960E94526BF1E0FD15C0F0F701E5
:108A40009485D1100CC00230110548F02B81911192
:108A500002C080E001C080E8822B8B8308C02A819D
:108A6000911102C080E001C080E8822B8A830F5FF1
:108A7000F7011581F48061E0812F75D761E08F2DBA
:108A800072D760E0812F6FD754018A2D8819801723
:108A900050F4F50141915F01612F8F2D49DF612F66
:108AA0008F2DFAD8F2CF612F8F2D0F900F900F904E
:108AB0000F900F90DF91CF911F910F91FF90EF904A
:108AC000DF90BF90AF909F908F900CC9182F1D1909
:108AD000412F50E02D2DC70180DFF701628573859E
:108AE00080E090E00E94914D0D5F011B11E0F701C5
:108AF0004681041788F050E0B501610F711D20E038
:108B0000C7016BDFF7016285738580E090E00E940A
:108B1000914D01501F5FEBCF0F900F900F900F9072
:108B20000F90DF91CF911F910F91FF90EF90DF9009
:108B3000BF90AF909F908F900895FF920F931F93D7
:108B4000CF93DF93CDB7DEB7C058D1090FB6F894F5
:108B5000DEBF0FBECDBF4138510510F040E850E0F8
:108B60009E012F5F3F4FDB018B01040F151FB901E1
:108B7000A017B10779F0ED91E0323CF00E2E000C19
:108B8000FF0BE75BFE4BF49001C0F12CF901F19271
:108B90009F01EECFFC01218520DFC058DF4F0FB6CB
:108BA000F894DEBF0FBECDBFDF91CF911F910F9123
:108BB000FF9008951F93CF93DF93EC01162F8985C3
:108BC0009E81891327C090E0BE01635F7F4F20E044
:108BD000E22FF0E0E817F90730F4E60FF71F3181D4
:108BE00030832F5FF5CF898590E0103244F0E12F7C
:108BF000012E000CFF0BE75BFE4BE49101C0E0E0AF
:108C0000DE01A80FB91F1D96EC934E8150E020E0C5
:108C1000CE01E3DE49858E814817F0F450E0103232
:108C20003CF0E12F110FFF0BE75BFE4BE49101C01D
:108C3000E0E0DE01A40FB51F1D96EC934F5F5F4F80
:108C400020E0BE01635F7F4FCE01C7DE89858F5F65
:108C5000843008F083E08987DF91CF911F910895D8
:108C6000DC01862F653608F084E618968C931897F9
:108C70006AE00E941269893008F088E081508830EB
:108C800030F4E82FF0E0E456FD4F408101C040E8A9
:108C900015966C91159714968C9180CE1F920F9219
:108CA0000FB60F9211240BB60F922F933F934F9351
:108CB0005F936F937F938F939F93AF93BF93EF9344
:108CC000FF93E0913209F0913309309709F451C0D4
:108CD000968DA685B785858591FF04C09C918923D3
:108CE00029F447C09C91892309F043C0A389B48922
:108CF0009C918589809589238C9386899789019792
:108D0000F1F7608D718DA685B785558538E020E037
:108D1000CB010197F1F7822F90E095958795282F49
:108D20004C91452309F02068315091F7868D81FDE3
:108D300020958091310990E001968F7399273091A9
:108D40003009381749F0A0913109B0E0A159B54F69
:108D50002C938093310903C0868D8160868F828D2C
:108D6000938D0197F1F7A389B4899C918589892B0B
:108D70008C93FF91EF91BF91AF919F918F917F91D4
:108D80006F915F914F913F912F910F900BBE0F907C
:108D90000FBE0F901F901895FC014481558160E033
:108DA00070E0808591850C945B6BFF920F931F930D
:108DB000CF93DF93EC01FF24F394F60E2F81F2168C
:108DC00079F1088519852150B9F06F3F59F430E0E9
:108DD00040E050E06FEF7FEF80E090E00E94B367EB
:108DE000B9010CC08F2D90E0982F88270197622F32
:108DF00070E00E941E6902C060E070E0F8014C81E2
:108E00005D81CF01801B910B8417950740F4408151
:108E1000469FC001479F900D11249193F0CFFF8290
:108E2000DF91CF911F910F91FF9008950F931F93A2
:108E3000DC0112968D919C9113976817790708F0C1
:108E400043C017968C911797882361F0489FA00123
:108E50001124452F829F90011124232F809F800190
:108E60001124012F1D968C911D971A969C911A978B
:108E70001896ED91FC911997891308C0CB01880FC2
:108E8000991F680F791F6E0F7F1F0AC0660F771F2B
:108E9000660F771F6E0F7F1FFB01E80FF11D108219
:108EA0001A968C911A97FB01E80FF11D40831B96CF
:108EB0008C911B97FB01E80FF11D20831C968C9170
:108EC000FB01E80FF11D00831F910F910895CF92D0
:108ED000DF92EF92FF920F931F93CF93DF93CDB763
:108EE000DEB729970FB6F894DEBF0FBECDBF8C0159
:108EF000DC0118968D919C911997892B09F4A1C0DA
:108F0000EBD5F801C684D784E088F188DC01CB0179
:108F10008C199D09AE09BF098C329140A105B1059C
:108F200078F3F894D80114968D919C9115979A83B3
:108F300089831896ED91FC9119977F01BFEFEB1A89
:108F4000FB0A80818987F80190810288F389E02DEE
:108F5000D80154968C91992309F430C09081982BB4
:108F600098879081809589238F838F818C8388E077
:108F70008B8358856F8149853B812C8189819A81BA
:108F8000D701508347FD252F3A952083262F39F0AE
:108F9000441F00C000006083000000C0F2CF38E032
:108FA0004D9160830000019761F7D8015396FC93BF
:108FB000EE93529749873B832C833AC09081982B3C
:108FC00098879081809589238F838F818E8388E015
:108FD0008D8358856F8149853D812E8189819A8154
:108FE000D701508347FD252F00C000C0208300C05B
:108FF00000C000C000C000C060830000262F3A956A
:1090000041F0441F000000C000C000C000C000C00C
:10901000E8CF38E04D9100C0608300C0019709F7A8
:10902000D8015396FC93EE93529749873D832E8344
:109030009A838983789450D5F80166877787808BE7
:10904000918B29960FB6F894DEBF0FBECDBFDF918E
:10905000CF911F910F91FF90EF90DF90CF900895E7
:10906000CF93DF93EC018E8187FD05C061E0D9D4F9
:1090700060E08E8178D481E08983DF91CF9108957B
:109080001F93CF93DF93EC01162F0E949D67181753
:1090900039F0612FCE01DF91CF911F910C94A5671C
:1090A000DF91CF911F9108950C949D6760E177E265
:1090B00080E090E036D50E9406354EE353E068E04C
:1090C00081E00E9429340E94F1348CE59CE00E94EA
:1090D000363448E253E06EE18EE10E94293476D3C3
:1090E0008CE893E00E9436341092550910926A0978
:1090F0001092660910926509109262091092670930
:1091000081E0809309021092640961E08AE12BD426
:1091100010925A0910925B0910925C0910925D0935
:109120001092460910924709109248091092490975
:1091300084E690E09093080280930702E2D00C94BA
:10914000F430EF92FF920F93CF93DF9360E971E0D9
:1091500080E090E0E6D41092110C1092140C68E4B8
:1091600078E088E09CE00E940F350E9406358CE58F
:109170009CE00E9436344DE658E06EE18EE10E949C
:10918000293444E758E06DE282E10E9429341ED37D
:109190008CE893E00E94363461E074E08FE03DD2C9
:1091A00089E1E82EF12CC0E0D0E000E020E04FEFB4
:1091B000BE0182EE9BE03ADE20E04FEFBE018DEC77
:1091C0009BE034DE82EE9BE082DE8DEC9BE07FDE76
:1091D0006AE070E080E090E0A4D420E040E0BE01CE
:1091E00082EE9BE023DE20E040E0BE018DEC9BE0C0
:1091F0001DDE82EE9BE06BDE8DEC9BE068DE6AE0BC
:1092000070E080E090E08DD42196C830D10569F6F9
:1092100081E0E81AF10809F0C6CFDF91CF910F91F4
:10922000FF90EF9043CFEF92FF920F93CF93DF9396
:109230001092110C1092140C6DE578E088E09CE01F
:109240000E940F350E9406358CE59CE00E94363462
:1092500041E254E06EE188E20E9429344EE758E092
:109260006DE287E10E942934B1D28CE893E00E943C
:10927000363462E074E08FE0D0D189E1E82EF12C41
:10928000C0E0D0E00FEF20E040E0BE0182EE9BE0C6
:10929000CDDD82EE9BE01BDE20E040E0BE018DECE8
:1092A0009BE0C4DD8DEC9BE012DE6AE070E080E0C4
:1092B00090E037D400E020E040E0BE0182EE9BE089
:1092C000B5DD82EE9BE003DE20E040E0BE018DECE8
:1092D0009BE0ACDD8DEC9BE0FADD6AE070E080E0C5
:1092E00090E01FD42196C830D10561F681E0E81ADC
:1092F000F10809F0C5CFDF91CF910F91FF90EF906A
:10930000D5CE0F931F93CF93DF9380915109909106
:1093100052099C01215031091092000C2B33310568
:1093200080F511E01093030CCAE0D0E0BE010E946A
:10933000326987EF9BE00E9411351093000C8091F9
:10934000510990915209BE010E943269BC0187EF18
:109350009BE00E94113582E08093000C809107020F
:1093600090910802BE010E94326987EF9BE00E9443
:10937000113583E08093000C8091070290910802E0
:109380003CC0C1E0C093030C68E572E00E94326902
:1093900087EF9BE00E941135C093000C809151092A
:1093A000909152090CE310E0B8010E943269CB01A0
:1093B000CAE0D0E0BE010E943269BC0187EF9BE0A9
:1093C0000E94113582E08093000C809151099091A8
:1093D0005209B8010E943269BE010E94326987EFCA
:1093E0009BE00E94113583E08093000C809151092D
:1093F00090915209B8010E943269BE010E943269FF
:10940000BC0187EF9BE0DF91CF911F910F910C94EE
:10941000113547E858E063E283E20E942934D6D14F
:1094200068EE73E080E090E07CD30C9406350F93F7
:109430001F93CF93DF938091190C90911A0CDC014C
:10944000ED91FC910084F185E02D1995892B09F4AB
:10945000AEC0C091370C8091190C90911A0CDC01B0
:10946000ED91FC910284F385E02DC1110AC019959C
:109470008093230C8E37F9F610923D0C8091370CB7
:1094800092C01995EC2FF0E0E75EF34F8287809150
:10949000370C823069F0893089F0813009F083C05F
:1094A0009091240C9F3F09F47EC01092370C74C039
:1094B0009091250C963009F476C004C080912C0C54
:1094C0008F3E19F01092370C66C0E4E2FCE08AE2AD
:1094D0009CE020E030E04191240F311D8E179F0762
:1094E000D1F780912A0C90E0982F882740912B0C7F
:1094F000840F911D3195219531091092370C8217F7
:10950000930709F048C0E091260CE0933A0C2091B3
:10951000280C30E0322F22278091290C280F311D92
:1095200030933C0C20933B0C8E2F90E0FC01FA977B
:10953000E631F105D8F48827EE58FF4F8F4F0C9491
:10954000456985E00DC021FF1CC084E009C021FFF2
:1095500018C082E005C021FF14C083E001C086E08E
:109560008093390C81E080933D0C0BC081E08093A7
:10957000390C10923C0C10923B0C80933D0C1092D5
:109580003E0CD0913D0CDD2309F441C08091310C9B
:1095900081113DC037C081E08093390C10923C0CA2
:1095A00010923B0C2DC08F5F8093370C44CF80917D
:1095B0003E0C882351F1EDD200911B0C10911C0C34
:1095C00020911D0C30911E0CDC01CB01801B910BF6
:1095D000A20BB30B00911F0C1091200C2091210CB9
:1095E0003091220C80179107A207B30770F01092F8
:1095F000370C1092390C10923C0C10923B0C81E00D
:1096000080933D0C10923E0C02C0D0913D0C8D2FEA
:10961000DF91CF911F910F9108958093300C70933B
:10962000320C6093330CEEE2FCE024E33CE080E09B
:1096300090E04191840F911D2E173F07D1F791952E
:10964000819591099093340C8093350C8091310C65
:10965000882331F080913E0C882339F0E8DEFACF80
:109660006AE070E080E090E05CD28091190C90910B
:109670001A0CDC01ED91FC910280F381E02D4AE0AF
:1096800050E06DE27CE0199584D260931B0C7093DE
:109690001C0C80931D0C90931E0C81E09091310C5A
:1096A000911101C080E080933E0C0895FF920F93CA
:1096B0001F93CF93DF93182FC62FF42ED62FD20FE0
:1096C000282F240F0D2F462F682F84E99CE05ED8A9
:1096D000882369F0DC1759F0FF2039F000E02F2DC6
:1096E0004C2F612F84E99CE077D8CF5FF3CFDF91D7
:1096F000CF911F910F91FF900895DC011496ED9189
:10970000FC91159720E030E040E060E11994AF92C1
:10971000BF92CF92DF92EF92FF920F931F93CF935E
:10972000DF9300D01F921F92CDB7DEB78C01DC0112
:10973000D796AC90D797D896EC90D897ED91FC91AE
:10974000B188FE2CC12CD12CD801ED91FC91119740
:109750008089D5964D915C91D6971C82FD828B8332
:10976000B8E08B9FC00111248C9D90018D9D300D20
:109770009C9D300D1124CA01820F931F9A83898307
:10978000D8011496ED91FC9115979E012F5F3F4FE4
:1097900041E06FE0C8011995F3948F2D8E198A1559
:1097A00028F4BFEFCB1ADB0AFB1470F20F900F9076
:1097B0000F900F900F90DF91CF911F910F91FF901D
:1097C000EF90DF90CF90BF90AF90089584E99CE038
:1097D0009EDF84E99CE091CFE0E9FCE084AF07A83C
:1097E000F0ADE02D0190F081E02D84E99CE019942A
:1097F000E0E9FCE0A481B58150968C9143AD849F53
:10980000A001112483E0440F551F8A95E1F760E021
:1098100070E081AD92AD0C945B6B90E0FC013197F0
:10982000E231F10508F04EC08827E857FF4F8F4F0F
:109830000C944569809180008F7703C080918000EF
:109840008F7D80938000089580918000877FF9CF7D
:1098500084B58F7702C084B58F7D84BD08958091D3
:10986000B0008F7703C08091B0008F7D8093B000EF
:109870000895809190008F7707C0809190008F7D30
:1098800003C080919000877F80939000089580911D
:10989000A0008F7707C08091A0008F7D03C08091CA
:1098A000A000877F8093A0000895809120018F778A
:1098B00007C0809120018F7D03C080912001877FA8
:1098C000809320010895CF93DF93EA0191E0909374
:1098D000E80980930A0A1092E90910920B0A8CE4B5
:1098E0009BE00E941C3968818CE49BE00E941C393B
:1098F00081E00E94B83791E0811190E0892FDF91DB
:10990000CF9108959B01DC011896ED91FC91199778
:1099100041E067E11994CF93DF93282F30E0F901FC
:10992000ED55FD4B8491F901ED5BFD4BD491F901AF
:10993000E350FE4BC491CC2389F081116EDFEC2FF4
:10994000F0E0EE0FFF1FE753FE4BA591B491EC91B1
:10995000ED2381E090E021F480E002C080E090E01F
:10996000DF91CF9108951F93CF93DF93282F30E09D
:10997000F901ED55FD4B8491F901ED5BFD4BD4915F
:10998000F901E350FE4BC491CC23B9F0162F81119D
:1099900044DFEC2FF0E0EE0FFF1FED51FE4BA591E1
:1099A000B4919FB7F894111104C08C91D095D8232D
:1099B00002C0EC91DE2BDC939FBFDF91CF911F9112
:1099C000089510921F1110921E111092E909109221
:1099D0000B0A1092E70981E08093E6091092C10911
:1099E00061E084E1C0DF61E085E1BDDFE9EBF0E04B
:1099F00080818E7F808380818D7F808388E48093C7
:109A0000B80085E48093BC0082EC98E390931D112C
:109A100080931C1183EC98E390931B1180931A118F
:109A20000895CF93DF9390E0FC01ED5BFD4B249113
:109A3000FC01E350FE4B8491882361F190E0880F94
:109A4000991FFC01E757FD4BC591D491FC01ED51E5
:109A5000FE4BA591B491611109C09FB7F89488811C
:109A6000209582238883EC912E230BC0623061F411
:109A70009FB7F8948881322F309583238883EC91A7
:109A80002E2B2C939FBF06C08FB7F894E8812E2B06
:109A900028838FBFDF91CF910895863308F08653D6
:109AA00090917B00282F2870977F922B90937B00BA
:109AB0008770806480937C0080917A0080648093BA
:109AC0007A0080917A0086FDFCCF80917800209109
:109AD000790090E0922B08953FB7F894809125117A
:109AE00090912611A0912711B091281126B5A89B1D
:109AF00005C02F3F19F00196A11DB11D3FBFBA2F20
:109B0000A92F982F8827820F911DA11DB11DBC017F
:109B1000CD0142E0660F771F881F991F4A95D1F744
:109B200008958F929F92AF92BF92CF92DF92EF9261
:109B3000FF926B017C01D0DF4B015C01C114D104A9
:109B4000E104F104E9F0C8DFDC01CB0188199909CF
:109B5000AA09BB09883E9340A105B10578F321E02D
:109B6000C21AD108E108F10888EE880E83E0981E39
:109B7000A11CB11CC114D104E104F10421F7DECF12
:109B8000FF90EF90DF90CF90BF90AF909F908F901D
:109B900008952FB7F894609121117091221180914E
:109BA0002311909124112FBF0895CF92DF92EF924D
:109BB000FF921F93CF93DF93EC0188858B7F88877B
:109BC000CE010E94C344182F88858695817018178E
:109BD00049F0DFDF6A837B838C839D83988582E0F5
:109BE000892721C0D6DFCA80DB80EC80FD80AB01F5
:109BF000BC014C195D096E097F098E819F81A0E02F
:109C0000B0E0481759076A077B0770F088858170B4
:109C1000181751F0BEDF6A837B838C839D83988500
:109C200081E0892784608887888582FB882780F97E
:109C3000DF91CF911F91FF90EF90DF90CF9008952B
:109C40001F920F920FB60F9211242F933F938F9371
:109C50009F93AF93BF938091211190912211A09176
:109C60002311B09124113091201123E0230F2D37BF
:109C700020F40196A11DB11D05C026E8230F029610
:109C8000A11DB11D209320118093211190932211C9
:109C9000A0932311B0932411809125119091261146
:109CA000A0912711B09128110196A11DB11D80939B
:109CB000251190932611A0932711B0932811BF91DD
:109CC000AF919F918F913F912F910F900FBE0F9069
:109CD0001F901895CF93DF93CDB7DEB72D970FB6B2
:109CE000F894DEBF0FBECDBF789484B5826084BD8A
:109CF00084B5816084BD85B5826085BD85B5816090
:109D000085BD80916E00816080936E00109281000D
:109D100080918100826080938100809181008160C8
:109D20008093810080918000816080938000809189
:109D3000B10084608093B1008091B0008160809315
:109D4000B000809191008260809391008091910099
:109D50008160809391008091900081608093900059
:109D60008091A10082608093A1008091A100816018
:109D70008093A1008091A00081608093A0008091D9
:109D80002101826080932101809121018160809373
:109D900021018091200181608093200180917A00CF
:109DA000846080937A0080917A00826080937A0048
:109DB00080917A00816080937A0080917A00806837
:109DC00080937A001092C100E091BF0AF091C00A1E
:109DD00082E08083E091BB0AF091BC0A1082E0919E
:109DE000BD0AF091BE0A8FEC80831092C70AE09101
:109DF000C30AF091C40A86E08083E091C10AF09121
:109E0000C20A808180618083E091C10AF091C20A18
:109E1000808188608083E091C10AF091C20A8081CC
:109E200080688083E091C10AF091C20A80818F7DB1
:109E3000808310925A0C1092590C1092580C109268
:109E4000570C1092560C1092550C8DE991E090939E
:109E50005C0C80935B0C80914B0C96EF980F9430C8
:109E600048F02EEC280F243028F022EC280F283060
:109E700008F06BC02DEB30E03093560C2093550C5E
:109E80002BE931E03093580C2093570C2CE231E051
:109E900030935A0C2093590C943058F02EEC280F24
:109EA000243038F022EC280F283038F4A8E6B0E04F
:109EB00006C0A8E6B0E00C94205EA0E0B0E0283038
:109EC00010F40C94205EE0E0F0E02081943010F477
:109ED0000C94FC5D9EEC980F943010F40C94FC5D97
:109EE0008E53883010F00C94FC5D84E0822B8C93B0
:109EF00080914B0C96EF980F943010F40C94FF5D0A
:109F00002EEC280F243010F40C94FF5D22EC280F67
:109F1000283010F00C94035E2DE630E03093530CA3
:109F20002093520C943010F00C94075E9AEF980F27
:109F300081E001C0880F9A95EAF78093540C8091D4
:109F40005B0C90915C0C0197F1F78091590C90910A
:109F50005A0C892B49F1E0913209F09133092CE038
:109F6000EF33F20709F1309739F0A389B4899C9156
:109F70008589809589238C9380915D0C8E7F809359
:109F80005D0C10923109109230098FE39CE09093A0
:109F9000330980933209E091520CF091530C908177
:109FA0008091540C892B808311E01093310C8FE346
:109FB0009CE090931A0C8093190C80911F0C909147
:109FC000200CA091210CB091220C8854944FAF4FDB
:109FD000BF4F80931F0C9093200CA093210CB09343
:109FE000220C60E070E08CE018DB10933E0C1FDA6E
:109FF0008823E9F380911F0C9091200CA091210CF3
:10A00000B091220C885B9B40A109B10980931F0C81
:10A010009093200CA093210CB093220C68EC70E07C
:10A0200080E090E07EDD10923D0CF090390C34E041
:10A03000F3120C94545A84EF91E0A0E0B0E08093C6
:10A040001F0C9093200CA093210CB093220C80E065
:10A0500090E02AD8682F70E086E0DFDA60E070E0F8
:10A0600087E0DBDA62E070E089E0D7DA68EC70E084
:10A0700080E090E056DDA5DC01E023E042E06BE605
:10A0800080910B0D0E94FC3D00E022E044E06BE17A
:10A0900080910B0D0E94FC3D22E044E06CE1809138
:10A0A0000B0D0E94FC3DE0900B0D08EE13E09E01AD
:10A0B0002F5F3F4F41E06BE68E2D0E94F13C89817E
:10A0C0008F7B89838D87AE01435F5F4F6BE68E2D5B
:10A0D000FADBE091BF0AF091C00A82E08083E09150
:10A0E000BB0AF091BC0A1082E091BD0AF091BE0A51
:10A0F00080E180831092C70AE091C30AF091C40AFC
:10A1000086E08083E091C10AF091C20A808180617B
:10A110008083E091C10AF091C20A808188608083C7
:10A12000E091C10AF091C20A808180688083E09149
:10A13000C10AF091C20A80818F7D8083E091980CE2
:10A14000F091990C20E030E040E06AE084E99CE086
:10A1500019950E940134E091980CF091990C20E03F
:10A1600030E040E06BE084E99CE019958CE893E0F6
:10A170000E943634F0920E0C11E010930F0C88E020
:10A180009CE00E94983782E090E00E945448682F3B
:10A1900088E09CE00E943046F092FD0B1093FE0B8D
:10A1A00087EF9BE00E94983782E090E00E9454483D
:10A1B000682F87EF9BE00E94304682EE9BE00E9472
:10A1C000304881E090E00E945448682F82EE9BE086
:10A1D0000E94D54682EE9BE00E9467478DEC9BE093
:10A1E0000E94304881E090E00E945448682F8DEC36
:10A1F0009BE00E94D5468DEC9BE00E94674760E0A3
:10A2000088E10FDC60E08CE10CDC60E084E009DCDC
:10A2100060E085E006DC60E086E003DC61E08AE186
:10A2200000DC60E086E3FDDB68E170E086E89CE04E
:10A230000E94343805E010E010938D0C00938C0CD4
:10A240006CE170E08CE79CE00E9434381093830C42
:10A250000093820C64E070E082E79CE00E94343856
:10A260001093790C0093780C65E070E088E69CE030
:10A270000E94343810936F0C00936E0C66E070E00F
:10A280008EE59CE00E9434381093650C0093640CBA
:10A2900088E09CE00E94983787EF9BE00E94983707
:10A2A00081E4FBDBBC01990F880B990B61157105EB
:10A2B0008105910511F00E94FA630E94AF63FAE0F4
:10A2C000CF2ED12CE12CF12CA70196010E94B3676F
:10A2D000609305020E94AF63A70196010E94B367D5
:10A2E000609304020E94AF63A70196010E94B367C6
:10A2F000609303020E94AF63A70196010E94B367B7
:10A300006093020280E090E00E945448882341F06C
:10A310008A3031F0843121F08E3111F00C94595A89
:10A3200081E090E00E945448843131F0883221F07D
:10A33000803411F00C94605A82E090E00E945448FE
:10A340008A3031F0823321F0843611F00C94675A50
:10A3500083E090E00E945448853041F08F3031F026
:10A360008E3121F08C3311F00C946E5A84E090E021
:10A370000E945448982F9B7F913031F08A3021F011
:10A380008F3011F00C94755A85E090E00E9454488B
:10A39000853031F08A3021F08F3011F00C947C5AE6
:10A3A00089E090E00E945448853031F08A3021F0F5
:10A3B0008F3011F00C94835A86E090E00E9454484C
:10A3C000853041F08F3031F08E3121F08C3311F037
:10A3D0000C948A5A88E090E00E945448882341F007
:10A3E000853031F08A3021F08F3011F00C94915A81
:10A3F00087E090E00E945448982F977F923031F088
:10A40000853021F0883C11F00C94985A8AE090E055
:10A410000E945448853031F08A3021F08F3011F09D
:10A420000C949F5A8BE090E00E945448853041F094
:10A430008F3031F08E3121F08C3311F00C94A65A0C
:10A440008CE090E00E945448982F9B7F913031F02F
:10A450008A3021F08F3011F00C94AD5A62E173E034
:10A4600087EF9BE00E940F3562E173E088E09CE09B
:10A470000E940F350E9406350EE212E022E344E30B
:10A4800061E084E20E94243747E153E06EE381E01B
:10A490000E94293440E253E06EE38CE50E942934A7
:10A4A00086E3FBDABC01990F880B990B0E948A6640
:10A4B00020E030E040EA50E40E94E96620E030E02D
:10A4C00040E85AE30E94E96623ED3BE94EE55EE38E
:10A4D0000E9475680E94FF2CBC01CE0107960E9465
:10A4E000F83663E070E0CE0107960E94E5361A82E6
:10A4F00019821C821B821E821D82BE01695F7F4FF2
:10A50000CE0101960E94F04266E273E0CE01019610
:10A510000E94B236BC01CE0107960E94F042CE01E5
:10A5200001960E9405438FE58093090D88E0809392
:10A530000A0DCE0107960E94A936CE0107960E9409
:10A54000054344D961E08AE10EDA61E071E08FE011
:10A5500064D868E873E180E090E0E3DA0E940635B1
:10A5600060E08AE100DA87E70E94692D0E94AA2153
:10A5700080910B02813009F056C083E090E00E9488
:10A5800054484CE3849FC001112490934B0980935D
:10A590004A0983E090E00E9454485CE3859FC00133
:10A5A0001124909354098093530984E090E00E9411
:10A5B00054482CE3829FC001112490933609809364
:10A5C00035090E9480310E94F4300E94063541E036
:10A5D00055E068E081E00E9429340E94F1348CE566
:10A5E0009CE00E94363448E253E06EE18EE10E9426
:10A5F00029348CE893E00E943634E8D861E08AE19F
:10A60000B2D98CE60E94692DFF24F39458EE852E72
:10A6100053E0952EA12CB12C6AE5262E73E0372E3F
:10A62000E6E4EE2E81C08230B9F41092500986E043
:10A6300090E00E9454483CE3839FC0011124909312
:10A640004B0980934A090E949D2F0E94622F0E940D
:10A6500006354EE253E018C08330B1F6109250092F
:10A660008BE090E00E9454484CE3849FC001112489
:10A6700090934B0980934A090E9481490E94F430CB
:10A680000E9406354EE353E068E081E00E942934E1
:10A690000E94F1348CE59CE00E94363448E253E09D
:10A6A0006EE18EE10E9429348CE893E00E943634FA
:10A6B0008DD88CE893E00E943634A0CFC60168EEB6
:10A6C00073E00E94326977FF03C07195619571094B
:10A6D000E60FF71FC90168EE73E00E94326977FF49
:10A6E00003C0719561957109E60FF71F8091000213
:10A6F000909101028E179F0714F4F09263098091E4
:10A700006A09882309F455C080910B02813009F44D
:10A7100055C080910B02823009F02FC580916A09E3
:10A72000811111C30E94863F86E89CE03EDA8CE7E7
:10A730009CE03BDA82E79CE038DA88E69CE035DA98
:10A740008EE59CE032DA08EE13E02CE03DE046E0D6
:10A7500063E480910B0D0E94F13C80910C0D90916F
:10A760000D0D9827892798279093700980936F097A
:10A77000C0900E0DD0900F0DDC24CD24DC24D0929F
:10A780006E09C0926D092091100D3091110D322784
:10A790002327322730936C0920936B0968EE73E00E
:10A7A0000E943269FB0177FF89CFF195E195F109AC
:10A7B00085CF80917A0C80FDD7C6A6CF80916A099B
:10A7C000882309F4DAC4E5D960935A0970935B09C8
:10A7D00080935C0990935D09DCD96093860970933E
:10A7E00087098093880990938909D3D900918209B8
:10A7F0001091830920918409309185092B013C0136
:10A80000401A510A620A730A930182010436110543
:10A810002105310540F0609382097093830980938C
:10A8200084099093850920918209309183092C59DC
:10A830003F4FC901861B970B909308028093070234
:10A840000E94F43080916909882329F0A2D90E94DE
:10A8500031300E948031809168098330B9F4809151
:10A860000A02811104C080916909882379F09091CE
:10A870008E0C80913B0990FF07C09091840C90FF53
:10A8800003C0811103C059C781115EC78091680957
:10A89000833029F57ED9009137091091380920912C
:10A8A000390930913A09DC01CB01801B910BA20BD5
:10A8B000B30B883E9340A105B10588F080910A0250
:10A8C00081114DC780916909811149C762D960938F
:10A8D0003709709338098093390990933A09409168
:10A8E0008609509187096091880970918909809142
:10A8F0007E0990917F09A0918009B09181092A0178
:10A900003B01481A590A6A0A7B0A2091550930E02E
:10A910002F5F3F4F032E000C440B550BC501B401B4
:10A920000E94DF67421653066406750608F495C058
:10A930008091530990915409019790935409809301
:10A94000530980916909882349F0809135099091D4
:10A950003609019790933609809335090E9480311A
:10A960000E94F4308091530990915409892B31F45D
:10A9700080916909811102C00E94D032809135090D
:10A9800090913609892B11F40E9457328091680901
:10A99000823031F580910A02811104C080916909E9
:10A9A0008823F1F085E090E00E9454489091450999
:10A9B0009817B0F480918E0C80FFDEC78091840CD4
:10A9C00080FDB6C7D9C7853049F444E1D49E402DF7
:10A9D000112424E168E28FE00E94564B0E94E64B6E
:10A9E00080916909882349F164E071E08FE00E9459
:10A9F0000D4B85E090E00E94544890E0209145097D
:10AA000030E02817390714F00E94D0328091620993
:10AA1000863010F00E94573290916309809162094C
:10AA2000992331F08F5F809362091092630905C00A
:10AA3000882319F081508093620980918609909152
:10AA40008709A0918809B091890980937E09909324
:10AA50007F09A0938009B0938109809169098111D0
:10AA60006AC085E090E00E94544890E0209145093A
:10AA700030E02817390724F080910A0281118DC730
:10AA80009091660C8091440990FF2AC0811188C77B
:10AA900090910A02911184C761E08AE10E94B34C4F
:10AAA0000E94063549E453E068E080E00E942934C2
:10AAB0000E94F1348CE59CE00E9436344AED53E06C
:10AAC0006EE18EE10E9429340E94E64B8CE893E00F
:10AAD0000E94363482E70E94692DF09244092BC00F
:10AAE000882309F45DC760E08AE10E94B34C0E94AC
:10AAF000063549E453E068E080E00E9429340E9472
:10AB0000F1348CE59CE00E94363480910A0288235F
:10AB100009F486C748E253E06EE18EE10E942934D1
:10AB200087E60E94692D0E94E64B8CE893E00E9424
:10AB3000363410924409809168098D7F813009F084
:10AB4000E8CD80910A02811105C0809169098823AE
:10AB500009F4DFCD0E945E35182F882309F4D9CD82
:10AB600064E071E08FE00E940D4B10330CF4D1CD06
:10AB7000809106028130C9F400ED010F009379093C
:10AB80008CE59CE00E9436348EE18093090D82E3CF
:10AB900080930A0D602F80E99CE00E94EA340E94B5
:10ABA000E64B8CE893E00E943634809106028230B6
:10ABB000C1F400ED010F009378098CE59CE00E9440
:10ABC000363482E38093090D80930A0D602F80E96B
:10ABD0009CE00E94EA340E94E64B8CE893E00E94DD
:10ABE0003634809106028330C1F400ED010F0093EA
:10ABF00077098CE59CE00E943634E092090D82E3EF
:10AC000080930A0D602F80E99CE00E94EA340E9444
:10AC1000E64B8CE893E00E94363480910602843043
:10AC200009F08DC01053109376098CE59CE00E94CA
:10AC300036342092090D82E380930A0D612F80E95A
:10AC40009CE00E94EA340E94E64B8CE893E00E946C
:10AC50003634F09206022091790990910502809194
:10AC6000690929131AC020917809909104022913C7
:10AC700014C0209177099091030229130EC02091EE
:10AC8000760990910202291308C0882319F00E94C6
:10AC9000D0323FCD0E94D82F3CCD882309F440C04C
:10ACA000809155098230C9F180E00E94303424E15E
:10ACB00040E56EE189E10E94564B0E94E64B81E03F
:10ACC0000E9430346091550911E0160F1093550918
:10ACD0001092110C1092140C61E873E088E09CE073
:10ACE0000E940F353092110C612F70E088E09CE0DB
:10ACF0000E941135F092140C68EE73E080E090E051
:10AD00000E94914D1092110C62E173E088E09CE08A
:10AD10000E940F35F0920602FCCC0E945732F9CC0B
:10AD200080E00E94303424E140E56EE189E10E9438
:10AD3000564B0E94E64B81E00E943034EACC8F5F94
:10AD400080930602E6CC0E94C94D2B013C01609322
:10AD500086097093870980938809909389090E94D6
:10AD6000C94D60935A0970935B0980935C09909375
:10AD70005D0980917E0990917F09A0918009B09131
:10AD80008109A3019201281B390B4A0B5B0BDA01E5
:10AD9000C901883E9340A105B10508F4E6C10E94AF
:10ADA000B12D80915009813061F480914E099091CC
:10ADB0004F09019690934F0980934E090E94622F8C
:10ADC0000DC0823059F480914C0990914D09019643
:10ADD00090934D0980934C090E949D2F8091860984
:10ADE00090918709A0918809B091890980937E0983
:10ADF00090937F09A0938009B09381090E94642EEB
:10AE000080914A0990914B092C01990F66087708A7
:10AE100080915A0990915B09A0915C09B0915D09FC
:10AE2000009146091091470920914809309149093C
:10AE3000BC01CD01601B710B820B930BA50194012A
:10AE40000E94DF67241535054605570508F48DC1B6
:10AE500060E070E08EE00E940D4B61E070E089E1FF
:10AE60000E940D4B0E94063520914C0930914D09EE
:10AE700080914E0990914F09821793070CF082C080
:10AE80008CE59CE00E94363445E853E063E284E1BF
:10AE90000E9429344EE853E062E38DE20E94293497
:10AEA0000E94E64B8CE893E00E9436344FE0642E1B
:10AEB000712CC12CD12C00E020E04FEFB60182EEC6
:10AEC0009BE00E94164720E04FEFB6018DEC9BE01F
:10AED0000E94164782EE9BE00E9467478DEC9BE044
:10AEE0000E9467476AE070E080E090E00E94914D28
:10AEF00020E040E0B60182EE9BE00E94164720E091
:10AF000040E0B6018DEC9BE00E94164782EE9BE08C
:10AF10000E9467478DEC9BE00E9467476AE070E003
:10AF200080E090E00E94914D4FEFC41AD40A58E09F
:10AF3000C516D10409F0BFCF81E0681A710809F085
:10AF4000B8CFC12CD12C00E020E04FEFB60182EE4B
:10AF50009BE00E94164720E04FEFB6018DEC9BE08E
:10AF60000E94164782EE9BE00E9467478DEC9BE0B3
:10AF70000E9467472FEFC21AD20A38E0C316D104E5
:10AF800011F78FC0281739070CF083C08CE59CE0BF
:10AF90000E94363444E953E063E284E10E9429349C
:10AFA0004EE853E062E38DE20E9429340E94E64BB2
:10AFB0008CE893E00E9436343FE0632E712CC12C64
:10AFC000D12C0FEF20E040E0B60182EE9BE00E9422
:10AFD000164720E040E0B6018DEC9BE00E9416474A
:10AFE00082EE9BE00E9467478DEC9BE00E946747E2
:10AFF0006AE070E080E090E00E94914D00E020E087
:10B0000040E0B60182EE9BE00E94164720E040E05F
:10B01000B6018DEC9BE00E94164782EE9BE00E94F9
:10B0200067478DEC9BE00E9467476AE070E080E034
:10B0300090E00E94914D4FEFC41AD40A58E0C51613
:10B04000D10409F0BECF81E0681A710809F0B7CFCA
:10B05000C12CD12C0FEF20E040E0B60182EE9BE046
:10B060000E94164720E040E0B6018DEC9BE00E9474
:10B07000164782EE9BE00E9467478DEC9BE00E94A2
:10B0800067472FEFC21AD20A38E0C316D10411F76E
:10B0900008C04EE953E064E084E00E9429340E9435
:10B0A000E64B60E177E280E090E00E94914D0E94E3
:10B0B00006354EE253E068E081E00E9429340E94A8
:10B0C000F1348CE59CE00E94363448E253E06EE1B6
:10B0D0008EE10E9429340E94E64B8CE893E00E94A6
:10B0E000363461E08AE10E94B34C82EE9BE00E941C
:10B0F000CC4682EE9BE00E9467478DEC9BE00E946D
:10B10000CC468DEC9BE00E9467471092500910924C
:10B110004D0910924C0910924F0910924E0910924D
:10B120004609109247091092480910924909109255
:10B130005A0910925B0910925C0910925D091092F5
:10B140007E0910927F091092800910928109109255
:10B150008609109287091092880910928909109225
:10B160006A090E94622F0E949D2F88E090E00E9451
:10B170005448811102C00E94B12D80910B0283308E
:10B1800009F0D0CA80916A09882309F4CBCA0E94C9
:10B19000C94D60935A0970935B0980935C09909341
:10B1A0005D090E94C94D6093860970938709809359
:10B1B0008809909389090E94C94D009182091091D4
:10B1C000830920918409309185092B013C01401AA3
:10B1D000510A620A730A930182010436110521059E
:10B1E000310540F06093820970938309809384094C
:10B1F0009093850920918209309183092C593F4F02
:10B20000C901861B970B90930802809307020E9446
:10B21000F43080916709882309F445C00E94C94D24
:10B220000E9431300E94C94D60937A0970937B0966
:10B2300080937C0990937D0900918A0910918B0974
:10B2400020918C0930918D092B013C01401A510A43
:10B25000620A730A2091620930E02F5F3F4F032E8C
:10B26000000C440B550BC501B4010E94DF67421668
:10B27000530664067506A8F064E071E08FE00E9452
:10B280000D4B80917A0990917B09A0917C09B09136
:10B290007D0980938A0990938B09A0938C09B093C0
:10B2A0008D090E94814940918609509187096091DA
:10B2B00088097091890980917E0990917F09A091F8
:10B2C0008009B09181092A013B01481A590A6A0A8A
:10B2D0007B0A2091550930E02F5F3F4F032E000C71
:10B2E000440B550BC501B4010E94DF67421653069B
:10B2F0006406750608F491C0809153099091540931
:10B30000019790935409809353098091670988238A
:10B3100049F08091510990915209019790935209F7
:10B32000809351090E9481490E94F4308091530911
:10B3300090915409892B31F480916709811102C0E1
:10B340000E9413498091510990915209892B11F45F
:10B350000E94A14880910902811104C0809167096F
:10B36000882311F18AE090E00E94544890E02091F7
:10B3700065093091660928173907B4F480918E0C5D
:10B3800080FF56C38091840C80FD65C351C3853016
:10B3900049F444E1C49E402D112424E168E28FE089
:10B3A0000E94564B0E94E64B80916709882329F141
:10B3B0008AE090E00E94544890E020916509309125
:10B3C00066092817390714F00E9413498091620911
:10B3D000863010F00E94A148909163098091620923
:10B3E000992331F08F5F809362091092630905C041
:10B3F000882319F081508093620980918609909189
:10B400008709A0918809B091890980937E0990935A
:10B410007F09A0938009B093810980916709811108
:10B4200081C98AE090E00E94544890E0209165092B
:10B43000309166092817390724F08091090281119B
:10B4400035C39091660C8091640990FF2AC08111E8
:10B4500084C390910902911180C361E08AE10E9446
:10B46000B34C0E94063548E553E068E080E00E9456
:10B4700029340E94F1348CE59CE00E94363447EE7A
:10B4800053E06EE185E00E9429340E94E64B8CE88F
:10B4900093E00E94363482E70E94692DF09264099D
:10B4A00041C9811129C359C383EA93E00E944B35F6
:10B4B000FFCF6AE080E090E00E9440480C949051F9
:10B4C00064E181E090E00E9440480C949C516AE065
:10B4D00082E090E00E9440480C94A8516FE083E025
:10B4E00090E00E9440480C94B65165E084E090E002
:10B4F0000E9440480C94C45165E085E090E00E94B1
:10B5000040480C94D05165E089E090E00E944048AA
:10B510000C94DC516FE086E090E00E9440480C946F
:10B52000EA5165E088E090E00E9440480C94F851B0
:10B5300065E087E090E00E9440480C94065265E088
:10B540008AE090E00E9440480C9412526FE08BE039
:10B5500090E00E9440480C94205265E08CE090E01E
:10B560000E9440480C942E5210910B02113009F0A9
:10B5700055C00E94063549E453E068E080E00E942F
:10B5800029340E94F1348CE59CE00E9436344AE76D
:10B5900053E06EE187E10E9429340E94E64B8CE87B
:10B5A00093E00E94363460E08AE10E94B34C87E663
:10B5B0000E94692D1092440910936A09109237096C
:10B5C000109238091092390910923A090E94C94D17
:10B5D00060934609709347098093480990934909FD
:10B5E00087E090E00E94544890E09093010280939D
:10B5F000000284E090E00E9454485CE3859FC00113
:10B600001124909336098093350983E090E00E94DD
:10B6100054482CE3829FC001112489C01230C1F527
:10B62000F0926A0960E08AE10E94B34C0E940635FC
:10B6300087E70E94692D0E94C94D60934609709367
:10B64000470980934809909349090E94C94D609326
:10B650005A0970935B0980935C0990935D090E947D
:10B66000C94D60937E0970937F0980938009909300
:10B67000810980913409882319F063E070E002C0E9
:10B6800062E070E087E10E940D4B0E94642E3CC88E
:10B69000133009F039C80E94063548E553E068E0E8
:10B6A00080E00E9429340E94F1348CE59CE00E94E5
:10B6B000363449E653E06EE183E20E9429340E9469
:10B6C000E64B8CE893E00E94363460E08AE10E9409
:10B6D000B34C87E60E94692D10926409F0926A09C2
:10B6E0000E94C94D609346097093470980934809A9
:10B6F0009093490987E090E00E94544890E090932D
:10B700000102809300028CE090E00E9454483CE3E8
:10B71000839FC001112490935209809351098BE0BB
:10B7200090E00E9454484CE3849FC0011124909300
:10B730005409809353090C948453F0923B098EEA88
:10B7400093E00E944B3508C010923B0983EC93E0D4
:10B750000E944B35109275090E94F42F97C8809172
:10B760003B09882309F4B2C889E090E00E9454485C
:10B7700090917509981748F480918E0C80FF6AC0EB
:10B780008091840C80FD72C065C00E94C94D4090BC
:10B790007109509072096090730970907409930157
:10B7A0008201005D1A482F4F3F4F061717072807E1
:10B7B000390708F491C045284628472809F48CC069
:10B7C0004FE653E06CE187E20E94293480E00E945A
:10B7D000303424E140E86EE180E00E94564B81E085
:10B7E0000E9430348CE59CE00E9436348EE18093D8
:10B7F000090D12E310930A0D6091050280E99CE0A7
:10B800000E94EA341093090D10930A0D609104020E
:10B8100080E99CE00E94EA34E092090D10930A0D41
:10B820006091030280E99CE00E94EA342092090DB5
:10B8300010930A0D6091020280E99CE00E94EA34B4
:10B840008CE893E00E9436340E94E64B81E00E942F
:10B8500030343CC81092750980E00E94303424E1F5
:10B8600040E867E380E00E94564BEECF8091690983
:10B87000811105C064E071E08FE00E940D4BD09013
:10B880007509D394D092750989E090E00E945448DC
:10B890008A3061F08F3099F08530D1F444E1D49E44
:10B8A000402D112424E167E38FE010C0DD0C4D2D05
:10B8B000440F440F4D0D24E167E38AE007C04D2D8E
:10B8C000440F4D0D440F24E167E384E10E94564B81
:10B8D0000E94E64B0C94665442D72AE0422E512C2B
:10B8E000612C712CA30192010E94B3676093050241
:10B8F00036D7A30192010E94B367609304022FD749
:10B90000A30192010E94B3676093030228D7A301A9
:10B9100092010E94B367609302020E94C94D609336
:10B92000710970937209809373099093740948CFD9
:10B9300064E071E08FE00E940D4BD0904509D394F4
:10B94000D092450985E090E00E9454488A3049F43D
:10B95000DD0C4D2D440F440F4D0D24E168E28AE0CB
:10B960003BC88F3009F02FC84D2D440F4D0D440FAB
:10B9700024E168E284E130C81092450980E00E9429
:10B98000303424E140E868E280E00E94564B0E9497
:10B99000E64B81E00E94303423C80E94D82F70C843
:10B9A00090917A0C90FFC7C8882309F4C4C880918D
:10B9B0000A028111C0C8F09269090E94063549E463
:10B9C00053E068E080E00E9429340E94F1348CE565
:10B9D0009CE00E94363440EE53E06EE18EE10E941E
:10B9E00029340E94E64B8CE893E00E94363460E0F4
:10B9F0008AE10E94B34C8CE60E94692D63E071E0FD
:10BA00008FE00E940D4B68E077E080E090E00E94BC
:10BA1000914D10926309109262090E94C94D8BC822
:10BA200048E753E06EE184E10E94293489E779C850
:10BA3000109266091092650980E00E94303424E17A
:10BA400040E868E280E00E94564B0E94E64B81E0AD
:10BA50000E943034A9CC64E071E08FE00E940D4B6D
:10BA6000C0906509D09066092FEFC21AD20AD09211
:10BA70006609C09265098AE090E00E9454488A30C5
:10BA800051F44C2D440F842F880F880F480F24E168
:10BA900068E28AE085CC8F3009F079CC4C2D440FD8
:10BAA0004C0D440F24E168E284E17ACC0E94063513
:10BAB00048E553E068E080E00E9429340E94F134B8
:10BAC0008CE59CE00E94363448E753E06EE189E063
:10BAD0000E9429340E94E64B8CE893E00E943634A1
:10BAE00089E70E94692D109209021092660910924E
:10BAF00065090E94E64BA5CC60E08AE10E94B34C48
:10BB00000E94063548E553E068E080E00E94293451
:10BB10000E94F1348CE59CE00E9436348091090249
:10BB2000882341F049E653E06EE183E20E94293424
:10BB300087E607C048E753E06EE189E00E942934B8
:10BB400089E70E94692D0E94E64B8CE893E00E94F1
:10BB50003634109264090C94925390917A0C90FDB3
:10BB600002C00C949253882311F40C949253809148
:10BB7000090281110C949253F09267090E940635D4
:10BB800048E553E068E080E00E9429340E94F134E7
:10BB90008CE59CE00E94363442EF53E06EE187E191
:10BBA0000E9429340E94E64B8CE893E00E943634D0
:10BBB00060E08AE10E94B34C8CE60E94692D61E04E
:10BBC00074E08FE00E940D4B68E077E080E090E049
:10BBD0000E94914D10926309109262090E94C94D12
:10BBE0000E94C94D60938A0970938B0980938C09D8
:10BBF00090938D090C94925381E00C94764F2BE630
:10BC000030E00C948E4F20E030E00C948E4F823365
:10BC100059F0833361F0843369F092EC980F9830D7
:10BC200060F492EC0C94974F88E00C949D4F84E064
:10BC30000C949D4F82E00C949D4F81E00C949D4F9D
:10BC4000E8E6F0E00C94654F1F93CF93DF93EC018F
:10BC5000162F19821F821E861F86188A198A81E074
:10BC60008D878A871B8692E09C87888388E190E095
:10BC70009D838C830E944D6999878887009751F036
:10BC800028E1FC0111922A95E9F788E090E09B8376
:10BC90008A8304C01D821C821B821A821E838981B2
:10BCA000882341F061E0812F0E94114D60E0812FD7
:10BCB0000E94B34C812F90E0FC01E350FE4BE491D5
:10BCC000F0E0EE0FFF1FED51FE4B259134913B8BC1
:10BCD0002A8BFC01ED5BFD4BE491EC8BDF91CF9166
:10BCE0001F910895CF93DF93EC01862F1B821A8258
:10BCF0002FE232E0398328836C834D8361E00E9418
:10BD0000114D61E08D810E94114D61E08C810E9496
:10BD1000B34C61E08D810E94B34C19868CE291E0B6
:10BD20009B878A871C8664E6CE010E94304640E4E9
:10BD30006D818C81DF91CF910C94CE4488E59BE09E
:10BD40000E9405438091D50B9091D60B0E94E56926
:10BD50008091D30B87FD03C060E00E94114D80915C
:10BD6000EA0B9091EB0B0E94E5698091E80B87FD4F
:10BD700003C060E00E94114D80EE92E09093400C71
:10BD800080933F0C80913209909133098F539C40EE
:10BD900071F4E091520CF091530C90818091540C0D
:10BDA0008095892380831092330910923209089577
:10BDB000CF930E94063542E455E068E080E00E949F
:10BDC00029340E94F13443E958E064E189E00E949B
:10BDD00029344AE958E06EE189E00E94293441EAB9
:10BDE00058E068E289E00E94293443EE54E06CE3B5
:10BDF00089E00E94293481E090E00E945448883212
:10BE000041F0803451F0843171F44FE356E064E145
:10BE100007C04FE356E06EE103C04FE356E068E22F
:10BE200080E00E9429340E94E64B0E945E35C82FB4
:10BE30008823D9F364E071E08FE00E940D4B0E94EB
:10BE40000635C13359F549EA58E063E288E20E94B9
:10BE500029340E94E64B64E182EE9BE00E94D546C5
:10BE600064E18DEC9BE00E94D54682EE9BE00E944F
:10BE700067478DEC9BE00E94674764E181E090E0BA
:10BE80000E9440486AE088E09CE00E9430466AE0F8
:10BE900087EF9BE00E9430466AE02CC0C233D9F5A0
:10BEA00044EB58E063E288E20E9429340E94E64BAA
:10BEB00068E282EE9BE00E94D54668E28DEC9BE052
:10BEC0000E94D54682EE9BE00E9467478DEC9BE086
:10BED0000E94674768E281E090E00E94404862E388
:10BEE00088E09CE00E94304662E387EF9BE00E947E
:10BEF000304662E382E090E00E94404868EE73E0E2
:10BF000080E090E00E94914D67EF74E088E59BE04F
:10BF1000CF910C94DB42C33359F54FEB58E063E209
:10BF200088E20E9429340E94E64B60E482EE9BE0A6
:10BF30000E94D54660E48DEC9BE00E94D54682EEDF
:10BF40009BE00E9467478DEC9BE00E94674760E49E
:10BF500081E090E00E94404864E688E09CE00E9416
:10BF6000304664E687EF9BE00E94304664E6C2CF2D
:10BF7000C33251F2CF910C94094ACF930E940635F7
:10BF800049E355E068E080E00E9429340E94F134E2
:10BF900046E857E064E189E00E9429344DE857E023
:10BFA0006EE189E00E94293444E957E068E289E0C3
:10BFB0000E9429344BE957E062E389E00E9429346A
:10BFC00043EE54E06CE389E00E94293480E090E085
:10BFD0000E9454488A3079F030F4811116C04FE342
:10BFE00056E064E10FC0843151F08E3171F44FE3BB
:10BFF00056E062E307C04FE356E06EE103C04FE353
:10C0000056E068E280E00E9429340E94E64B0E94DC
:10C010005E35C82F8823D9F364E071E08FE00E9479
:10C020000D4B0E940635C13379F44BEC58E063E2C6
:10C030008EE10E9429340E94E64B60E070E086E0C9
:10C040000E940D4B60E010C0C233F9F447ED58E098
:10C0500063E28EE10E9429340E94E64B6AE070E0C0
:10C0600086E00E940D4B6AE080E090E00E9440482C
:10C0700068EE73E080E090E00E94914D67EF74E01D
:10C0800088E59BE0CF910C94DB42C33379F443EE17
:10C0900058E063E28EE10E9429340E94E64B64E19D
:10C0A00070E086E00E940D4B64E1DECFC43379F48A
:10C0B0004FEE58E063E28EE10E9429340E94E64B85
:10C0C0006EE170E086E00E940D4B6EE1CDCFC33291
:10C0D000A9F2CF910C94094ACF930E94063545ED01
:10C0E00056E068E080E00E9429340E94F1344CEF71
:10C0F00058E064E189E00E94293447E059E06EE1AC
:10C1000089E00E94293444E159E068E289E00E9414
:10C11000293442E259E062E389E00E94293443EE87
:10C1200054E06CE389E00E94293488E090E00E94AA
:10C130005448853079F030F4811116C04FE356E051
:10C1400064E10FC08A3051F08F3071F44FE356E054
:10C1500062E307C04FE356E06EE103C04FE356E0F1
:10C1600068E280E00E9429340E94E64B0E945E351E
:10C17000C82F8823D9F364E071E08FE00E940D4B53
:10C180000E940635C13351F44FEF58E063E288E274
:10C190000E9429340E94E64B60E00BC0C233D1F408
:10C1A0004AE059E063E288E20E9429340E94E64BAB
:10C1B00065E088E090E00E94404868EE73E080E02F
:10C1C00090E00E94914D67E175E088E59BE0CF919A
:10C1D0000C94DB42C33351F447E159E063E288E257
:10C1E0000E9429340E94E64B6AE0E3CFC43351F445
:10C1F00045E259E063E288E20E9429340E94E64B5E
:10C200006FE0D7CFC332F9F2CF910C94094ACF93A4
:10C21000DF931092B20A1092B10A88EE93E0A0E088
:10C22000B0E08093B30A9093B40AA093B50AB09398
:10C23000B60A22EB32E03093B00A2093AF0A25EC25
:10C2400030E03093BC0A2093BB0A24EC30E03093FA
:10C25000BE0A2093BD0A20EC30E03093C00A209340
:10C26000BF0A21EC30E03093C20A2093C10A22ECCD
:10C2700030E03093C40A2093C30A26EC30E03093B8
:10C28000C60A2093C50A1092C80A1092C90A1092D1
:10C29000CA0A1092CB0A10924F0B10924E0B809349
:10C2A000500B9093510BA093520BB093530B84EC13
:10C2B00092E090934D0B80934C0B88E680930B0D8E
:10C2C0001092930C1092920C8FEF90E49093080DC3
:10C2D0008093070D1092090D10920A0D1092A90C6F
:10C2E0008AEF92E09093910C8093900C1092950CB1
:10C2F0001092940C1092A50C1092A80C8FEF8093C2
:10C30000A60C8093AB0CEFEAFCE085EC9CE02FEFF1
:10C31000DFEF21938E179F07D9F785E490E4909380
:10C32000990C8093980C8DE392E490939B0C8093EE
:10C330009A0C83EA99E390939D0C80939C0C88ED72
:10C3400099E390939F0C80939E0C20E030E040E0B6
:10C3500069E084E99CE00E9445401092D90C10925B
:10C36000D80C84EB91E49093C60C8093C50C8AE1C1
:10C370009DE09093CA0C8093C90C88E08093CB0C0D
:10C380001092CC0C1092E50C1092040DC1E0C093F9
:10C39000050DC093060D8EE093E09093C80C80933A
:10C3A000C70C84E99CE00E94684180E192E490938C
:10C3B000DB0C8093DA0C1092E80CD093BA0CD0937B
:10C3C000BB0CD093BC0C22EF32E03093870C20934F
:10C3D000860C1092880C1092890C10928A0C109284
:10C3E0008B0C8AE090E090938D0C80938C0C1092D3
:10C3F0008E0C10928F0C30937D0C20937C0C10923D
:10C400007E0C10927F0C1092800C1092810C9093F5
:10C41000830C8093820C1092840C1092850C3093C4
:10C42000730C2093720C1092740C1092750C109275
:10C43000760C1092770C9093790C8093780C109274
:10C440007A0C10927B0C3093690C2093680C10923C
:10C450006A0C10926B0C10926C0C10926D0C9093F5
:10C460006F0C80936E0C1092700C1092710C3093C4
:10C470005F0C20935E0C1092600C1092610C109275
:10C48000620C1092630C9093650C8093640C109274
:10C49000660C1092670C1092420C1092410C88EEC0
:10C4A00093E0A0E0B0E08093430C9093440CA09301
:10C4B000450CB093460C80EE92E09093400C809334
:10C4C0003F0C1092560C1092550C1092580C109272
:10C4D000570C10925A0C1092590C10925C0C10923E
:10C4E0005B0C80915D0C8E7F8D7F80935D0C8695BB
:10C4F0008170682F6C278DE00E94B34C61E08DE065
:10C500000E94114DE0E5F2E4E491E0934F0CEAE083
:10C51000F2E4E491F0E0EE0FFF1FED51FE4B859148
:10C5200094919093510C8093500C60E08CE00E94A9
:10C53000114D80915D0C81FD04C061E08CE00E9492
:10C54000B34C8CE080934B0CEFE4F2E4E491E09385
:10C550004C0CE9E0F2E4E491F0E0EE0FFF1FE7534A
:10C56000FE4B8591949190934E0C80934D0C84EFEB
:10C5700091E0A0E0B0E080931F0C9093200CA0937A
:10C58000210CB093220C8AE0E4EAF2E0ADE2BCE0D8
:10C5900001900D928A95E1F71092370C82E080931A
:10C5A000380C10923D0C10923E0C4EE260E388E095
:10C5B0009CE098DB4EE36FE387EF9BE093DB6AE25E
:10C5C00082EE9BE041DB60E48DEC9BE03DDB109272
:10C5D000600B1092640B1092630B1092650B86ED4A
:10C5E00092E090935F0B80935E0BEEE5FBE0148E80
:10C5F00010A2178E11A236968BE0EA39F807B9F728
:10C6000081E192E09093C10B8093C00B8EE092E0A9
:10C610009093C30B8093C20B84E08093C40B83E0A0
:10C620008093C50B85E192E09093BF0B8093BE0B86
:10C630008AE090E09093C70B8093C60B84EF91E063
:10C640009093C90B8093C80B1092CC0B1092CB0B1C
:10C650001092BA0B1092BB0B1092BC0B1092BD0B38
:10C660001092CA0B1092590B1092580B10925B0B40
:10C6700010925A0B10925D0B10925C0B44E050E04C
:10C6800069EF73E088E59BE0DF91CF910C94BC42A9
:10C69000EF920F931F93CF93DF93E80147FD02C002
:10C6A00034E001C034E1042E000C550B57FF03C0E9
:10C6B000519541955109E32E022F242FAE01C6D08A
:10C6C000CE01DF91CF911F910F91EF9008958F923E
:10C6D0009F92AF92BF92CF92DF92EF92FF92CF9351
:10C6E000DF93EC01688179818A819B8161157105F5
:10C6F0008105910521F464E279ED8BE597E02DE168
:10C7000033EF41E050E02FD449015A019B01AC01C5
:10C71000A7EAB1E444D46B017C01ACEEB4EFA5010F
:10C72000940149D4DC01CB018C0D9D1DAE1DBF1DB4
:10C73000B7FF03C00197A109B04888839983AA83F2
:10C74000BB83BC01CD019F77DF91CF91FF90EF902C
:10C75000DF90CF90BF90AF909F908F9008958F9271
:10C760009F92AF92BF92CF92DF92EF92FF92609131
:10C77000210270912202809123029091240261157E
:10C7800071058105910521F464E279ED8BE597E06F
:10C790002DE133EF41E050E0E6D349015A019B011E
:10C7A000AC01A7EAB1E4FBD36B017C01ACEEB4EFC2
:10C7B000A501940100D4DC01CB018C0D9D1DAE1DA3
:10C7C000BF1DB7FF03C00197A109B04880932102A4
:10C7D00090932202A0932302B0932402BC01CD01C6
:10C7E0009F77FF90EF90DF90CF90BF90AF909F909A
:10C7F0008F90089560932102709322028093230208
:10C80000909324020895BB274A3031F4992322F4EF
:10C81000BDE2909581959F4F01C0BB27FB01552735
:10C82000AA27880F991FAA1FA41710F0A41B83958D
:10C830005051B9F7A05DAA3308F0A95DA193009704
:10C8400079F7B111B1931192CB014EC28F929F92A1
:10C85000AF92BF92CF92DF92EF92FF920F931F930E
:10C86000CF93DF93CDB7DEB729970FB6F894DEBF2D
:10C870000FBECDBF6A01122FB02E2BE3201720F080
:10C88000FF24F394F00E02C02CE3F22E0F2D27E0CC
:10C89000AE014F5F5F4F50D1BC014981842F897039
:10C8A000813031F0E1FC06C0E0FE06C090E205C038
:10C8B0009DE203C09BE201C090E05E2D507143FFFA
:10C8C0003CC0911102C083E001C084E0811718F4DC
:10C8D000212F281B01C020E051110BC0F601822F2F
:10C8E00030E2882319F031938150FBCFC20ED11C66
:10C8F00020E0992329F0D6019C93F60131966F012F
:10C90000C6010396E2FE0AC03EE4D6013C9341E430
:10C9100011964C93119712963C9306C03EE6F60191
:10C92000308341E641833283FC01322F40E23323DE
:10C9300009F442C041933150FACF42FF44C09111F3
:10C9400002C083E001C084E0811718F4212F281B66
:10C9500001C020E051110BC0F601822F30E2882384
:10C9600019F031938150FBCFC20ED11C20E09923E6
:10C9700029F0D6019C93F60131966F01C60103960A
:10C98000E2FE0BC039E4D6013C933EE411963C93A1
:10C99000119736E412963C9307C039E6F6013083CE
:10C9A0003EE6318336E63283FC01322F40E2332308
:10C9B00019F041933150FBCFFC01E20FF11D1082C1
:10C9C0008EEF9FEFA6C021E030E0911102C020E081
:10C9D00030E0161617061CF4FB01319602C0E1E0A8
:10C9E000F0E02E0F3F1FBB2021F0EB2DF0E0319641
:10C9F00002C0E0E0F0E02E0F3F1FE12FF0E02E1725
:10CA00003F071CF4121B212F01C020E08E2D8871DE
:10CA100059F4F601822F30E2882319F031938150C6
:10CA2000FBCFC20ED11C20E0992329F0D6019C93A4
:10CA3000F60131966F0151110BC0F601822F90E380
:10CA4000882319F091938150FBCFC20ED11C20E0B6
:10CA50000F2D060F9A81342F307144FF03C091339C
:10CA600009F40150101624F4093018F008E001C050
:10CA700001E0AB0177FF02C040E050E0FB01E41BA6
:10CA8000F50BA1E0B0E0AC0FBD1FEA0FFB1F8EE27B
:10CA9000A82E4B01801A91080B2D10E011950195DD
:10CAA00011094F3FBFEF5B0721F4D601AC921196FD
:10CAB0006D01641775072CF08416950614F48181B6
:10CAC00001C080E3415051093196D60111967D0194
:10CAD0004017510724F0D6018C936701E2CF641709
:10CAE000750739F4963320F4953319F4311101C0E8
:10CAF00081E3F6018083F701822F90E2882319F009
:10CB000091938150FBCFF701E20FF11D108280E07D
:10CB100090E029960FB6F894DEBF0FBECDBFDF912F
:10CB2000CF911F910F91FF90EF90DF90CF90BF902A
:10CB3000AF909F908F900895283008F027E033271A
:10CB4000DA01990F311D87FD91600096610571052D
:10CB500039F432602E5F3D9330E32A95E1F7089572
:10CB60009F3F30F080387105610509F03C5F3C5F04
:10CB70003D93913008F08068911DDF93CF931F9310
:10CB80000F93FF92EF92192F987F9695E92F969524
:10CB90009695E90FFF27E257FE4F99273327EE249A
:10CBA000FF24A701E70105900894079428F4360FA5
:10CBB000E71EF81E491F511D660F771F881F991F1A
:10CBC0000694A1F70590079428F4E70EF81E491F74
:10CBD000561FC11D770F881F991F661F0694A1F766
:10CBE0000590079428F4F80E491F561FC71FD11D42
:10CBF000880F991F661F771F0694A1F70590079469
:10CC000020F4490F561FC71FD81F990F661F771FA3
:10CC1000881F0694A9F784911095177041F0D69556
:10CC2000C79557954795F794E7941A95C1F7E4E3AC
:10CC3000F1E0689415901591359165919591059065
:10CC40007FE27395E118F10A430B560BC90BD0092B
:10CC5000C0F7E10CF11E431F561FC91FD01D7EF403
:10CC6000703311F48A95E6CFE894015030F0080F44
:10CC70000AF40027021708F4202F2395022F7A3395
:10CC800028F079E37D932A95E9F710C07D932A95E2
:10CC900089F6069497956795379517951794E11837
:10CCA000F10A430B560BC90BD00998F023957E91DE
:10CCB00073957A3308F070E37C932013B8F77E9174
:10CCC00070617D9330F0839571E37D9370E32A95D5
:10CCD000E1F71124EF90FF900F911F91CF91DF9119
:10CCE000992787FD90950895DC01FC01672F7191CC
:10CCF0007723E1F7329704C07C916D937083629142
:10CD0000AE17BF07C8F3089540D008F481E0089536
:10CD1000E89409C097FB3EF49095809570956195D5
:10CD20007F4F8F4F9F4F9923A9F0F92F96E9BB278B
:10CD30009395F695879577956795B795F111F8CF07
:10CD4000FAF4BB0F11F460FF1BC06F5F7F4F8F4F72
:10CD50009F4F16C0882311F096E911C0772321F068
:10CD60009EE8872F762F05C0662371F096E8862F00
:10CD700070E060E02AF09A95660F771F881FDAF757
:10CD8000880F9695879597F90895990F0008550F84
:10CD9000AA0BE0E8FEEF16161706E807F907C0F041
:10CDA00012161306E407F50798F0621B730B840B49
:10CDB000950B39F40A2661F0232B242B252B21F423
:10CDC00008950A2609F4A140A6958FEF811D811DC3
:10CDD00008950BD078C069D028F06ED018F0952354
:10CDE00009F05AC05FC01124A2C07ED0A0F3959F65
:10CDF000D1F3950F50E0551F629FF001729FBB2742
:10CE0000F00DB11D639FAA27F00DB11DAA1F649FED
:10CE10006627B00DA11D661F829F2227B00DA11DA0
:10CE2000621F739FB00DA11D621F839FA00D611D26
:10CE3000221F749F3327A00D611D231F849F600D47
:10CE4000211D822F762F6A2F11249F5750408AF080
:10CE5000E1F088234AF0EE0FFF1FBB1F661F771F0C
:10CE6000881F91505040A9F79E3F510570F014C0A3
:10CE70005EC05F3FECF3983EDCF38695779567954F
:10CE8000B795F795E7959F5FC1F7FE2B880F911D2A
:10CE90009695879597F9089597F99F6780E870E0D0
:10CEA00060E008959FEF80EC089500240A94161620
:10CEB000170618060906089500240A941216130688
:10CEC000140605060895092E0394000C11F4882316
:10CED00052F0BB0F40F4BF2B11F460FF04C06F5F32
:10CEE0007F4F8F4F9F4F089557FD9058440F551F08
:10CEF00059F05F3F71F04795880F97FB991F61F0DC
:10CF00009F3F79F087950895121613061406551F52
:10CF1000F2CF4695F1DF08C0161617061806991FBE
:10CF2000F1CF86957105610508940895E894BB27B3
:10CF300066277727CB0197F90895F999FECF92BD1F
:10CF400081BDF89A992780B50895262FF999FECFCB
:10CF50001FBA92BD81BD20BD0FB6F894FA9AF99A16
:10CF60000FBE01960895052E97FB16F400940FD07E
:10CF700057FD05D024D007FC02D046F408C05095D8
:10CF80004095309521953F4F4F4F5F4F08959095B5
:10CF90008095709561957F4F8F4F9F4F089531D049
:10CFA000A59F900DB49F900DA49F800D911D1124FD
:10CFB0000895B7FFF4CFF3DF821B930B0895A1E22E
:10CFC0001A2EAA1BBB1BFD010DC0AA1FBB1FEE1F03
:10CFD000FF1FA217B307E407F50720F0A21BB30B4E
:10CFE000E40BF50B661F771F881F991F1A9469F7CA
:10CFF00060957095809590959B01AC01BD01CF0126
:10D000000895A29FB001B39FC001A39F700D811D21
:10D010001124911DB29F700D811D1124911D089541
:10D020005058BB27AA270ED04ECF3FDF30F044DF49
:10D0300020F031F49F3F11F41EF434CF0EF4E0954C
:10D04000E7FB2ACFE92F50DF80F3BA176207730797
:10D050008407950718F071F49EF568CF0EF4E095FB
:10D060000B2EBA2FA02D0B01B90190010C01CA01A2
:10D07000A0011124FF27591B99F0593F50F4503E4D
:10D0800068F11A16F040A22F232F342F4427585F3F
:10D09000F3CF469537952795A795F0405395C9F757
:10D0A0007EF41F16BA0B620B730B840BBAF091500F
:10D0B000A1F0FF0FBB1F661F771F881FC2F70EC0AE
:10D0C000BA0F621F731F841F48F487957795679581
:10D0D000B795F7959E3F08F0B3CF9395880F08F06A
:10D0E0009927EE0F9795879508950CD0ECCEE4DE46
:10D0F00040F0DBDE30F021F45F3F19F0CDCE51116E
:10D1000016CFD0CEF1DE98F39923C9F35523B1F3AE
:10D11000951B550BBB27AA2762177307840738F0A6
:10D120009F5F5F4F220F331F441FAA1FA9F333D005
:10D130000E2E3AF0E0E830D091505040E695001CB9
:10D14000CAF729D0FE2F27D0660F771F881FBB1F75
:10D15000261737074807AB07B0E809F0BB0B802D4F
:10D16000BF01FF2793585F4F2AF09E3F510568F09B
:10D1700093CEDDCE5F3FECF3983EDCF3869577955A
:10D180006795B795F7959F5FC9F7880F911D96959D
:10D19000879597F90895E1E0660F771F881FBB1FF9
:10D1A000621773078407BA0720F0621B730B840BA6
:10D1B000BA0BEE1F88F7E095089504D06894B1117A
:10D1C000B6CE089599DE88F09F5790F0B92F992731
:10D1D000B751A0F0D1F0660F771F881F991F1AF082
:10D1E000BA95C9F712C0B13081F0A0DEB1E0089560
:10D1F0009DCE672F782F8827B85F39F0B93FCCF3E1
:10D20000869577956795B395D9F73EF49095809577
:10D21000709561957F4F8F4F9F4F0895B6DD08F44D
:10D220008FEF0895991B79E004C0991F961708F0B5
:10D23000961B881F7A95C9F780950895AA1BBB1B7A
:10D2400051E107C0AA1FBB1FA617B70710F0A61B06
:10D25000B70B881F991F5A95A9F780959095BC0127
:10D26000CD01089597FB072E16F4009406D077FDA4
:10D2700008D0E4DF07FC05D03EF4909581959F4FE0
:10D280000895709561957F4F0895EE0FFF1F881FD9
:10D290008BBF0790F691E02D19940F931F93CF93B6
:10D2A000DF938230910510F482E090E0E0912B1141
:10D2B000F0912C1120E030E0A0E0B0E0309719F1BF
:10D2C000408151810281138148175907C8F08417A2
:10D2D000950769F4109731F012960C9312971396F4
:10D2E0001C9327C000932B1110932C1122C02115E1
:10D2F000310519F04217530718F49A01BD01EF01E7
:10D30000DF01F801DBCF21153105F9F0281B390BBE
:10D310002430310580F48A819B816115710521F0EB
:10D32000FB019383828304C090932C1180932B1173
:10D33000FE01329644C0FE01E20FF31F81939193E8
:10D3400022503109398328833AC020912911309124
:10D350002A11232B41F42091270230912802309387
:10D360002A1120932911209125023091260221159E
:10D37000310541F42DB73EB74091290250912A0260
:10D38000241B350BE0912911F0912A11E217F307C4
:10D39000A0F42E1B3F0B2817390778F0AC014E5F25
:10D3A0005F4F2417350748F04E0F5F1F50932A1127
:10D3B000409329118193919302C0E0E0F0E0CF0106
:10D3C000DF91CF911F910F910895CF93DF93009735
:10D3D00009F481C0FC01329713821282A0912B11B3
:10D3E000B0912C11109781F420813181820F931F0D
:10D3F0002091291130912A112817390751F5F093FE
:10D400002A11E093291167C0ED0120E030E0CE172A
:10D41000DF0740F44A815B819E0141155105F1F01F
:10D42000EA01F5CFD383C28340815181840F951FD8
:10D43000C817D90759F488819981840F951F0296DE
:10D44000918380838A819B81938382832115310517
:10D4500029F4F0932C11E0932B113DC0E901FB83DB
:10D46000EA8349915991C40FD51FEC17FD0761F468
:10D4700080819181840F951F0296E90199838883A9
:10D48000828193819B838A83E0E0F0E012968D9104
:10D490009C911397009719F0FD01DC01F7CF8D9156
:10D4A0009C9111979D012E5F3F4F820F931F2091FA
:10D4B000291130912A112817390769F4309729F476
:10D4C00010922C1110922B1102C013821282B09371
:10D4D0002A11A0932911DF91CF9108956F927F9225
:10D4E0008F929F92AF92BF92CF92DF92EF92FF9274
:10D4F0000F931F93CF93DF93009781F4CB01DF91BC
:10D50000CF911F910F91FF90EF90DF90CF90BF9040
:10D51000AF909F908F907F906F90BFCEFC01E60FF1
:10D52000F71F9C0122503109E217F30708F4A5C048
:10D53000EC01D9010D911C91119706171707A8F05E
:10D540000530110508F497C0C8010497861797079E
:10D5500008F491C002501109061B170B0193119397
:10D560006D937C93CF0131DF86C05B01A01AB10AB5
:10D570004C01800E911EA0912B11B0912C11612CA9
:10D58000712CE12CF12C109709F446C08D919C91DF
:10D590001197A815B905B1F56C0142E0C40ED11C74
:10D5A000CA14DB0478F14C018A189B08640142E03C
:10D5B000C40ED11C1296BC9012971396AC91B5E094
:10D5C000CB16D10440F0B282A38391828082D9012C
:10D5D0006D937C9309C00E5F1F4F800F911FF9015F
:10D5E00091838083EB2DFA2FE114F10431F0D70100
:10D5F0001396FC93EE9312973EC0F0932C11E09398
:10D600002B1139C06816790608F43C017D01129689
:10D610000D90BC91A02DB7CF8091291190912A1126
:10D6200088169906E1F466167706C8F480912502FB
:10D6300090912602009741F48DB79EB74091290240
:10D6400050912A02841B950BE817F907B0F4F09368
:10D650002A11E0932911F901718360830CC0CB0179
:10D660001CDE7C01009749F0A801BE011BD0CE0151
:10D67000ACDEC70104C0CE0102C080E090E0DF91C3
:10D68000CF911F910F91FF90EF90DF90CF90BF90BF
:10D69000AF909F908F907F906F90089581E090E081
:10D6A000F8942BC0FB01DC0102C001900D924150A7
:10D6B0005040D8F70895DC0101C06D9341505040AF
:10D6C000E0F70895FC018191861721F08823D9F7AE
:10D6D000992708953197CF010895FB01DC018D91C1
:10D6E000019080190110D9F3990B0895FB01DC0119
:10D6F00001900D920020E1F7089511E2C6E7D1E212
:10D7000000E005C0802FFE01C0DD2196011DC73756
:0CD71000D10780E00807B1F7F894FFCFC4
:10D71C0003000101010101640001010101013B3D14
:10D72C00393C37383A3132333435363738392A3098
:10D73C00230100000000002D11800000000000DA21
:10D74C00459D45382C372C1815A015C019FF1815F8
:10D75C00A115C819FF1815AE19FF1815AF19FF1828
:10D76C0015AE15D5168015A8163F15D31600154005
:10D77C00158D16141520160015A115C815DA1612DC
:10D78C00158116CF15D916F115DB1640152E15A4DB
:10D79C0015A619FF0001140A6464323200093D0019
:10D7AC0003042896100802028000400088898A8BA6
:10D7BC008C8D8E8F7EFF06000100000000EF0000B4
:10D7CC000000193F873EB13E653FE23EC03ED43E6D
:10D7DC00000000001C39F038382CC438E838D43834
:10D7EC00C53800000000BF44B844CC440000000021
:10D7FC001044873E382CC43860447744F84300000A
:10D80C000000C344BB4400000000D62C0F2C382C65
:10D81C00372C000000001242873E382C372C684110
:10D82C0009412D2D2D2D00426F6F6D20426F780018
:10D83C0076312E3036002500524541445900446F54
:10D84C006D696E6174696F6E204D6F646500566909
:10D85C00727573204D6F646500426F6D6220537456
:10D86C00617475733A20200043617073756C652088
:10D87C00506F7765723A2020004D41494E5300435A
:10D88C006F6D706C65746500554E4C4F434B454441
:10D89C000045727200526564205465616D005769D1
:10D8AC006E732100426C7565205465616D0054499E
:10D8BC004521007768696C65207472756500626F2C
:10D8CC006D624465636F64696E67466C6167207353
:10D8DC00657400626F6D624465636F64696E674660
:10D8EC006C616720756E7365740041524D45440040
:10D8FC0041435449564500534146455459204F46DF
:10D90C0046004241434B5550006D61696E004D61BC
:10D91C00696E204D656E7500312920426F6D620075
:10D92C00322920446F6D696E6174696F6E00332902
:10D93C002056697275730023292053657474696EBF
:10D94C00677300626F6D626D6F64650073657474EC
:10D95C00696E6773004D6172676172697461204D05
:10D96C006F6465004143544956415445442100318C
:10D97C00292050494E00322920486F6C640033290D
:10D98C00204465636F6465002329204261636B004A
:10D99C0050494E204D6F64650053657420626F6D65
:10D9AC00622061636365737300636F64653A00435F
:10D9BC006F64652041636365707465643A00486FF9
:10D9CC006C64204D6F646500646F6D696E61746981
:10D9DC006F6E0076697275730031292047616D6531
:10D9EC00204F7074696F6E730032292053797374F1
:10D9FC00656D00232920457869740067616D656F3A
:10DA0C007074696F6E730073797374656D0031296E
:10DA1C0020426F6D62204D6F646500626F6D626FA6
:10DA2C007074696F6E7300646F6D696E6174696F89
:10DA3C006E6F7074696F6E730076697275736F7048
:10DA4C0074696F6E7300312920566F6C756D6500AB
:10DA5C003229204272696768746E657373003329CA
:10DA6C0020416363656C65726F6D6574657200341B
:10DA7C002920426174742E2053746174757300767E
:10DA8C006F6C756D65006272696768746E6573732F
:10DA9C0000616363656C6F7074696F6E73006261B3
:10DAAC00747473746174757300426F6D62204F707F
:10DABC0074696F6E730031292047616D6520436C6A
:10DACC006F636B00322920426F6D6220436C6F6371
:10DADC006B00332920486F6C64204C656E6774684A
:10DAEC00003429204465636F64652054696D6500BA
:10DAFC00626F6D6267616D65636C6F636B00626F03
:10DB0C006D62626F6D62636C6F636B00626F6D62EE
:10DB1C00686F6C6400626F6D626465636F646574DA
:10DB2C00696D650031292035206D696E73003229CD
:10DB3C00203135206D696E73003329203330206D10
:10DB4C00696E73003429203630206D696E73003E87
:10DB5C00003135206D696E75746573003330206D3E
:10DB6C00696E75746573003630206D696E757465F9
:10DB7C00730031292031206D696E00322920352047
:10DB8C006D696E73003329203130206D696E73001E
:10DB9C003429203135206D696E730031206D696E2A
:10DBAC00757465003130206D696E75746573003164
:10DBBC00292035207365637300322920313020739E
:10DBCC00656373003329203135207365637300441A
:10DBDC006F6D696E6174696F6E204F7074696F6ED2
:10DBEC007300322920486F6C642054696D650064A1
:10DBFC006F6D696E6174696F6E67616D65636C6F73
:10DC0C00636B00646F6D696E6174696F6E686F6CC5
:10DC1C006474696D65005669727573204F70746910
:10DC2C006F6E7300322920566972757320436C6FC6
:10DC3C00636B00766972757367616D65636C6F6396
:10DC4C006B0076697275737669727573636C6F634A
:10DC5C006B007669727573686F6C64004163636501
:10DC6C006C204F7074696F6E730031292053656E90
:10DC7C00736974697669747900616363656C736543
:10DC8C006E736974697669747900416363656C209D
:10DC9C006C6576656C003129204F66660032292050
:10DCAC004C6F77003329204D656400342920486976
:10DCBC00676800416363656C3A204F666600416398
:10DCCC0063656C3A204C6F7700416363656C3A2056
:10DCDC004D656400416363656C3A20486967680070
:10DCEC00616363656C63616C6962726174696F6EA8
:10DCFC000043616C6962726174696E672E2E2E002E
:10DD0C00446F206E6F74206D6F7665206465766944
:10DD1C00636500560054696D652052656D61696ECE
:10DD2C00696E673A005365744465636F6465536349
:10DD3C007265656E004465636F64696E670041636C
:10DD4C006365737320436F64650052656365697620
:10DD5C00696E67204F5450004641494C005465721F
:10DD6C00726F72697374730057696E210053414668
:10DD7C004500436F756E746572000D0A0053616D3A
:10DD8C00706C650044657374726F796564004F62E2
:10DD9C007461696E656400496E76616C6964206BB0
:10DDAC006579003129204C6F77003229204D65644C
:10DDBC000033292048696768004C696768743A2009
:10DDCC004C6F77004C696768743A204D6564004C61
:10DDDC00696768743A204869676800566F6C756D9E
:10DDEC00653A204F666600566F6C756D653A204C2F
:10DDFC006F7700566F6C756D653A204D65640056F3
:10DE0C006F6C756D653A2048696768003129204947
:10DE1C006E7374616E740032292035207365636FE4
:10DE2C006E6473003329203130207365636F6E6428
:10DE3C0073003429203135207365636F6E64730071
:00000001FF
